:020000040800F2
:20300000F82A0020013100088B1E010885C90008891D0108014B0008E960010800000000D7
:20302000000000000000000000000000DF390108AD6E000800000000ED21010831490108B2
:203040001B3100081B3100081B3100081B3100081B3100081B3100081B3100081B310008D0
:20306000A97400081B3100081B310008495C00081B3100081B3100081B3100081B31000886
:203080001B3100081B310008C14200081B310008295A0108054B00081B3100081B3100089D
:2030A0001B3100085D4A01081B3100081B3100081B3100081B3100081B3100081B31000814
:2030C0001B3100081B3100081B3100081B3100081B3100081B3100081B3100083D59010805
:2030E0009D7400081B3100081B310008DFF80CD001F096F8004800479D420008F82A002025
:203100000648804706480047FEE7FEE7FEE7FEE7FEE7FEE7FEE7FEE7FEE7FEE7054A0108BB
:20312000ED3000082DE9FF1F002000210022002300240025002600275FF000085FF000096B
:203140005FF0000A5FF0000B5FF0000C002001210222032304240525062607275FF00808CA
:203160005FF009095FF00A0A5FF00B0B5FF00C0C00281DD101291BD1022A19D1032B17D167
:20318000042C15D1052D13D1062E11D1072F0FD1B8F1080F0CD1B9F1090F09D1BAF10A0FDA
:2031A00006D1BBF10B0F03D1BCF10C0F00D101E004F08ABCBDE8FF1F7047000073B4002029
:2031C00000210124002501262046A04226D1A94224D12846A84221D1A9421FD14FEA440498
:2031E00006F10106202EEFDD5FF0FF305FF0FF317FF000445FF0FF3501262046A0420DD137
:20320000A9420BD12846A84208D1A94206D14FEA740406F10106202EEFDD01E004F054BC46
:2032200073BC7047E7B40021002000220125002601272946A94230D1B0422ED1B2422CD1F9
:203240003146B14229D1B04227D1B24225D14FEA450507F10107202FEBDD5FF0FF315FF0CE
:20326000FF305FF0FF327FF000455FF0FF3601272946A94211D1B0420FD1B2420DD13146E8
:20328000B1420AD1B04208D1B24206D14FEA750507F10107202FEBDD01E004F015BCE7BCB7
:2032A00070472DE9CE01002200210023012600275FF001083246B24233D1B94231D1BB42FC
:2032C0002FD13A46BA422CD1B9422AD1BB4228D14FEA460608F10108B8F1200FEADD5FF014
:2032E000FF325FF0FF315FF0FF337FF000465FF0FF375FF001083246B24212D1B94210D1E0
:20330000BB420ED13A46BA420BD1B94209D1BB4207D14FEA760608F10108B8F1200FEADD79
:2033200001E004F0D1BBBDE8CE0170472DE99C0300230022002401275FF000085FF001090B
:203340003B46BB4233D1424531D144452FD1434643452CD142452AD1444528D14FEA470740
:2033600009F10109B9F1200FEADD5FF0FF335FF0FF325FF0FF347FF000475FF0FF385FF09B
:2033800001093B46BB4212D1424510D144450ED1434643450BD1424509D1444507D14FEA0A
:2033A000770709F10109B9F1200FEADD01E004F08BBBBDE89C0370472DE9381C0024002324
:2033C00000255FF0010A5FF0000B5FF0010C5446544533D15B4531D15D452FD15C465C45FA
:2033E0002CD15B452AD15D4528D14FEA4A0A0CF1010CBCF1200FEADD5FF0FF345FF0FF335D
:203400005FF0FF357FF0004A5FF0FF3B5FF0010C5446544512D15B4510D15D450ED15C46D1
:203420005C450BD15B4509D15D4507D14FEA7A0A0CF1010CBCF1200FEADD01E004F044BBDD
:20344000BDE8381C70472DE9701C0025002400265FF0010A5FF0000B5FF0010C5546554566
:2034600033D15C4531D15E452FD15D465D452CD15C452AD15E4528D14FEA4A0A0CF1010CF1
:20348000BCF1200FEADD5FF0FF355FF0FF345FF0FF367FF0004A5FF0FF3B5FF0010C5546C7
:2034A000554512D15C4510D15E450ED15D465D450BD15C4509D15E4507D14FEA7A0A0CF1BA
:2034C000010CBCF1200FEADD01E004F0FDBABDE8701C70472DE9E01C0026002500275FF0F5
:2034E000010A5FF0000B5FF0010C5646564533D15D4531D15F452FD15E465E452CD15D45A2
:203500002AD15F4528D14FEA4A0A0CF1010CBCF1200FEADD5FF0FF365FF0FF355FF0FF374D
:203520007FF0004A5FF0FF3B5FF0010C5646564512D15D4510D15F450ED15E465E450BD1AA
:203540005D4509D15F4507D14FEA7A0A0CF1010CBCF1200FEADD01E004F0B6BABDE8E01C23
:2035600070472DE9C01D002700265FF000085FF0010A5FF0000B5FF0010C5746574533D1B0
:203580005E4531D1D8452FD15F465F452CD15E452AD1D84528D14FEA4A0A0CF1010CBCF12B
:2035A000200FEADD5FF0FF375FF0FF365FF0FF387FF0004A5FF0FF3B5FF0010C57465745AF
:2035C00012D15E4510D1D8450ED15F465F450BD15E4509D1D84507D14FEA7A0A0CF1010C2A
:2035E000BCF1200FEADD01E004F06EBABDE8C01D70472DE9801F5FF0000800275FF0000967
:203600005FF0010A5FF0000B5FF0010CD046D04533D15F4531D1D9452FD1D846D8452CD16F
:203620005F452AD1D94528D14FEA4A0A0CF1010CBCF1200FEADD5FF0FF385FF0FF375FF040
:20364000FF397FF0004A5FF0FF3B5FF0010CD046D04512D15F4510D1D9450ED1D846D845C9
:203660000BD15F4509D1D94507D14FEA7A0A0CF1010CBCF1200FEADD01E004F025BABDE837
:20368000801F70472DE970075FF000095FF000085FF0000A012400250126A146A14530D100
:2036A000A8452ED1AA452CD1A946A94529D1A84527D1AA4525D14FEA440406F10106202EC4
:2036C000EBDD5FF0FF395FF0FF385FF0FF3A7FF000445FF0FF350126A146A14511D1A84594
:2036E0000FD1AA450DD1A946A9450AD1A84508D1AA4506D14FEA740406F10106202EEBDD14
:2037000001E004F0E1B9BDE8700770472DE9700E5FF0000A5FF000095FF0000B012400257E
:203720000126A246A24530D1A9452ED1AB452CD1AA46AA4529D1A94527D1AB4525D14FEADA
:20374000440406F10106202EEBDD5FF0FF3A5FF0FF395FF0FF3B7FF000445FF0FF35012618
:20376000A246A24511D1A9450FD1AB450DD1AA46AA450AD1A94508D1AB4506D14FEA740403
:2037800006F10106202EEBDD01E004F09DB9BDE8700E70472DE9701C5FF0000B5FF0000ABB
:2037A0005FF0000C012400250126A346A34530D1AA452ED1AC452CD1AB46AB4529D1AA45C5
:2037C00027D1AC4525D14FEA440406F10106202EEBDD5FF0FF3B5FF0FF3A5FF0FF3C7FF06B
:2037E00000445FF0FF350126A346A34511D1AA450FD1AC450DD1AB46AB450AD1AA4508D106
:20380000AC4506D14FEA740406F10106202EEBDD01E004F059B9BDE8701C70472DE97018AE
:203820005FF0000C5FF0000B012400250126A446A44526D1AB4524D1AC46AC4521D1AB45EE
:203840001FD14FEA440406F10106202EEFDD5FF0FF3C5FF0FF3B7FF000445FF0FF3501266F
:20386000A446A4450DD1AB450BD1AC46AC4508D1AB4506D14FEA740406F10106202EEFDD7F
:2038800001E004F021B9BDE8701870472DE9F0030024002546594E51445105F10405182D2C
:2038A000F8DB04255FF0000801245FF0010944514659B4425FD105F10407C659B0455AD19D
:2038C0002F1FC659B04556D140F805804659B04551D105F10407C659B0454CD12F1FC6594D
:2038E000B04548D14FEA440409F10109B9F1200FDDDD05F10405142DD6DB5FF0FF3400250A
:20390000445105F10405182DFADB04255FF0FF387FF000445FF0010944514659B4422AD119
:2039200005F10407C659B04525D12F1FC659B04521D140F805804659B0451CD105F10407E9
:20394000C659B04517D12F1FC659B04513D14FEA740409F10109B9F1200FDDDD05F10405DE
:20396000142DD5DB00254E59465105F10405182DF9DB012000E00020BDE8F00370472DE955
:20398000F00300240025445105F104058D42FADB00255FF0000801245FF001094451465985
:2039A000B44268D1002D03D02F1FC659B04562D105F104078F4202DAC659B0455BD140F81D
:2039C00005804659B04556D1002D03D02F1FC659B04550D105F104078F4202DAC659B04562
:2039E00049D14FEA440409F10109B9F1200FD5DD05F104058D42CEDB5FF0FF3400254451EA
:203A000005F104058D42FADB00255FF0FF387FF000445FF0010944514659B4422BD1002DF9
:203A200003D02F1FC659B04525D105F104078F4202DAC659B0451ED140F805804659B04559
:203A400019D1002D03D02F1FC659B04513D105F104078F4202DAC659B0450CD14FEA7404E6
:203A600009F10109B9F1200FD5DD05F104058D42CDDB012000E00020BDE8F0037047202A87
:203A800004DB203A21FA02F00021704721FA02F3D040C2F12002914008431946704740EAB7
:203AA00001039B0703D009E008C9121F08C0042AFAD203E011F8013B00F8013B521EF9D249
:203AC0007047D2B201E000F8012B491EFBD270470022F6E710B513460A4604461946FFF7AF
:203AE000F0FF204610BD10B5044604E00B7800F8013B03B1491C521EF8D2204610BD421C16
:203B000010F8011B0029FBD1801A704730B505460020034600E05B1C934205D2EC5CC85C33
:203B2000201A01D1002CF6D130BD2DE9F0410546002090460E46044600E0641C44450BD2AD
:203B4000285D00F083FA0746305D00F07FFA381A02D1295D0029F0D1BDE8F081F0B480EA77
:203B60000102D40F4200B2EB410F02D20246084611464A0042D0C30DDDB2C1F3C752AD1A20
:203B8000202D35DAC1F3160141F4000204B15242C5F1200602FA06F12A411044B3EBD05F23
:203BA00023D0C4B1012DA0EBC35009DCF0BC4FF0004202EAC352DBB200F5000000F055BA3D
:203BC000400000F1807000EBC350A0F1807040EAD170490009E0490841EAC071A0EBC3505D
:203BE00000F50000400800EBC350F0BC00F034BA6142012202EB4101001BF6E7F0BC7047B0
:203C000081F00041AAE780F00040A7E780EA010210B502F00043400022D04A001FD0010E42
:203C200001EB1261C0F35600C2F3560240F4000042F40002A0FB022000047F39140400D042
:203C4000401C50EA124001D44000491EC2B20C0604EBD010401C4008802A02D003E0002088
:203C600010BD20F00100002900DA0020184310BD2DE9FE4F804681EA0300C00F0C460090D3
:203C800021F0004123F00045B8EB0200A94105D24046214690461C460B46024623F0004003
:203CA000104347D0270DC7F30A00C3F30A510290401A019040286BDAC3F3130040F4801BCF
:203CC0000098924620B10023D2EB030A63EB0B0B01985946C0F14002504600F096F90646C6
:203CE0000D4650465946019A00F09EF910EB08006141002487EA115284EAE7731A4340D048
:203D0000009A62B3019A012A4FEA075215DC001B61EB02014FF0004202EA0752CDE9004283
:203D2000001C41F5801132462B4600F0D9F903B0BDE8F08F40462146F9E7001B61EB0201E7
:203D4000001C41F5801300185B412018A2F5001747EB030140EAD570B6196D4111E06D085C
:203D60004FEA360645EAC0754FEA0752001B61EB0201001C41F5801149084FEA30000019B8
:203D8000514132462B4603B0BDE8F04F00F09BB90098012240000023D0EB020263EBE0734F
:203DA000009821464FEAE074B8EB000061EB0401E9E783F000435BE781F0004158E72DE9B4
:203DC000F04D81EA030404F0004B21F0004514464FF0000A23F0004150EA050220D054EA39
:203DE00001021DD0C5F30A570246C5F31303C1F31300C1F30A5640F4801543F48013A7EBA4
:203E00000608101BD64608F2FD3873EB050002D308F1010801E092185B41B8F1000F03DA28
:203E200000200146BDE8F08D00204FF48011064684460EE0171B73EB050705D3121B63EB12
:203E4000050306434CEA010C49084FEA300092185B4150EA0107EDD152EA030012D082EA41
:203E6000040083EA0501084305D0101BAB4106D20122002306E000224FF0004302E06FF0AB
:203E8000010253101AEB06004CEB085110EB0A0041EB0B01BDE8F04D00F015B99623002269
:203EA000114600F0E2B80EB5C10F80EAE0700844CA07002140F233438DE80E000A460B46CA
:203EC00000F00EF903B000BD0EB540F2334102910021CDE900110A460B4600F001F903B059
:203EE00000BD00F0004220F00040C10DC0F3160040F400007F2901DA00207047962903DCC0
:203F0000C1F19601C84001E096398840002AF4D04042704720F00040C10DC0F3160040F496
:203F200000007F2901DA00207047962903DCC1F19601C840704796398840704770B5C1F35A
:203F40000A5201F000450024C1F3130140F2FF3341F480119A4201DA002070BD40F233430D
:203F60009A42A2F2334203DC5242FFF788FD00E090402C43F1D0404270BDC1F30A5210B50A
:203F8000C1F3130140F2FF3341F480119A4201DA002010BD40F233439A42A2F2334203DC1F
:203FA0005242FFF76CFD10BD904010BD00F0004230F000400AD0C10D01F56071C0F31600DA
:203FC00042EA0151C20840071143704700200146704701F0004330B421F0004150EA010282
:203FE00006D00A0DA2F56072C1F31301002A02DC30BC00207047440F44EAC104C100E018D9
:2040000030BC00EBC25000F027B8202A04DB203A00FA02F1002070479140C2F1200320FAE0
:2040200003F3194390407047202A06DBCB17203A41FA02F043EAE07306E041FA02F3D0406D
:20404000C2F120029140084319467047A0F14101192900D8203070470029A8BF7047401CC2
:20406000490008BF20F00100704710B4B0FA80FC00FA0CF050EA010404BF10BC704749B109
:20408000CCF1200421FA04F411FA0CF118BF012121430843A3EB0C01CB1D4FEA00614FEA26
:2040A000102042BF002010BC704700EBC35010440029A4BF10BC7047401C490008BF20F04F
:2040C000010010BC704710B5002B08DA401C41F1000192185B411A4301D120F0010010BDA8
:2040E0002DE9F04D92469B4611B1B1FA81F202E0B0FA80F220329046FFF787FF04460F4693
:2041000040EA0A0041EA0B0153465A46084313D0114653EA010019D0C8F140025046FFF7C8
:20412000AEFC05460E46504659464246FFF76DFF084305D0012004E020463946BDE8F08DEB
:204140000020054346EAE0762C4337430A986305E40AA0EB08000022FD0A44EA47540A30D1
:2041600002D500200146E9E7010510196941DDE9084500196941BDE8F04DA4E72DE9F04DC2
:2041800000231A461B1A8A4103DB00200146BDE8F08DC1F30A52C1F3130141F480154FF054
:2041A000000BD10702D100186D41521E0027044640F2FF11384601EB620A3E4680460246F8
:2041C00000204FF48011FFF75AFCC2197141BB1846EB0100B4EB030C75EB000C04D3E41A1E
:2041E00065EB000517460E46241908F101006D4180463428E3DDF91946EB0600091BA8419C
:2042000003D24FF0FF32134601E0002213461BEB070046EB0A51BDE8F04DFFF754BF000020
:20422000064C074D06E0E06840F0010394E8070098471034AC42F6D3FEF75CFF7C860108BE
:204240009C86010870B58C1810F8015B15F0070301D110F8013B2A1106D110F8012B03E0B8
:2042600010F8016B01F8016B5B1EF9D12B0705D40023521E0DD401F8013BFAE710F8013B49
:20428000CB1A921C03E013F8015B01F8015B521EF9D5A142D8D3002070BD000010B572B6E6
:2042A00006480079AA2801D00FF09AFA00200349087162B612F028FC10BD0000003002409F
:2042C00010B5024804F0D6FF10BD0000201F002070B5044600252068806800F00100F0B144
:2042E0002068806820F001002168886006F07CFC05460EE006F078FC401B022809D9A06A4A
:2043000040F01000A062E06A40F00100E062012070BD2068806800F001000028EAD10020EC
:20432000F6E770B505466C6AA06A00F05000E0B9A06A40F40070A0622068806800F46020E3
:20434000B0F5602F0DD1E06858B9A06A20F48070A062A06A00F4805018B9A06A40F0010008
:20436000A062204604F05EFC03E0206A016B2846884770BD70B505466C6AA06A40F0400084
:20438000A062E06A40F00400E062204604F071FF70BD70B50446656A284604F069FF70BD2F
:2043A00038B504460025002000902068806800F0010080BB2068806840F001002168886043
:2043C000164800681649B0FBF1F0009002E00098401E009000980028F9D106F005FC054668
:2043E00013E006F001FC401B02280ED9A06A40F01000A062E06A40F00100E06200BF002083
:2044000084F8240000BF012038BD2068806800F001000028E5D00020F6E7000000000020CC
:2044200040420F0070B505460E4606F0DDFB22490968401A02283DD3002418E01F4850F81E
:2044400024001F4931F81410C0EB81201B4951F8241001EBE010194941F82400084650F825
:204460002400C0F38F2025F81400601CC4B20B2CE4DB002418E0134850F82400124931F836
:204480001410C0EB81200F4951F8241001EBE0100C4941F82400084650F82400C0F38F202D
:2044A00026F81400601CC4B2032CE4DB06F09CFB0149086070BD000050050020941F002036
:2044C000C41E0020C01F0020FC04002010B5154804F06CF8144804F069F8124805F080F8C9
:2044E000114805F07DF8104804F070FA0B220F490C4805F00DF90B48006A0068006820F0D2
:2045000004000849096A09680860094807F0C3FB0C21074807F036FE0C21054807F0DCFA06
:2045200010BD0000F01E0020201F0020C41E0020041E002001460022664881420DD1664877
:2045400048604A68824201D000207047634848604A68824201D00020F7E7614881420DD1B3
:20456000604848604A68824201D00020EDE75E4848604A68824201D00020E6E740F2555057
:2045800048614A69824201D00020DEE740F6AA2048614A69824201D00020D6E740F25550A0
:2045A00088618A69824201D00020CEE740F6AA2088618A69824201D00020C6E740F25550A0
:2045C000C861CA69824201D00020BEE740F6AA20C861CA69824201D00020B6E740F25550A0
:2045E00008620A6A824201D00020AEE740F6AA2008620A6A824201D00020A6E740F255509C
:2046000048624A6A824201D000209EE740F6AA2048624A6A824201D0002096E740F255509B
:2046200088628A6A824201D000208EE740F6AA2088628A6A824201D0002086E72B48C862D5
:20464000CA6A824201D000207FE72948C862CA6A824201D0002078E7264808630A6B824216
:2046600001D0002071E7244808630A6B824201D000206AE71F4848634A6B824201D0002023
:2046800063E71D4848634A6B824201D000205CE71A4888638A6B824201D0002055E7184880
:2046A00088638A6B824201D000204EE700204860C860086148618861C861086240F6FF700D
:2046C000486200208862C86208634863886301203BE700000024014055554500AAAA8A0086
:2046E0000028014055554000AAAA800055555500AAAAAA0055555515AAAAAA2A555515009B
:20470000AAAA2A0088B001460022086800904868019088680290CB6803930B6904934B692F
:204720000593552008600A68552A02D0002008B07047AA2008600A68AA2A01D00020F6E76C
:2047400045F2555048604A68824201D00020EEE74AF6AA20486048684AF6AA2300EA03023B
:204760001846824201D00020E1E745F2555088608A68824201D00020D9E742F6AA20886049
:204780008A68824201D00020D1E745F25553CB60CA681846824201D00020C8E742F6AA23B7
:2047A000CB60CA681846824201D00020BFE745F255530B610A691846824201D00020B6E775
:2047C00042F6AA230B610A691846824201D00020ADE745F255534B614A691846824201D01D
:2047E0000020A4E742F6AA234B614A691846824201D000209BE7009808600198486002983A
:204800008860039BCB60049B0B61059B4B6101208DE70246002004E0002322F81030431CD3
:2048200098B28842F8DB70472DE9F04704460E4692461F464FF065087748007801286FD166
:2048400006F0D2F940F6C411884202D20020BDE8F08772480088401C70490880608A704930
:20486000096808446E4908606C480088012801DC1920ECE769480088032801DC3220E6E7AE
:2048800066480088052801DC4B20E0E763480088072801DC6420DAE700205F490870182F9B
:2048A0000AD15F480068C0F3CF0000EB80004000072190FBF1F010E0302F0AD1584800681B
:2048C000C0F3CF0000EB800040000D2190FBF1F003E053480068C0F3CF0052490880002561
:2048E00013E0B01C30F815004E490988884208DC30886843642190FBF1F03188A1EB000944
:2049000005E04FF00009681C85B24545E9DB00BFC4F80490A8EB0500401EC0B297E7FFE786
:20492000414880F800A0007840490870607C00286ED143F698216069B0FBF1F081B23C481C
:2049400002780078401C3A4B187004F11C0020F81210184600780C2825DB182F0BD10C2157
:2049600004F11C0003F06CFD00EB80004000072190FBF1F012E0302F0BD10C2104F11C0020
:2049800003F05EFD00EB800040000D2190FBF1F004E00C2104F11C0003F052FD214908802E
:2049A000002023490870002513E0B01C30F815001C490988884208DC30886843642190FBBB
:2049C000F1F03188A1EB000905E04FF00009681C85B24545E9DB00BFC4F80490A8EB0500CB
:2049E000401E12490870084600780F49097888420ADD0E4801780C4800781430814203DAB7
:204A000009480078094908700020606101206074064800781BE70000560300205203002077
:204A20005C0300205803002055030020540300205703002030B51E2A04DB0CDB64280ADAB0
:204A40000A2908DA9C891C809C89DC819C895C8000245C6030BD40F6EB244C43B4EB002F8E
:204A600001D2040202E040F6EB244C43950405EB85056D00B5FBF4F41C801C88B4F5FA7F2D
:204A800002DA4FF4FA7407E01C88B4F5FA5F02DD4FF4FA5400E01C881C801D885C68C4EB54
:204AA00085245D6805EB64145C605C68C4F38F245C805C88DC8100BFCCE7000038B5044670
:204AC0000B48012300220A2100900A4808F046F90948012300220A210090084808F03EF928
:204AE00003480078044909780840207038BD00002A040020501D00202B040020641D00208D
:204B000000BFFEE710B5024804F062FF10BD00002C24002000B58BB00020069007900120F2
:204B200008904CF220000190002002904DF2E01003904FF6FF7004900020059001200990C3
:204B400001A9244804F0A4FE20B14FF4A47122A011F070FD01200690002007900120089029
:204B60004FF460400190002002904CF2E01003904FF6FF700490002005900120099001A9ED
:204B8000144804F085FE20B140F25D1112A011F051FD0220069000200790012008904FF267
:204BA00040500190002002904FF6C07003904FF6FF70049001200590099001A9054804F098
:204BC00067FE20B14FF4B97103A011F033FD0BB000BD00002C2400202E2E5C436F72655CD9
:204BE0005372635C63616E2E630000002DE9F04104460D46002700260DB9666B00E0A66BB5
:204C0000206800F5D87000EB0510006800F00400B060B06858B9206800F5D87000EB051075
:204C2000006840F2FF7101EA505030600AE0206800F5D87000EB051000686FF0604101EA4D
:204C4000D0007060206800F5D87000EB0510006800F00200F060206800F5D87000EB051080
:204C6000406800F00F0030613562206800F5D87000EB05104068C0F30720F061206800F550
:204C8000D87000EB051080683075206800F5D87000EB05108068010A7175206800F5D870DC
:204CA00000EB05108068010CB175206800F5D87000EB05108068000EF075206800F5D870F4
:204CC00000EB0510C0683076206800F5D87000EB0510C068010A7176206800F5D87000EB77
:204CE0000510C068010CB176206800F5D87000EB0510C068000EF0764DB920202168C860EB
:204D00002068406920F00A002168486108E02020216808612068406920F050002168486139
:204D200094F83C70222F01D0322F05D12068406920F40F4021684861EDB994F83C00422844
:204D400004D0622806D072280CD107E0122084F83C000BE0322084F83C0007E0522084F80D
:204D60003C0003E0012084F83C0000BF00BF204605F0B6F81CE094F83C00522804D0622818
:204D800006D072280CD107E0122084F83C000BE0222084F83C0007E0422084F83C0003E02C
:204DA000012084F83C0000BF00BF204605F060F80020BDE8F08100002DE9F34F83B00446DE
:204DC00060790B287EDB0021204611F07DFD00906449009808700121204611F075FD82465C
:204DE000604981F801A0009855286CD1BAF1AA0FFBD12088000A88702078C870022120466B
:204E000011F062FD064657490E71112E03D0162E01D00C2E7ED10321204611F055FD804674
:204E2000504880F805800521204611F04DFD83460421204611F048FD0BEB00201FFA80F9C4
:204E40004FEA19204749887181F807900521204611F03AFD0546A8EB0500022872D1617959
:204E600008F10900814217DA207C012804D105F0BBFEE0600020207405F0B6FEE168411AF3
:204E80000498814205D96179204611F0D9FC0120207405B0BDE8F08F0120207400270EE067
:204EA000B81DC1B2204611F00FFD2F49C8550846C15D07F108002B4A1154781C87B2AF429E
:204EC000EEDB01E04CE047E0A81DC1B2204611F0FBFC4FEA006BE81DC1B2204611F0F4FCCC
:204EE0000BEB004B05F10800C1B2204611F0ECFC0BEB002B05F10900C1B2204611F0E4FCD7
:204F00000BEB0001019105F10801164800F038F9029000E01BE0DDE90110081A0CD120889F
:204F2000114B4A46314600F017FF08F10900C1B2204611F085FCACE70121204611F080FC13
:204F40000EE0FFE70121204611F07AFC08E00121204611F075FC03E00121204611F070FCC4
:204F600000BF96E7770C0020780B002030B50A4600211CE00F4B5B6B14335B5CC578846816
:204F80006355C3785B1CDBB2C3708478A34201DB0023C37043795B1CDBB243718478A3427F
:204FA00003DD83784371012383714B1CD9B29142E0DB30BD2C2400202DE9F047824688468A
:204FC0001446002C5FDD2046E11704EB5171C910A4EBC1018FB237B90827E11704EB5171CD
:204FE000C1F3CF0907E02046E11704EB5171C910491C1FFA81F92548006BC0F800A000200E
:205000002249096BC8602149096B886000261CE008201E49096B086100250AE0082000FB03
:20502000065018F800101948006B14304155681C85B2082DF2DB0A21144804F0C1FF012833
:2050400001D10CF091FC701C86B2A9F10100B042DEDC0E48006B076100250AE0082000FB8F
:20506000065018F800100948006B14304155681C85B2BD42F2DB0A21044804F0A1FF012869
:2050800001D10CF071FCBDE8F08700002C24002010B504462068406920F0010021684861C6
:2050A00094F83C00122805D12068406920F40F402168486194F83C00422804D0522806D0FC
:2050C00072280CD107E0222084F83C000BE0322084F83C0007E0622084F83C0003E001205E
:2050E00084F83C0000BF00BF204605F0C1F8002010BD000010B5014600224C69CB695520ED
:2051000008600A68552A01D0002010BDA82008600A6802F0A802A82A01D00020F5E70A4849
:2051200048614A69824201D00020EEE7074848614A69824201D00020E7E74C61CB614FF43F
:20514000004008600120E0E7550501002A8A020030B503460C460021002200BF09E0985C4F
:2051600080EA1120C0B2054D35F8100080EA0121521CA242F3D388B230BD000074790108D2
:20518000F0B502460B460025681E00210FE0565C7040002407E0060E064F57F82650000279
:2051A0006840661CB4B2042CF5DB4E1CB1B29942EDDBF0BD747B010800B585B000BF184841
:2051C000806940F00400164988610846806900F00400009000BF00BF00BF0846806940F00B
:2051E000080088610846806900F00800009000BF00BF08200190002002900120039001A9B8
:20520000084805F051FB4FF400400190002002900120039001A9044805F046FB05B000BDE5
:2052200000100240000C0140000801402DE9F84F04460D4616461F4600F0FAF8009000F069
:20524000F7F8804600F0F4F881460098404504D1C84502D16A4880F800906A48007830B957
:2052600067480078664948700120664908706448007863494978884238D0614840786049EB
:20528000097801F00301604A515C884209D1002060705E4908805E4908806068401C60606B
:2052A00024E0574840785649097801F00301594A515C88420DD155480088401C53490880E1
:2052C00008460088042811DB01206070002008800CE04F480088401C4D49088008460088EC
:2052E0000A2803DD01206070002008804FF0020A4348007800F001004149497801F0010186
:2053000088422DD005F070FC43490968401A4FF47A71B1FBF0F04149088005F065FC3E4965
:20532000086017B94FF0010A00E0B246607858B93B480078401C3A4908700846007850457D
:2053400004DB0120A07001E00020A07035490888012111F0FFFD208105F046FC3249086044
:20536000324800682D490988C0EB81202F49096801EB20202D49086008460068C0F38720F5
:2053800020704FF0640B25480088142802DA4FF496700DE021480088282801DD642007E002
:2053A0001E48008800EB80004FF4FA71A1EB40001FFA80FB0BFB05F0642190FBF1F085B263
:2053C00005F012FC18490968401AA84211D90020A0700220607000202070104908801349BB
:2053E00008600F4908700F490888002111F0B2FD20810348007802494870BDE8F88F000029
:20540000980300209A030020608301089C0300209E03002064830108A0030020A80300202A
:20542000AA0300200A050020AC030020A403002070B54FF40041084805F0C4FB05462C4670
:205440000821064805F0BEFB064644EA4600C4B204F0030070BD000000080140000C014037
:2054600000BF084A1268526A91B201EB810292004FF47A7392FBF3F202800022014B1B688C
:205480005A627047441E002010B54FF4FA710948FFF792FC4FF4FA710748FFF78DFC4FF410
:2054A000FA710648FFF788FC4FF4FA710448FFF783FC10BD780500208C050020A00500206A
:2054C000B4050020F0B58DB007460E46154618A103C9CDE90B0118A103C9CDE9070109ABD7
:2054E000002231460BA811F059FA05AB0022314607A811F053FA002405E009A8005D01A905
:205500000855601CC4B2082CF7DB002407E005A8015D01AA04F108001154601CC4B2082CED
:20552000F5DB294601A801F0C8FC0DB0F0BD000039FF6C063454333029270957FFFFFFFF23
:2055400038B505460C46002000906A462146284601F072FE601CC1B20DF10102284601F0DC
:205560006BFEA01CC1B20DF10202284601F064FEE01CC1B20DF10302284601F05DFE9DF80F
:2055800000009DF8011008409DF8021008409DF80310FF2901D1012100E00021084080F0B1
:2055A000010038BD30B502460B460021002400BF0EE0481C84B207E0505C155DA84201D12A
:2055C000002030BD601C84B29C42F5DB481C81B29942EEDB0120F4E731B581B0BDF8040057
:2055E000ADF80000BDF9040044F6E61500FB05F1C913BDF9060000FB05F2D2130C4613460C
:205600006042C01AC01A00B2ADF8020000983CBD70B504460AB9084670BD081B800290FB6D
:20562000F2F086B2934202DD0D462846F4E706FB03F004EBA02085B22846EDE710B51022ED
:2056400049494A480DF008FA044624B9102246494748FEF724FA10224349444814300DF012
:20566000FBF904462CB910223F4941481030FEF716FA20223C493D4828300DF0EDF90446AE
:2056800024B9202238493B48FEF709FA1022364936484C300DF0E0F9044624B9102232499A
:2056A0003548FEF7FCF910222F49304860300DF0D3F9044624B910222B493048FEF7EFF9E6
:2056C00010222949294874300DF0C6F9044624B9102225492A48FEF7E2F920222249234834
:2056E00088300DF0B9F9044624B920221E492548FEF7D5F9234800782349087020221A49D7
:205700001A48AC300DF0A8F9044624B9202216491E48FEF7C4F9102213491448D0300DF0E6
:205720009BF9044624B910220F491948FEF7B7F908220D490D48E4300DF08EF904462CB982
:20574000144809490A68026049684160CC2206490648F0300DF080F9044624B9CC220249F4
:205760000D48FEF79CF910BD5017002008FC010854080020780A0020980A0020A80A002037
:20578000B80A0020E809002091010020080A0020280A002098040020EC08002010B5044601
:2057A000684B0C220421204602F092FE401C28B9644B0C220421204602F08AFE624B01220C
:2057C0001221204602F084FE401C28B95E4B01221221204602F07CFE5B4B183B1822152145
:2057E000204602F075FE401C30B9574B183B18221521204602F06CFE544B01222F212046FA
:2058000002F066FE401C28B9504B01222F21204602F05EFE4D4B183B18223221204602F063
:2058200057FE401C30B9494B183B18223221204602F04EFE464B01224C21204602F048FEF7
:20584000401C28B9424B01224C21204602F040FE3F4B183B18224F21204602F039FE401CE6
:2058600030B93B4B183B18224F21204602F030FE384B30226921204602F02AFE401C28B91A
:20588000344B30226921204602F022FE31480068401C304908600B463022692120460EF086
:2058A0005CFC401C28B92B4B3022692120460EF054FC294B10229B21204602F009FE401C30
:2058C00028B9254B10229B21204602F001FE234B1022AD21204602F0FBFD401C28B91F4BCD
:2058E0001022AD21204602F0F3FD1D4B0822C321204602F0EDFD401C28B9194B0822C321F9
:20590000204602F0E5FD174B1022CD21204602F0DFFD401C28B9134B1022CD21204602F084
:20592000D7FD114B0222DF21204602F0D1FD401C28B90D4B0222DF21204602F0C9FD0020F6
:2059400010BD0000FC0A0020DC150020F615002010160020380A0020680A0020580B00205B
:2059600093010020680B0020EA0300201CB53049304801F047FD10222F492E4808300EF086
:2059800089FB10222C4910312A481C300EF082FB20222A49274830300EF07CFB10222849C6
:2059A000244854300EF076FB10222649214868300EF070FB102224491E487C300EF06AFB69
:2059C000202222491B4890300EF064FB202220491848B4300EF05EFB10221E491548D83056
:2059E0000EF058FB08221C491248EC300EF052FBCC221A490F48F8300EF04CFB1848007819
:205A000000061749497800EB01401549897800EB01201349C9780844009004211048FFF7DC
:205A2000AFFB019002226946024801F0C1FE1CBDFFFF010800FC010854080020780A00205B
:205A4000980A0020A80A0020B80A0020E8090020080A0020280A002098040020EC0800206B
:205A60006883010838B50546002410F081FD10F059FD284601F04AFB284601F003FB1F489A
:205A8000008800909DF800200021284601F02AFC401C28B99DF800200021284601F022FC03
:205AA0009DF801200121284601F01CFC401C28B99DF801200121284601F014FC0221684642
:205AC000FFF746FB044622120221284601F00AFC401C20B922120221284601F003FCE2B20B
:205AE0000321284601F0FEFB401C20B9E2B20321284601F0F7FB002038BD00006C830108DF
:205B000010B5094A0949A2F10C00FFF7DBFC064B0C22042106480EF020FB0648006820F4DA
:205B200000100449086010BDFC0A002093010020180400208401002070B505460026394801
:205B40000078C8B9002404E03748C0880644601C84B20A2CF8DB0A20B6FBF0F033490880B9
:205B600005F042F83249086005F03EF83149086001202C4908704FE005F036F82D490968BF
:205B8000401AB0F5FA7F03D905F02EF8284908602868C0F3804000283ED105F025F8244904
:205BA0000968401AB0F5FA6F36D9002404E01E48C0880644601C84B20A2CF8DB0A20B6FB67
:205BC000F0F01A49088008460088B0F57A7F05DB0846008840F6B831884219DD286820F44D
:205BE000802000F5802028600720134948800F4800888880084601F0D9FC00200F490870B2
:205C00000F484089401C0E49488102200D49087004F0EAFF0649086004F0E6FF05490860D5
:205C200070BD000040000020C41E0020200500204400002048000020E41400206903002020
:205C4000680A00209201002010B5024804F092FB10BD0000501F00203FB504460025206828
:205C6000009060680190A0680290E06803900020206045F2555020602568854202D0002084
:205C800004B030BD0020206042F6AA2020602568854201D00020F3E70020206045F25550A6
:205CA000606005200DF08CFE656845F25550854201D00020E4E74AF6AA20606005200DF060
:205CC0007FFE65684AF6AA20854201D00020D7E74FF05530A060A568B5F1553F01D00020FE
:205CE000CEE74FF0AA30A060A568B5F1AA3F01D00020C5E74FF05530E060E568B5F1553F12
:205D000001D00020BCE74FF0AA30E060E568B5F1AA3F01D00020B3E7019860600298A0603C
:205D20000398E060009820600120A9E730B590F840500124AC40C56B6C60046863604468DA
:205D4000102C04D10468A2600468E16003E00468A1600468E26030BD2DE9F84F07468846B4
:205D600015461C4605F0FF0A40F23171781A8F4273D00CDCA7F25160002801F04F80CF28DD
:205D80000ED0D0280DD0DF2841F0618064E00F287ED010287DD01F287CD02028F4D1A0E3C6
:205DA00000BF41F20C61681A8D4236D00BDCA5F58050A0F1100070B1B0F53E7F23D0B0F520
:205DC000806F45D123E0B0F5807F2CD0A0F5C850F93878BB2FE052462146FE48FDF75FFE65
:205DE000FC48407AFC49C8730020FC49887604F0FBFEFA49C8610020F949087004F0F4FEA9
:205E0000F749486025E001200CF010FB21E052462146F448FDF743FE1BE052462146F248C8
:205E2000FDF73DFE15E052462146EF480C30FDF736FE0EE00CE052462146ECA0FDF766FEE7
:205E400028B9EC48007820F00100EA49087000E000BF00BFF2E300E000BFB5F5545F7DD07D
:205E600025DC43F20511A5EB01008D427AD014DCA5F58050A0F10800B0B3B0F5017F38D0A9
:205E8000B0F5417F3BD0A0F5F850FA38002802E01FE21FE224E372D138E0A0F20310002848
:205EA00071D0F8287FD0B0F5007FF4D1B1E0B5F5824F67D00DDCA5F55850A0F1050000281D
:205EC0006FD0A0F2FB2000286CD0B0F5E16FE2D13FE1A5F58440083800287DD0F8287CD02B
:205EE000B0F5067FD7D1D4E1FFE701200CF09EFAEDE152462146C048FDF7D1FDE7E1524689
:205F00002146BD480C30FDF7CAFDE0E1BB48007801280DD052462146B948FDF7C0FDB8482B
:205F20000078C043B7490870B5484078C0434870B3480078A8494873B148407888730B46E2
:205F40004FF481520C214FF4E2600EF09DF90020AD49087004F048FEAB4901E093E001E0F4
:205F60004860B4E152462146A0A0FDF7CFFD28B9A048007820F002009E490870A7E1A5E125
:205F800001E010E0F3E052462146A048FDF787FD9FA345F203320C2140F213700EF074F903
:205FA00095E179E0ACE0202221469A480CF054FD202221469848FDF772FD9748007B2070D8
:205FC00095484078607094480079A0709248C07EE0700120207101E0D0E0E2E00F2060718A
:205FE0002022A11D8B4824300CF036FD2022A11D8A48FDF754FD8948007CA0710020E07165
:20600000234645F208420C2140F213700EF03CF95DE1207840B28049C876084690F91B00C0
:206020000A2801DD0A20C8767B4890F91B0010F10A0F02DAF6207849C87660787649487027
:20604000207940B275490874084690F91000002802DD0020087408E0704890F9100010F1B7
:20606000140F02DAEC206D49087400206C49087001F0F4FE66A345F203320C2140F213705C
:206080000EF002F923E1674B41F210520C214FF4E2600EF0F9F81AE15246214662A0FDF72B
:2060A00035FD60BB00205F498860C8600922604960A0FDF72BFD80B15A480068B0F57A7FF2
:2060C00003D20020574908604860092259A15848FDF709FD002052490870524B1022AD218C
:2060E00057480EF03AF84AA345F203320C2140F213700EF0C9F80020374908834883E6E01B
:206100005048007820BB10224F49424888380CF0A3FC10224C4910313E4874380CF09CFC17
:206120000C214A48FFF72CF806464748C66203464FF492520C214FF4E2600EF0A5F8444B37
:206140004FF4B9520C214FF4E2600EF09DF800BFBDE0524621463F48FDF7A1FC2CA345F233
:2061600003320C2140F213700EF08EF8AFE03A4A3A493B48007802F0B7F8A8E052462146CB
:206180003648FDF78CFC00202549087001F066FE1FA345F203320C2140F213700EF074F830
:2061A00095E0202221461B480CF056FC202221461948FDF774FC20222146164824300CF04B
:2061C0004BFC202221461548FDF769FC12480E30016847E0B408002014080020E0020020D7
:2061E000C0010020DC080020C4080020524541445900000088010020B8090020D0000020DF
:20620000D2000020D4000020B00100208901002041434B0090FC0108E8090020080A002076
:2062200011040020580B0020434C454152000000980A0020434C4541525F4F444F000000D5
:2062400018040020D601002054080020F00A002094080020900400207004002098040020B5
:20626000A104002021604168616000892081F6480168C4F80A104168C4F80E1000896082D9
:20628000234645F220620C2140F213700DF0FCFF1DE0EE482168016061684160218901814F
:2062A000E948D4F80A100160D4F80E104160618A01810020E6490870AFF2AC0345F20332EB
:2062C0000C2140F213700DF0DFFF00E000BF00BFC0E500BFB5F5445F5ED010DCA5F580506E
:2062E000A0F58670C8B1B0F5807F1CD0B0F57F7F20D0A0F5F050F438002872D122E0A5F56F
:2063000048500838F0B3FD286CD0B0F5FC7F6AD0A0F2FD200028F0D1A7E052462146CD4814
:20632000FDF7BDFBDAE052462146CA480C30FDF7B6FBD3E00020C849087004F055FCC64955
:206340004860CBE0C548007828BB1022C449C5480CF082FB1022C2491031C24814300CF0F5
:206360007BFB0C21C048FEF70BFF0646BC48C66203464FF492520C214FF4E2600DF084FF59
:20638000BA4B00E030E04FF4B9520C214FF4E2600DF07AFF00BFA1E020222146B1488830F8
:2063A0000CF05AFB20222146A8480E38FDF777FBA6480E38007B2070A4480E38407860704E
:2063C000A2480E380079A070A0480E38C07EE070234647F208320C2140F214700DF054FF39
:2063E0007CE07AE02AE037E0207840B297490E39C876084690F91B000A2801DD0A20C8766D
:2064000092480E3890F91B0010F10A0F03DAF6208E490E39C87660788C490E394870002083
:206420008B49087001F01AFDAFF21C2347F203420C2140F214700DF027FF4FE05246214676
:20644000AFF25820FDF762FB28B98948007820F004008749087041E0864B41F210520C2198
:206460004FF4E2600DF010FF38E052462146AFF24820FDF74BFB78BB00207E498860C86007
:2064800009227D49AFF25420FDF740FB88B179480068B0F57A7F03D2002076490860486003
:2064A0000922AFF270217448FDF71DFB002068490870704B1022AD2170480DF04EFEAFF211
:2064C000B02347F203420C2140F214700DF0DCFE00206B490883488300BF00BF00BFB9E4AD
:2064E00000BF42F22041681A8D4278D04DDCB5F5D05F75D028DCB5F5A85F72D015DCB5F5D6
:20650000905F6FD008DCB5F5805F6CD0A5F588500838002868D1CCE0B5F5985F79D0A5F561
:20652000A05010380028F5D119E1A5F5B050103800286FD0F0286ED0B0F5007F6CD0A0F2AA
:20654000F1200028E6D15EE1B5F5F85F74D00DDCB5F5D95F71D0B5F5E05F70D0A5F5E850C0
:20656000103800286CD0F028D4D1B4E1B5F5005F67D0B5F5045F65D0A5F508501038002839
:2065800061D0B0F5807FC5D1E3E1B0F51E6F79D02BDC40F2E152A0EB0201904273D011DC55
:2065A000B0F53A7F70D006DCE5286ED0A0F2E5100028AFD10DE2A0F2E230002875D0FE28BB
:2065C000A8D1B3E2A1F2011000286FD0FF286ED0A0F2062000286BD0E8289BD1F3E2CBE125
:2065E0002DE1CEE080E051E0FDE340F6E162811A904275D011DCB0F52E6F72D0B0F53E6F80
:2066000070D0B0F5506F6ED0A0F6E15000288AD152E395E0C4E0D5E0E3E0A1F201100028BC
:206620007DD0FE287CD0A0F20750002879D0A0F2C310002886D1DCE35EE10FE1EDE329E195
:2066400037E168E168E170E11A0A0020F609002011040020D0090020B8010020D6010020DE
:206660005408002008FC0108F00A00209408002088010020580B0020980A00201804002091
:2066800014080020E6E252E2CFE187E1FE4B0822C321FE4801F01CFFFB4B4AF208420C2108
:2066A00040F215700DF0F0FDB6E3DAE140E254E257E252462146F448FDF7F1F9F24B0822D4
:2066C000C321F2480DF049FDAFF2BC434AF603120C214FF4E2600DF0D7FDFFF711FA9BE362
:2066E00018E3C0E2C8E2D5E2E948007838BB1022E849E9480CF0B0F91022E6491031E648F7
:2067000014300CF0A9F90C21E448FEF739FD0646E048C66203464FF492520C2102E00FE306
:2067200041E34FE34FF4E2600DF0AEFDDC4B4FF4B9520C214FF4E2600DF0A6FD00BF6BE302
:206740001022D849D4484C300CF086F9D54B4AF210620C2140F215700DF096FD5CE35246BA
:206760002146D048FDF79BF90020CF490870AFF260534AF603120C214FF4E2600DF084FD89
:206780004AE31022C949C44860300CF065F9C74B4AF210720C2140F215700DF075FD3BE351
:2067A00052462146C148FDF77AF90020BE490870AFF2A4534AF603120C214FF4E2600DF02F
:2067C00063FD29E31022BA49B34874300CF044F9B74B4AF610020C2140F215700DF054FDBA
:2067E0001AE352462146B248FDF759F90020AE490870AFF2E4534AF603120C214FF4E260EF
:206800000DF042FD08E32078AA49087008460078C043A9490870A748007878B1A748006834
:2068200020F48060A54908600846006820F4805008600846006820F400600860ECE220226A
:206840002146954888300CF007F923464AF220020C2140F215700DF017FDDDE252462146C6
:206860009748FDF71CF9964800789649087000208D4908709249487B0FF0D4F901F0EEFAD2
:20688000AFF274634AF603120C2140F215700DF0FBFCC1E2102221467F48D0300CF0DCF880
:2068A00023464AF210120C2140F215700DF0ECFCB2E2524621468448FDF7F1F800207A4929
:2068C0000870AFF2B4634AF603120C2140F215700DF0DAFCA0E27D4B4AF230220C2140F245
:2068E00015700DF0D1FC7A4B4AF610420C2140F215700DF0C9FC8FE22022764966482830D4
:206900000CF0AAF8734B4AF220520C2140F215700DF0BAFC80E27FE26F4B41F201420C21B6
:206920004FF4E2600DF0B0FC76E2524621465948FDF7B5F800205C490870AFF22C734AF6D3
:2069400003120C214FF4E2600DF09EFCFFF7D8F862E2524621464F481030FDF7A0F800204D
:2069600051490870AFF258734AF603120C214FF4E2600DF089FC4FE2524621465548FDF74F
:206980008EF8002048490870AFF27C734AF603120C214FF4E2600DF077FC3DE25246214623
:2069A0004EA0FDF7B3F898B9AFF29C734AF603120C2140F215700DF067FC00200BF036FD62
:2069C000642003F02BFE01200FF00CFF04F02EFA22E252462146AFF2B070FDF797F818BBB6
:2069E000FF2304220021294800F01EFBFF236D226921264800F018FB3A492748083800F0E6
:206A000001FD25490939384800F0FCFCAFF600034AF603120C2140F215700DF035FC012030
:206A20000FF0E0FE04F002FAF6E1524621462FA0FDF76CF8A0B90FF09BFD144800F066FBEF
:206A4000FEF794FFAFF638034AF603120C2140F215700DF019FC01200FF0C4FE04F0E6F9CE
:206A6000DAE1524621462448FDF719F822480078C0432249087020484078C0434870002028
:206A80001F4908703EE000009301002018040020D60100205408002008FC0108F00A00206E
:206AA00094080020980A002011040020A80A0020B80A0020D0000020D100002084010020E9
:206AC000E809002091010020280A0020380A0020680A0020780A0020880100205245534533
:206AE00054000000FFFF010800F801085245434F5645525900000000D2000020D4000020E5
:206B0000B001002004F070F8D3494860D3480078D3494873D148407888730B464FF48152E7
:206B20000C214FF4E2600DF0AFFB75E174E173E152462146CB48FCF7B2FFCA4B0222DF210E
:206B4000C9480DF00AFBAFF638134AF603120C2140F215700DF098FB5EE12078C34908700E
:206B60005AE100BF20790006617900EB0140A17900EB0120E179084421780906627801EB3C
:206B80000241A27801EB0221E2781144401A461C20780006627800EB0240A27800EB022052
:206BA000E2788118324604F10800FCF778FF4AF60830304482B223460C2140F215700DF099
:206BC00063FB00BF28E100BF20780006617800EB0140A17800EB0120E178461820790006B2
:206BE000617900EB0140A17900EB0120E17900EB010BABEB060000F10109B6F1005F0FD993
:206C00004A4604F108013046FCF749FFAFF600234AF603120C2140F215700DF035FB17E010
:206C20009348864214D906F2FF31304600F0EAFB09F0FF0204F1080130460DF02BFAAFF61C
:206C400030234AF603120C2140F215700DF01CFB00BF00BF874B41F210520C214FF4E260FD
:206C60000DF012FBD8E0844B41F208620C214FF4E2600DF009FBCFE0202221467F480BF019
:206C8000EBFE23464AF620520C2140F215700DF0FBFAC1E0524621467948FCF700FF0020A7
:206CA00078490870AFF698234AF603120C2140F215700DF0E9FAAFE02078401E00EB400270
:206CC000C2EB40101530C1B2631C1822664801F0FFFB2078012804D0022807D003280FD10C
:206CE00009E06948C08AA4F8170009E06748C08AA4F8170004E06648C08AA4F8170000BF1A
:206D000000BF23464AF61A620C2140F215700DF0BBFA81E02078401E00EB4002C2EB401078
:206D20001230C1B2631C01224F4801F0D1FB23464AF602720C2140F215700DF0A5FA6BE0C0
:206D4000207801280AD160784F49087601F118030122122144480DF000FA1AE02078022807
:206D60000AD160784949087601F1180301222F213D480DF0F2F90CE02078032809D1607802
:206D80004349087601F1180301224C2136480DF0E4F9AFF684334AF603120C2140F215705F
:206DA0000DF072FA38E023460222DF212E4801F08FFB23464BF202020C2140F215700DF049
:206DC00063FA29E05246214632A0FCF79FFE78B90FF0A8FB244800F055F9AFF6CC334AF68B
:206DE00003120C2100E016E040F215700DF04CFA12E0524621462A48FCF751FE0020214952
:206E00000870AFF6F4334AF603120C2140F215700DF03AFA00E000BF00BF19E0A5F514506F
:206E2000053820B1A0F5F840063828B900E000BF02201C49087000E000BF00BF2B46424663
:206E400040F25161184800940DF06AFA00E000BF00BFBDE8F88F0000B0010020D2000020AC
:206E600014080020EA03002018040020A701002000300008580B0020C8010020B4FC010868
:206E8000080A002011040020C4150020DE150020F81500204C4F4720434C454152000000E9
:206EA000EC0800205D000020D8050020704700BF0100A0F10100FBD1704710B5024600208B
:206EC00016E0135C041D145D63400B54031DD35C00F10804145D6340041D0B55231DD35C69
:206EE0000834145D634000F108040B55431CD8B20428E6DB10BD00001FB54FF460400090FB
:206F000011200190022003906946194803F0CCFC4FF4E060009011200190022003906946F6
:206F2000144803F0C1FC00224FF48071114803F055FE00224FF400710E4803F04FFE0022C2
:206F40004FF480610B4803F049FE00224FF40051074803F043FE00224FF48041044803F0E2
:206F60003DFE00224FF40041014803F037FE1FBD000C01400008014010B500210D4805F01D
:206F800021F904210B4805F01DF90821094805F019F90021074804F0B5FD0421054804F057
:206FA000B1FD0821034804F0ADFD0C21014805F0E9F810BD041E0020F8B50446002000900F
:206FC0006A460021204600F037F90DF101020121204600F031F902216846FEF7B9F80646F4
:206FE0006A460221204600F027F90DF101020321204600F021F99DF801009DF8001000EB8D
:20700000012085B2A81B03D12046FEF7C7FBF8BD0448007818B92046FEF724FDF7E74FF081
:20702000FF30F4E7D80100202DE9F04780460C4616461F46301B00F0FF09002507E060195F
:20704000C1B23A46404600F04DF9681CC5B24D45F5DBBDE8F08700001FB504460220009038
:207060000120019003906946054803F01DFC01220221034803F0B2FD204605F0AFFC1FBDAE
:20708000000C014010B504461C4B3022692120460DF063F8401C28B9184B302269212046B1
:2070A0000DF05BF8164B10229B2120460DF055F8401C28B9124B10229B2120460DF04DF851
:2070C000104B1022AD2120460DF047F8401C28B90C4B1022AD2120460DF03FF80A4B1022FE
:2070E000CD2120460DF039F8401C28B9064B1022CD2120460DF031F810BD0000380A0020A5
:20710000680A0020580B0020680B002010B50446424B0C22042142480DF01FF8401C28B9FD
:207120003E4B0C2204213E480DF017F83D4B0122122120460DF011F8401C28B9394B0122B3
:20714000122120460DF009F8364B183B1822152120460DF002F8401C30B9324B183B1822A8
:20716000152120460CF0F9FF2F4B01222F2120460CF0F3FF401C28B92B4B01222F212046B2
:207180000CF0EBFF284B183B1822322120460CF0E4FF401C30B9244B183B18223221204677
:2071A0000CF0DBFF214B01224C2120460CF0D5FF401C28B91D4B01224C2120460CF0CDFF64
:2071C0001A4B183B18224F2120460CF0C6FF401C30B9164B183B18224F2120460CF0BDFF65
:2071E000134B0822C32120460CF0B7FF401C28B90F4B0822C32120460CF0AFFF0D4B0222DA
:20720000DF2120460CF0A9FF401C28B9094B0222DF2120460CF0A1FF10BD0000FC0A0020BA
:2072200018040020DC150020F61500201016002093010020EA0300202DE9F04106460F46E7
:2072400015460024304605F03CFCA021304605F07DFC00BF00BF601C84B240F6B830844253
:2072600003DD4FF0FF30BDE8F081304605F096FB0028F0D13946304605F068FC002400BF94
:20728000601C84B240F6B830844202DD4FF0FF30E9E7304605F082FB0028F1D1304605F0FE
:2072A00010FCA121304605F051FC002400BF601C84B240F6B830844202DD4FF0FF30D2E7C9
:2072C000304605F06BFB0028F1D12946304605F0A2FB304605F0D2FB304605F012FC0020AB
:2072E000C1E700002DE9F04106460F461546002400220221294803F071FC304605F0E1FB22
:20730000A021304605F022FC00BF00BF601C84B240F6B830844203DD4FF0FF30BDE8F081AB
:20732000304605F03BFB0028F0D13946304605F00DFC002400BF601C84B240F6B830844257
:2073400002DD4FF0FF30E9E7304605F027FB0028F1D12946304605F0F9FB002400BF601C6C
:2073600084B240F6B830844202DD4FF0FF30D5E7304605F013FB0028F1D1304605F0C1FB60
:207380000A2003F04BF901220221044803F026FC034803F057FC0020C0E70000000C014040
:2073A000F0070020F8B510480468001D0568200E8DF80000200C8DF80100200A8DF80200A5
:2073C000E0B28DF8030004216846FDF7D9FE0646701B02D1FEF732F904E00448007808B9C2
:2073E000FEF7C4FAF8BD000000FC0108D801002010B50446207818B9FEF7B8FA0120207057
:2074000010BD000038B504460D4600200C49086008468460281B401C800AC86003F0CCF9FD
:2074200000BF34200749C86000BF6946044803F009F903F05FF9642003F0F0F838BD000073
:20744000401700200020024010B504220E490F480BF002FB0446A4B904220B490CA0FCF702
:2074600055FB70B928220849084808300BF0F4FA044634B9282204490748FCF710FB00204C
:2074800010BD0120FCE700005017002000F40108464C414700000000C80A002010B54FF483
:2074A000805003F0F3F910BD10B5042003F0EEF910BD00001FB54FF46040009002200190C6
:2074C00003906946064803F0EFF94FF4E06000900220019003906946024803F0E5F91FBD42
:2074E000000C01400008014010B50021104804F049FE04210E4804F045FE08210C4804F05A
:2075000041FE0C210A4804F03DFE0021084804F0E3FA0421064804F0DFFA0821044804F093
:20752000DBFA0C21024804F0D7FA0BF005F810BD041E00202DE9F04107460C46207860BB9A
:20754000384600F057F846B2701C48B11448402101FB06054022394628460CF0D1FD1AE01A
:207560000F49491E0F48FFF74DFFF0220C4940310C4800F01DF90C490948FFF743FFF02291
:207580000849074800F014F9074D3F3D4022394628460CF0B5FD01202070BDE8F0810000BA
:2075A00000F8010800F40108FFFB010810B504460B480068A0600B484068E06020220A4930
:2075C00004F11000FCF76BFA0848016821634068606307480168A1634068E06310BD000032
:2075E00084010020380A002014080020C8010020D600002010B50246002119E0114C04EBF6
:207600008110B0F800384FF6FF7083420ED111B90120108008E04020C0EB8110094C2044E9
:20762000B0F80038581C1080084610BD481C41B21029E3DB04480388581C10804FF0FF30B4
:20764000F3E7000000F00108C0FB01080021074AD1610749096941F00401054A11611146DF
:20766000096941F0400111617047000008070020002002400021074AD1610749096941F0D5
:207680000201054A116111464861096941F040011161704708070020002002400022054B16
:2076A000DA61054A126942F00102034B1A61018070470000080700200020024000201E4977
:2076C000C96801F0100139B11C49C96941F002011A4AD16140F010001749C96801F0040165
:2076E00039B11649C96941F00101144AD16140F004001149C96901F0010169B10F49C969F5
:2077000041F004010D4AD16100BF0B49C96921F00101094AD16100BF00BF40F20111884241
:2077200006D10549C96921F00101034AD16101E00149C86000BF7047002002400807002006
:2077400070B5044603F050FA054609E0601C38B124B103F049FA401BA04201D9032070BD72
:207760001248C06800F001000028EFD10F48C06800F0200020B100BF20200C49C86000BF13
:207780000A48C06800F0100048B90848C06900F0010020B90548C06800F0040018B1FFF703
:2077A0008DFF0120DBE70020D9E70000002002402DE9F04104460E461746002502F0FCFFC4
:2077C00000BF0FE056F825C0624600232146022002F09AFF08B9241D03E002F08BFFBDE8E3
:2077E000F0816D1CBD4202D203488442EAD902F081FF00BFF3E70000FBFF0108022005496A
:20780000087000200449088048800449088048807047000030000020280000202C000020FB
:207820000120014908707047300000202DE9FF4704460E4617464FF0000A0CF07DFB0390B7
:207840000398FDF7C9FE029039B202980AF088FC00908B4800990160B0F9000089490968F4
:20786000C1EB80208749096801EBA0208549086008460068801200B2834908808048B0F9DA
:20788000020082490968C1EB80208049096801EBA0207E49086008460068801200B27C498A
:2078A00008807C48007C002849D17B480078042845D17A48408840F6B831884210DA784824
:2078C00004607848006810F1040F05DA75480068001D7449086077E000207249086073E0D5
:2078E0006E48408840F68A41884221DA6B484088A0F6B83000EB800040F21A41081A6A497E
:20790000086008460068844201DA204601E0664800686349086063480068801E6149086074
:207920000846006810F5D27F4EDA604808604BE000205B4908605D485A49086044E0574839
:20794000408840F61C41884210DA554804605548006810F1040F05DA52480068001D514966
:20796000086031E000204F4908602DE04B48408840F6EE41884221DA48484088A0F61C4092
:2079800000EB800040F21A41081A4749086008460068844201DA204601E0434800684049BB
:2079A000086040480068801E3E4908600846006810F5D27F08DA3D48086005E00020384981
:2079C00008603A4837490860394A2F48B0F900103348008800B20AF083FB054635480068C5
:2079E000C0EB45203349096801EBE0003149086031484088B7214843C0F3CF1947F69810B8
:207A00007043B9F57A7F02DA4FF47A7100E0494690FBF1FA274800680AEB602547F69810E7
:207A2000854200DD00E02846054628B223490880234A1748B0F900101A48008800B20AF020
:207A40004FFB80461F480068C0EB48201D49096801EBE0001B49086008460068401200B20B
:207A60001649488008460BF02DF81448006800900BF04EF8019001980BF0B2FFBDE8FF87DB
:207A8000280000200C00002020000020100000202200002024150020D6000020C41E00206F
:207AA0000400002008000020240000205CFEFFFF2C06002018000020280A00202C000020B6
:207AC000500600201C00002005F08EF809F094FF0AF034F862B60020124981F83C0009F086
:207AE00043FF72B60AF00AF80AF02EFDFFF704FA00200D4908600846006820F4005000F51A
:207B0000005008600DE0084B41F204120C214FF4E2600CF0B9FBC8200BF042FF034803F060
:207B200091F8F0E72C24002084010020F007002070B505460E46049CAC4208DAFF2E01D186
:207B400000210DE0281B7043C0F5806108E0944202DA4FF4806103E0A01A5843C0F58061FF
:207B6000002901DC002000E00846014688B270BD87B0014600220868009048680190C868F2
:207B800003903D4881423AD04FF0553008600A68B2F1553F02D0002007B070474FF0AA30B2
:207BA00008600A68B2F1AA3F01D00020F4E74FF0553048604A68B2F1553F01D00020EBE77B
:207BC0004FF0AA3048604A68B2F1AA3F01D00020E2E745F25550C860CA6890B245F2555395
:207BE000984201D00020D7E74AF6AA20C860CA6890B24AF6AA23984235D00020CCE70098FF
:207C00006FF30B0000F2555008600A68C2F30B0040F25553984201D00020BDE700986FF383
:207C20000B0000F6AA2008600A68C2F30B0040F6AA23984201D00020AEE7039820F00700CA
:207C4000C01DC860CA6802F00700072801D00020A2E7039820F00700C860CA6802F0070046
:207C600008B1002098E700980860019848600398C860012090E70000001401402DE9F04174
:207C800004460E46154629480078012812D1284801780078401C264A1070264820F8116052
:207CA00010460078322810DB002020490870114608700AE032221F4930460AF0CBF8643074
:207CC00087B22088B84200DD00BF2888C0F3C03050BB208840F2DC51884203DC02F084FFAA
:207CE0001549086002F080FF13490968401A42F21071884218D9286820F4004000F500409D
:207D0000286001200D494880208888800846FFF74DFC00200A4908700A488088401C09496C
:207D20008880022008490870BDE8F08163040020640400208C1D002068040020E4140020BE
:207D400069030020680A002092010020B1F5967F03DA0122044B1A7002E00022024B1A70E3
:207D600001F16402028070476204002010B502460020B2F5FA7F01DC01200EE0B2F5E16FBC
:207D800001DB084609E040F2145393FBF1F4A2F5FA7393FBF4F35B1CD8B210BD10B504466E
:207DA000207800284DD12749087002F01DFF25494860608840F2AA71884236D120792249CF
:207DC000087060794870A0798870E079C870617A207A01EB00201C4988801C48807EEE2892
:207DE00011D10846808820B94FF6FF701849886009E0154880884EF6602191FBF0F0144999
:207E000088600020C870A07A0F498871E07AC87108468079C0F3401018B100200D49087023
:207E20000DE001200B49087009E0608840F2AB71884204D1084861680160A1684160012065
:207E4000207010BD88040020F01D0020E8090020BC030020A10400206C04002010B500BF23
:207E60002A480078052803DA05202849087006E026480078182802DD18202449087023488D
:207E80000078401E43F2C82191FBF0F084B218211F48FCF7BEFC00200BE000FB04F10A22D8
:207EA00091FBF2F101F5FA71194A22F81010411CC8B216490978491E8142EEDC4FF4E16125
:207EC00012480078401E124A22F8101000BF00BF1048807900EB4000C0000A2190FBF1F08B
:207EE0000D4908700B48C07948700A48007B0949C97E08446438084948710448407888701C
:207F000002488078C87000BF10BD000098040020A2040020E80900207404002010B502F079
:207F200063FE40F6B831884206D9C1480078F02802D1C049C87710BDBF48FFF72FFFBF4865
:207F4000007858B902F050FEBC494968401A40F6B831884202D90120B8490870B448007876
:207F6000202823D040285CD080285BD0F02875D1AF480078AF49C87700BF02F035FEB0497E
:207F80000968401AC82809D90120AE490870084600F086F902F028FEA949086000BFA748D7
:207FA000007810B92020A24908703DE1A048007800F0E0009F49C87700BFA3480078052819
:207FC00000DB16E002F010FEA0490968401AC8280ED99F4A9F49A048007800F085F902F0B4
:207FE00003FE9A49086098480078401C9649087000BF00BF9948007890B19848007803288F
:2080000003D140208A4908700AE094480078042803D092480078082802D18020844908706A
:2080200002E100BF8D480078082805D18549087000204880888054E088480078032829D174
:2080400040207B49087003207E49087083484078012804DA82480088488017E0E3E07F48FD
:2080600040787C490978884208DD7A480078401E7B4931F810007349488007E077484078DC
:20808000401E774931F810006E49488000206D49888026E071480078042822D18020644989
:2080A00008700420674908706C48407869494978884204DA67484078624988800EE06748BE
:2080C000407864498978884204DD624880785D49888003E0614840785A498880002059498E
:2080E000488056480078012803D1F0205149C87725E04F480078402812D1564A1178594A91
:208100005278642302FB03F0FFF730FE00F01F004749097801F0E00108444649C8770EE000
:208120004348007880280AD14148007800F0E0004C49497801F01F0108443E49C87700BFB0
:2081400002F052FD48490968401AB0F57A7F39D94248007808280FD144480078052807DAAE
:20816000384800F09DF841480078401C3F49087000203F49087021E03D480078012808DA74
:208180003C4800F07DF83A480078401C3849087011E03748007805280DDA2A4800F080F8D1
:2081A00033480078401C3249087008460078052801DB0020087000202C49087002F014FD06
:2081C0002949086000BF00BF022402F00DFD2A490968401AB0F57A7F23D91F480078012845
:2081E00009D100BF1A4A1B49204600F07DF800202249087011E01848007870B900241F48D3
:208200000078052809DA124A1249204600F06CF81A480078401C1949087002F0E5FC164923
:20822000086000BF00E000BF00BF00BF83E60000A0040020140800207C0400208804002045
:20824000D4040020FA1D0020DC040020D80400207004002098040020A1040020900400202A
:20826000A2040020F01D0020E0040020E5040020E404002074040020E8040020EC04002042
:208280001CB5044600200090019020680090606801900822694640F2AC70FCF78DFE1CBD93
:2082A0001CB5044600200090019020788DF80000608800128DF80100A0788DF80200A088FE
:2082C00000128DF8030020798DF8040000208DF805008DF806008DF807000822694640F216
:2082E000AD70FCF769FE1CBD7FB506460C461546002000900190029003908DF8006020880E
:20830000ADF80100A0788DF8030028788DF804006B4645F210520C2140F213700BF0B4FF14
:208320007FBD000038B5044601234FF47A720A210248009404F012FD38BD0000781D0020C1
:2083400030B503460024002204E033F812502C44551CAAB28A42F8DBB4FBF1F5A8B230BD80
:2083600070B505462A480078012811D100202849087002F039FCB0F5E16F05D902F034FC73
:20838000C8302449088003E04FF4FA602149088002F02AFC1F490988884236D91E480078B6
:2083A000012832D11D48007858B11D480088C82807DC40F2C270854207DD40F63E008542A1
:2083C00003DA00201749C8721CE001201549C872002415E0144830F81400A8420EDB0922A2
:2083E00012A11548FBF77FFB1448015D1248203880F8271000200849087070BD601CC4B2DE
:20840000092CE7DB00200449087000BFF5E700006C0300206A030020D6010020A801002009
:20842000A4010020241500202483010854544B5A303139412E0000007408002036830108BA
:2084400010B502460B460020002107E032F81140844201DD32F811004C1CA1B29942F5DBD6
:2084600010BD10B502460B464FF6FF70002107E032F81140844201DA32F811004C1CA1B203
:208480009942F5DB10BD00000246002108E0064830F81100904201DC08467047481CC1B201
:2084A000C829F4DB0020F8E76E8301080246002108E0064830F81100904201DC0846704777
:2084C000481CC1B2BF29F4DB0020F8E7FE8401082DE9F84F82460D4614461F4600260EE039
:2084E0001C488219A819C1B25046FEF7A5FE401C18B94FF0FF30BDE8F88F701CC6B2A64268
:20850000EEDB21461348FCF723FE81462819C1B26A465046FEF790FE2819401CC1B20DF16A
:2085200001025046FEF788FE9DF801009DF8001000EB01201FFA80F8B8EB090006D1224664
:2085400004493846FBF7ABFA0020D4E74FF0FF30D1E70000501C00202DE9FC5F8046894626
:208560004FF0000A002549464046FFF7E9FE8346002407E038F81400ABEB000505FB05AA39
:20858000601C84B24C45F5DB5046FBF78CFC06460F46304639460EF0B7FCCDE90001FBF7C8
:2085A000CDFC05462846BDE8FC9F0000F8B5044600260020009000BF94F82400012801D1C2
:2085C0000220F8BD012084F8240000BF2046FBF77FFE0646002E62D1A06A20F4885040F09C
:2085E0000200A062022002F043FC30490968B1FBF0F04000009002E00098401E00900098DE
:208600000028F9D12046FBF7CBFE2068806840F008002168886002F0E7FA054611E002F02D
:20862000E3FA401B0A280CD9A06A20F0020040F01000A06200BF002084F8240000BF01202E
:20864000BFE72068806800F008000028E7D12068806840F004002168886002F0C5FA05461B
:2086600011E002F0C1FA401B0A280CD9A06A20F0020040F01000A06200BF002084F824000D
:2086800000BF01209DE72068806800F004000028E7D1A06A20F0020040F00100A06200BF24
:2086A000002084F8240000BF30468AE70000002038B50246002300200090906800B100BFC4
:2086C00000BF92F82400012801D1022038BD012082F8240000BF906890B94868012809D1A9
:2086E0001068806B6FF315000C6840EAC4301468A06338E0906A40F020009062012332E005
:208700000C694868A0421ED84C680869001BC0F1030000EB80041F20A04040F440141068DA
:20872000806BA0434D680C69641BC4F1030404EB84050C68AC400D8A6D1E44EA0554204322
:208740001468A0630FE04C680869001BC0F1030000EB80041F20A04040F440141068806B3E
:20876000A0431468A0631068806800F0010040B91068806847F20104A043CC6920431468B8
:20878000A060886901280FD1C869B0F5E04F06D11068406840F480601468606004E0906AB5
:2087A00040F0200090620123486901280DD1886930B91068406840F480501468606004E07D
:2087C000906A40F020009062012308680A2812D31068C0680C780A3C04EB44050724AC40F9
:2087E000A0430D780A3D05EB45058C68AC4020431468E0600FE0106800690C7804EB440505
:208800000724AC40A0430D7805EB45058C68AC402043146820610868102802D0086811283C
:2088200005D11068806840F400001468A0604868012806D002280DD0032814D004281BD175
:208840001BE0106840696FF30B00CC682043146860611BE0106880696FF30B00CC6820435B
:208860001468A06112E01068C0696FF30B00CC6820431468E06109E000BF1068006A6FF33B
:208880000B00CC6820431468206200BF00BF0868102802D00868112827D1174C1068A042E2
:2088A0001ED11068806800F40000F0B91068806840F400001468A0600868102815D10F48D7
:2088C00000680F4CB0FBF4F000EB80004000009002E00098401E009000980028F9D104E035
:2088E000906A40F020009062012300BF002082F8240000BF1846E9E600240140000000202A
:2089000040420F0010B504460121204600F044F84FF6FF7101EA00101A494880022120469F
:2089200000F03AF84FF6FF7101EA0010154988800321204600F030F84FF6FF7101EA0010AD
:2089400010490880104800880988401A00B20F4908800D4840880B494988401A00B20B4937
:2089600048800948808807498988401A00B2074988800749054809F03BFC0120054908705D
:2089800010BD0000FC0400200E050020140500201A050020080500200246002001290FD0A1
:2089A000022909D0032904D0042908D11368986C09E01368586C06E01368186C03E000BF7F
:2089C0001368D86B00BF00BF7047000070B50446002500BF94F82400012801D1022070BD57
:2089E000012084F8240000BF2046FBF7D9FC0546002D5BD1A06A42F20101884340F4805017
:208A0000A0622E492068884208D12D48006800F4702008B9012002E0002000E0012020B19B
:208A2000A06A20F48010A06203E0A06A40F48010A062A06A00F4807008B90020E06200BF03
:208A4000002084F8240000BF401F216808602068406840F08000216848602068406800F412
:208A6000806010BB2068806800F4E040B0F5E04F15D112492068884208D11148006800F4D2
:208A8000702008B9012002E0002000E0012030B12068806840F40210216888600BE02068E6
:208AA000806840F400402168886004E000BF002084F8240000BF284691E700000028014078
:208AC0000424014038B5024600230020009000BF92F82400012801D1022038BD012082F80B
:208AE000240000BF4868072812D21068406B0C79641E04EB84051F24AC40A0430D796D1E0B
:208B000005EB85050C68AC4020431468606327E048680D2812D21068006B0C79E41F04EBAF
:208B200084051F24AC40A0430D79ED1F05EB85050C68AC4020431468206311E01068C06A39
:208B40000C790D3C04EB84051F24AC40A0430D790D3D05EB85050C68AC4020431468E062F2
:208B600008680A2812D31068C0680C780A3C04EB44050724AC40A0430D780A3D05EB4505CC
:208B80008C68AC4020431468E0600FE0106800690C7804EB44050724AC40A0430D7805EBDB
:208BA00045058C68AC402043146820610868102802D00868112827D1174C1068A0421ED164
:208BC0001068806800F40000F0B91068806840F400001468A0600868102815D10F4800683B
:208BE0000F4CB0FBF4F000EB80004000009002E00098401E009000980028F9D104E0906A80
:208C000040F020009062012300BF002082F8240000BF184661E70000002401400000002087
:208C200040420F002DE9F0410746FE480068401CFC49086008460068B0F5967F01D90020EE
:208C40000860F9480078012805D14120F74948758875C87599E0F648C07A012808D1F5482C
:208C60000078012804D10020F249087008F024FDF1480088F14909680844F0490860EE4803
:208C80008088EF4909680844ED490860EA48408AEC4909680844EB490860EB480088401C98
:208CA000E94908800846008840F6B83188426CDBDF48C07A012822D1E0480068B0FBF1F05B
:208CC00086B23046FFF7F2FBD8494875DC48006840F6B831B0FBF1F086B23046FFF7E6FB69
:208CE000D2498875D748006840F6B831B0FBF1F086B23046FFF7DAFBCC49C8753CE0CF482C
:208D0000006840F6B831B0FBF1F086B23046FFF7BBFBC6494875CA48006840F6B831B0FBD6
:208D2000F1F086B23046FFF7AFFBC0498875C748007801280ED10846407DC5490870C148D5
:208D4000006840F6B831B0FBF1F0C24908800020BE490870BB48006840F6B831B0FBF1F0B8
:208D6000BC490988081A00EB40008001B849097801EBA020AD49C8750020B3490880AF4992
:208D80000860AF490860AF490860AB484088B2490968C1EB8020B049096801EB6020AE496B
:208DA000086008460068801244F2CE714843C0F38F209E49C8800846C0880989C91101EB84
:208DC000C10202EB011108449849C880A348007803280BD10846C088A0F5F850A43840F271
:208DE0007A514843C0F38F209049C8809C48407C01281FD101F0F8FEB0F5FA6F1AD38B482C
:208E0000C0880A2190FBF1F09549488208464069498A08449249486108468069401C8861B5
:208E20000846806943F69821884203D300208C49886148747E48C07A012815D17E48C088B2
:208E400088490988401A49F6192148438512002D01DC002006E049F61920854201DB401E32
:208E600000E02846054613E07348C0887D490988401A4CF250314843C512002D01DC002067
:208E800005E04CF25030854200DB00E02846054675480068C0EB85207349096801EB6020E6
:208EA0007149086008460068C0F38F205F4908816E48007807287DD2DFE800F0045592F702
:208EC000FEF5F4005C4800896949C98A401A642148436749097E90FBF1F004B2002C01DCAD
:208EE000002000E0204604461C2094FBF0F04F4908772546504840895E49C98A401A64215B
:208F000048435C49097E90FBF1F004B2002C01DC002000E0204604461C2094FBF0F0434988
:208F200048772544444880895349C98A401A642148435149097E90FBF1F004B2002C01DCCF
:208F4000002000E0204604461C2094FBF0F0374988772544002D01DC002002E0032095FB0F
:208F6000F0F0054630E1344840894249C98A401A642148433F49097E90FBF1F004B2002CCB
:208F800001DC002000E0204604461C2094FBF0F0264948772546284880893749C98A401A5A
:208FA000642148433449097E90FBF1F004B2002C03DC00E006E1002000E0204604461C20BD
:208FC00094FBF0F01949887728190546002D01DC002103E0284600EBD07149100D46F3E00E
:208FE000154800892249C98A401A642148432049097E90FBF1F004B2002C01DC002000E048
:20900000204604461C2094FBF0F0084908772546094880891849C98A401A642148431649E3
:20902000097E2BE024050020D601002014080020241500204C050020C41E002038050020F9
:20904000340500203C0500203005002040050020410500204205002028050020D001002091
:2090600000030020200500202C050020E8030020C4150020DE150020F815002090FBF1F087
:2090800004B2002C01DC002000E0204604461C2094FBF0F06B49887728190546002D05DC69
:2090A000002107E075E05BE006E040E0284600EBD07149100D4687E0634800896349C98A32
:2090C000401A642148436149097E90FBF1F004B2002C01DC002000E0204604461C2094FB4F
:2090E000F0F0584908772546574840895849C98A401A642148435649097E90FBF1F004B2F7
:20910000002C01DC002000E0204604461C2094FBF0F04C49487728190546002D01DC0021E0
:2091200003E0284600EBD07149100D464CE0464880894849C98A401A642148434549097EE0
:2091400090FBF1F004B2002C01DC002000E0204604461C2094FBF0F03A498877254633E089
:20916000394840893A49C98A401A642148433849097E90FBF1F004B2002C01DC002000E032
:20918000204604461C2094FBF0F02E49487725461AE02D4800892D49C98A401A64214843A8
:2091A0002A49097E90FBF1F004B2002C01DC002000E0204604461C2094FBF0F02149087746
:2091C000254601E0002500BF00BF23490D8023480078D8B91C48008A21490988451A002DBE
:2091E00001DC002000E0284605461E480068C0EB85201C49096801EB20201A4908600846A0
:209200000068C0F38F201449488002E00020124948800D48C08914490968C1EB8020124927
:20922000096801EB60201049086008460068C0F38F200E4908800449488809F0B9F8BDE82D
:20924000F081000014080020C41E0020C4150020DE150020F81500200A0500206204002071
:20926000600400204405002048050020D40100207047704710B504462068406800F02000E2
:2092800020282FD12068006800F00200022829D1A06A00F0100018B9A06A40F40070A062F5
:2092A0002068806800F46020B0F5602F13D1E06888B92068406820F0200021684860A06A8E
:2092C00020F48070A062A06A00F4805018B9A06A40F00100A0622046FFF7A4FC6FF012003F
:2092E000216808602068406800F0800080283BD12068006800F00400042835D1A06A00F019
:20930000100018B9A06A40F40050A0622068806800F4E040B0F5E04F0DD02068406800F483
:209320008060D0B92068806800F46020B0F5602F13D1E06888B92068406820F080002168F6
:209340004860A06A20F48050A062A06A00F4807018B9A06A40F00100A0622046FFF7D2FA51
:209360006FF00C00216808602068406800F0400040280FD12068006800F0010050B1A06AFD
:2093800040F48030A062204600F0A8F86FF001002168086010BD00002DE9F041044600271B
:2093A00000250026A84614B90120BDE8F081A06810B1606900B100BFA06A30B90020E06219
:2093C00084F82400204600F08BF82046FAF780FF0746A06A00F01000002873D1002F71D10A
:2093E000A06A20F4885040F00200A062E16960680843E16840EA41000643A068B0F5807F3D
:2094000002D0A068012802D14FF4807000E0002005436069012811D1E06838B9A069401E87
:209420004FF4006141EA4030054307E0A06A40F02000A062E06A40F00100E0622068406875
:2094400020F469402843216848602068806821490840304321688860A068B0F5807F02D02F
:20946000A068012802D14FF4807000E00020B0F5807F03D1208A401E4FEA00582068C06AF2
:2094800020F4700040EA08002168C8622068806811490840B04208D10020E062A06A20F00A
:2094A000020040F00100A06211E0A06A20F0020040F01000A062E06A40F00100E062012743
:2094C00005E0FFE7A06A40F01000A062012738466BE70000FDF7E1FFFE0E1FFF70470000C8
:2094E00010B586B004463249206888423CD100BF3048806940F400702E49886108468069F2
:2095000000F40070019000BF00BF3F2002900320039002A9284801F0C7F9B02002900320E0
:20952000039002A9254801F0BFF9254825490860002048600021234881608021C160490054
:20954000016189004161202181610021C16100F0DFFF20B14FF497711BA00DF06BF800BF54
:2095600018482062446221E01C49206888421DD100BF1048806940F480600E49886108461B
:20958000806900F48060019000BF00BF0E2002900320039002A9094801F086F901221146A3
:2095A000122001F0F0FB122001F0E0FB06B010BD00240140001002400010014000080140CB
:2095C00008000240501F00202E2E5C436F72655C5372635C6164632E63000000002801406F
:2095E00070B50446002500BF94F82400012801D1022070BD012084F8240000BF2046FAF747
:20960000CFFE0546002D77D1A06A40F20121884340F48070A0623C492068884208D13B483B
:20962000006800F4702008B9012002E0002000E0012078B1A06A20F48010A0622068406850
:2096400000F4806000B3A06A20F4005040F48050A06219E0A06A40F48010A0622B49091FAA
:209660002068884203D028492068884204D12748006800F4806000E0002028B1A06A20F48B
:20968000005040F48050A062A06A00F4805020B1E06A20F00600E06201E00020E06200BF31
:2096A000002084F8240000BFC01E216808602068806800F46020B0F5602F16D1124920687A
:2096C000884208D11148006800F4702008B9012002E0002000E0012038B12068806840F430
:2096E000A000216888600CE006E02068806840F480102168886004E000BF002084F824007F
:2097000000BF284675E7000000280140042401402DE9F04104460D4616460027574920685F
:20972000884203D056492068884205D15348001D006800F4702000E0002000287ED100BFEB
:2097400094F82400012802D10220BDE8F081012084F8240000BF2046FAF722FE0746002FB2
:209760006DD1A06A40F60161884340F48070A06243492068884209D14048001D006800F45F
:20978000702008B9012002E0002000E0012078B1A06A20F48010A0622068406800F4806077
:2097A00000B3A06A20F4005040F48050A06219E0A06A40F48010A06230492068884203D01B
:2097C0002F492068884205D12C48001D006800F4806000E0002028B1A06A20F4005040F4A1
:2097E0008050A062A06A00F4805020B1E06A20F00600E06201E00020E06200BF002084F8B8
:20980000240000BF1F48216A88621F48216AC8621E48216A08636FF0020021680860206837
:20982000806840F4807021688860226802F14C0133462A46206A00F0A3FE01E01AE014E00E
:209840002068806800F46020B0F5602F06D12068806840F4A000216888600CE02068806808
:2098600040F480102168886005E000BF002084F8240000E00127384667E700000024014016
:209880000028014023430008934300087543000830B5024600230C7D012000FA04F31068F0
:2098A000D0F8000220F47C5001254C6A45EA042420431468C4F800021068D0F81C029843F5
:2098C0001468C4F81C02C869E8B91068D0F80C0298431468C4F80C02888880B28C8940EA70
:2098E0000444106800F510704D6940F83540088880B20C8940EA0444106800F510704D6964
:2099000000EBC5004460C86901281DD11068D0F80C0218431468C4F80C02888880B20C88E6
:2099200040EA0444106800F510704D6940F83540888980B20C8940EA0444106800F510702E
:209940004D6900EBC5004460886938B91068D0F8040298431468C4F8040206E01068D0F896
:20996000040218431468C4F80402086938B91068D0F8140298431468C4F8140206E0106809
:20998000D0F8140218431468C4F81402086A012806D11068D0F81C0218431468C4F81C02BF
:2099A0001068D0F8000220F001001468C4F80002002030BD0168496941F0020102685161A2
:2099C0000168496941F0100102685161704700002DE9F0410446002500260027A8462068DE
:2099E000C068C0F3001520684069C0F3C0062DB126B148F4007810202168C8602068006992
:209A0000C0F3001520684069C0F380162DB126B148F480681020216808612068406900F0E8
:209A2000010000283BD0206880687A490840884201D1012000E00020054620688068764940
:209A40000840884201D1012000E0002006462068806872490840884201D1012000E0002085
:209A600007460DB906B9D7B120688068C0F3400520688068C0F340262068806800F0010733
:209A80000DB906B91FB12046FBF702FB01E048F40068206880686249084321688860206838
:209AA000C06800F0030520684069C0F3400625B11EB100212046FBF799F82068006900F0CC
:209AC000030520684069C0F3001625B11EB101212046FBF78BF8206C40EA08002064206818
:209AE000806900F0010520684069C0F3002620684069C0F3C0372DB126B11FB1206C40F061
:209B00000100206420688069C0F3400520684069C0F3402620684069C0F3C0372DB126B17D
:209B20001FB1206C40F00200206420688069C0F3800520684069C0F3802620684069C0F3FC
:209B4000C0372DB126B11FB1206C40F0040020642068806900F0700008B9012000E0002092
:209B6000054620684069C0F3C02620684069C0F3C03795BB8EB387B32068806900F0700554
:209B8000402D1BD006DC102D09D0202D0CD0302D24D10EE0502D16D0602D1FD118E0206CA8
:209BA00040F0080020641AE0206C40F01000206415E0206C40F02000206410E0206C40F09E
:209BC000400020640BE0206C40F08000206406E0206C40F48070206401E007E000BF00BFB6
:209BE0002068806920F0700021688861206C78B1042021684860012084F83C0020684069EE
:209C000048F65B718843216848612046FFF7D2FEBDE8F081010000040001000800000110DC
:209C2000090501002DE9F041044600270026002514B90120BDE8F08194F83C0028B9002045
:209C400084F83D00204600F0A5F8022084F83C002068006820F0020021680860206800689B
:209C600040F001002168086000F0BEFF06460EE000F0BAFF801B0A2809D9032084F83C00A8
:209C800000BF002084F83D0000BF0320D2E72068406800F001000028EAD02068406800F06E
:209CA0000100002867D0A069012802D145F0800501E025F08005E069012802D145F040054B
:209CC00001E025F04005206A012802D145F0200501E025F02005606A012802D145F010053E
:209CE00001E025F01005A06A012802D145F0080501E025F00805E06A012802D145F004058A
:209D000001E025F004052068006820F0FC00284321680860D4E90201084321690843616942
:209D200008436168491E08432168C8612068006820F001002168086000F056FF06460EE03A
:209D400000F052FF801B0A2809D9032084F83C0000BF002084F83D0000BF03206AE72068E5
:209D6000406800F001000028EAD12068406800F0010000B90127012F06D100202064012099
:209D800084F83C00002055E7042084F83C00012050E7000010B586B004462D49206888426E
:209DA00054D100BF2B48C06940F000702949C8610846C06900F00070019000BF00BF881565
:209DC000029000200390049002A9234800F06CFD4FF400700290022003900320059002A9DE
:209DE0001D4800F061FD00BF1C49486820F4C04040F0E06040F48040486000BF0122114683
:209E0000142000F0C0FF142000F0B0FF01221146152000F0B8FF152000F0A8FF104820638F
:209E2000104860631048A063FAF774FE0F480068406940F002000D49096848610B48006884
:209E4000406940F0100009490968486106B010BD0064004000100240000C014000000140A6
:209E6000CC1F0020E81F00200C2000202C240020816B896811B9416B096941B91649096865
:209E8000496941F01001144A126851617047816B0968A1F2AA7111B1012911D100E000BF15
:209EA000816B096908290AD100210C4A1170816B09885180816B4B6953608969916000E0DC
:209EC00000BF00BF04490968496941F01001024A1268516100BFD9E72C2400207C0400204B
:209EE00010B50446606B806810B9606B006940B92E480068406940F002002C490968486162
:209F000010BD606B006840F23172811A904214D009DCA0F2516080B3CF2818D0D02817D002
:209F2000DF2837D108E00F291CD010291BD01F2924D020292ED122E000BF606B00881C49E5
:209F40000880606B017C1A48FBF710F823E000BF606B008817490880606B017C1548FBF741
:209F600005F818E000BF606B008813490880606B017C1148FAF7FAFF0DE001E000BF00BF1F
:209F8000606B00880D490880606B017C0B48FAF7EDFF00E000BF00BF04480068406940F02D
:209FA000020002490968486100BFA9E72C240020780500208C050020A0050020B40500208F
:209FC0002DE9F04104460E46042500272068806800F08060B0F1806F0DD02068806800F03F
:209FE0000060B0F1006F06D02068806800F08050B0F1805F7ED100BF94F83D00012802D198
:20A000000220BDE8F081012084F83D0000BF94F83C00222804D0322806D062280CD107E00B
:20A02000422084F83C000BE0522084F83C0007E0722084F83C0003E0122084F83C0000BF34
:20A0400000BF2068806800F0806008B1002507E02068806800F0006008B1012500E0022596
:20A06000206800F5C07000EB0510006800F00101206800F5C07000EB05100160206B806858
:20A0800098B9206800F5C07000EB05100068216BC968226B128841EA42510843216801F5EE
:20A0A000C07101EB0511086015E0206800F5C07000EB05100068216B8968226B526841EA0C
:20A0C000C201226BD26811430143206800F5C07000EB05100160206B007C00F00F00216BBE
:20A0E0000861206800F5C07000EB0510406820F00F0100E0B1E0206800F5C07000EB051064
:20A100004160206800F5C07000EB05104068216B09690843216801F5C07101EB05114860A6
:20A12000206BC07D0106206B807D41EA0041206B407D41EA0020216B097D0843216801F5ED
:20A14000C07101EB05118860206BC07E0106206B807E41EA0041206B407E41EA0021206BFF
:20A16000007E0143206800F5C07000EB0510C160206800F5C07000EB0510006840F0010108
:20A18000206800F5C07000EB0510016000F02CFD074620E0701CF0B126B100F025FDC01B5A
:20A1A000B04218D9032084F83C001DB980202168886009E0012D03D1E8032168886003E0D0
:20A1C0004FF400002168886000BF002084F83D0000BF032015E74DB920688068214908402D
:20A1E000884201D1012016E0002014E0012D09D1206880681C490840884201D101200AE0CC
:20A20000002008E02068806818490840884201D1012000E000200028BCD094F83C0042287A
:20A2200004D0522806D072280CD107E0222084F83C000BE0322084F83C0007E0622084F8C8
:20A240003C0003E0012084F83C0000BF00BF00BF002084F83D0000BFD3E6042084F83C009C
:20A260000120CEE6010000040001000800000110704710B504460CB9012010BD607920B9BF
:20A2800000202071204600F005F8012060710020F3E7000008B5094A016891420DD100BFE5
:20A2A0000749496941F04001054A51611146496901F04001009100BF00BF08BD00300240A8
:20A2C0000010024070B50446002594F82100022803D00420A063012548E02068006820F079
:20A2E0000E00216808602068006820F00100216808601F492068884201D1012026E01C4955
:20A3000014312068884201D110201FE0184928312068884201D1801518E015493C312068E7
:20A32000884201D1801411E0114950312068884202D14FF4803009E00D49643120688842E3
:20A3400002D14FF4801001E04FF08070084908394860012084F8210000BF002084F82000D4
:20A3600000BF606B10B12046616B8847284670BD0800024070B50446E06B0568206806688F
:20A3800094F84010042088402840002846D006F00400002842D02068006800F0200028B93A
:20A3A0002068006820F004002168086057492068884201D1042027E0544914312068884285
:20A3C00001D1402020E0514928312068884201D1001519E04D493C312068884202D14FF4BB
:20A3E000804011E0494950312068884202D14FF4802009E0454964312068884202D14FF41D
:20A40000800001E04FF08060404908394860E06A00287AD02046E16A884776E094F84010DC
:20A42000022088402840A0B306F0020088B32068006800F0200040B92068006820F00A0041
:20A4400021680860012084F8210030492068884201D1022028E02D4914312068884201D1A7
:20A46000202021E0294928312068884201D140151AE026493C312068884202D14FF40050C9
:20A4800012E0224950312068884203D14FF400300AE017E01D4964312068884202D14FF401
:20A4A000001001E04FF0007018490839486000BF002084F8200000BFA06A30B32046A16A1A
:20A4C000884722E094F84010082088402840E0B106F00800C8B12068006820F00E002168D8
:20A4E000086094F8401001208840E16B48600120A06384F8210000BF002084F8200000BF40
:20A50000206B10B12046216B884770BD080002400146002209B901207047184B0868C01A07
:20A520001423B0FBF3F08000086414480838C863022081F821000868026843F6F0708243AF
:20A54000D1E901031843CB6818430B6918434B6918438B691843CB69184302430868026081
:20A5600000208862C862086348638863012081F82100002081F8200000BFCDE70800024075
:20A580002DE9F04104460D4616461F464FF0000800BF94F82000012802D10220BDE8F08130
:20A5A000012084F8200000BF94F8210001282CD1022084F821000020A0632068006820F06A
:20A5C0000100216808603B46324629462046FBF7ADFBE06A30B12068006840F00E0021683F
:20A5E00008600BE02068006820F00400216808602068006840F00A00216808602068006808
:20A6000040F001002168086006E000BF002084F8200000BF4FF002084046BFE770B5044614
:20A6200000F0E2FA06462546681C10B104480078054400BF00F0D8FA801BA842FAD370BD45
:20A64000580000202DE9F04104460E460127002500BF2648007E012802D10220BDE8F08171
:20A6600001202249087600BF2068022813D14CF25030FDF765F890BB0120FCF7E7FF4CF2E9
:20A680005030FDF75DF807461948006920F004001749086123E04CF25030FDF751F8F0B956
:20A6A0004FF0FF303060A56812E02846FCF7E2FF4CF25030FDF744F807460D48006920F052
:20A6C00002000B4908610FB1356007E005F58065D4E9021001EB8020A842E6D800BF00BF1F
:20A6E00000200249087600BF3846B7E708070020002002400348006940F0800001490861EE
:20A7000000207047002002402DE9FE4F05468B4617469846012600240020029000BF24481E
:20A72000007E012802D10220BDE8FE8F01202049087600BF4CF25030FDF702F8064686BB4B
:20A74000012D02D10120029006E0022D02D10220029001E00420029000241EE02201B946CE
:20A76000C24648465146F9F78AF980B20190022000FB04B000900199FCF790FF4CF250303B
:20A78000FCF7DEFF06460B48006920F001000949086106B104E0601CC4B202988442DDDB70
:20A7A00000BF00BF00200249087600BF3046BBE7080700200020024000200849096901F0F6
:20A7C000800151B10649054A5160064951601146096901F0800101B1012070470020024080
:20A7E00023016745AB89EFCD10B50446042C3BD100202149C8700846807840B900F0F4F970
:20A800001D494860601F88600120887011E000F0EBF919494968401A1749886008468068FA
:20A820004B2802D215480068886000F0DDF91249486011488068114908600F4880684B28A6
:20A8400018D30F480068401C0D4908600D48007E08B9012001E00B48007E09490968B1FB5E
:20A86000F0F00549C86005E0B4F5805F02D101200549087010BD0000BC0300207405002016
:20A8800070050020E8090020A402002010B5044604480068204020B1024804602046FFF74E
:20A8A000A3FF10BD140401402DE9F84703460024002000258446002700226EE14FF001081F
:20A8C00008FA02F4D1F8008008EA0400A0427DD1DFF8D0A2D1F80480A8EB0A09D0453AD0B6
:20A8E00014DCB8F1030F50D009DCB8F1000F31D0B8F1010F1CD0B8F1020F49D120E0B8F1CD
:20A90000110F18D0B8F1120F42D11EE0B9F5881F25D006DCB9F5803F20D0B9F5801F37D176
:20A920001AE0B9F5001F18D0B9F5041F30D117E0D1F80CC02DE0D1F80C8008F1040C28E097
:20A94000D1F80C8008F1080C23E0D1F80C8008F10C0C1EE000BF00BF00BF00BF00BF00BFB4
:20A96000D1F80880B8F1000F02D14FF0040C0BE0D1F80880B8F1010F03D14FF0080C1C6113
:20A9800002E04FF0080C5C6103E04FF0000C00E000BF00BFFF2801D8984601E003F104087A
:20A9A0004646FF2802D84FEA820803E0A2F108084FEA88084746D6F800804FF00F0909FAC3
:20A9C00007F928EA09080CFA07F900E088E048EA0908C6F80080D1F8048008F08058B8F1BF
:20A9E000805F7DD100BFDFF8C081D8F8188048F00108DFF8B491C9F81880C846D8F81880BF
:20AA000008F00108CDF8008000BF00BF4FEAB9384FEA920958F829504FEA82784FEA1879AE
:20AA20004FF00F0808FA09F825EA0805DFF87C81434502D14FF0000816E0DFF874814345E1
:20AA400002D14FF001080FE0DFF86881434502D14FF0020808E0DFF86081434502D14FF04E
:20AA6000030801E04FF004084FEA82794FEA197908FA09F848EA0505DFF840814FEA9209F5
:20AA800048F82950D1F8048008F48038B8F5803F0AD1DFF82C81D8F8008048EA0008DFF8D0
:20AAA0002091C9F8008009E0DFF81481D8F8008028EA0008DFF80891C9F80080D1F80480E7
:20AAC00008F40038B8F5003F10D1DFF8F48008F10408D8F8008048EA0008DFF8E49000E070
:20AAE0005AE009F10409C9F800800DE0DFF8D08008F10408D8F8008028EA0008DFF8C0902A
:20AB000009F10409C9F80080D1F8048008F48018B8F5801F0ED1DFF8A88008F10808D8F809
:20AB2000008048EA0008DFF8989009F10809C9F800800DE0DFF8888008F10808D8F80080EB
:20AB400028EA0008DFF8789009F10809C9F80080D1F8048008F40018B8F5001F0ED1DFF8CD
:20AB6000608008F10C08D8F8008048EA0008DFF8509009F10C09C9F800800DE0DFF84080D3
:20AB800008F10C08D8F8008028EA0008DFF8309009F10C09C9F80080521C102AFFF48EAE80
:20ABA000BDE8F887000011100010024000080140000C014000100140001401400800014079
:20ABC00000040140024693680B400BB1012000E000207047C2684A40C26070470AB1016164
:20ABE00001E00B040361704701480068704700005000002070B504460CB9012070BD4CF6AE
:20AC0000CC402168086045F2555021680860D4E9001048602168A0688860FFF7E5FF054657
:20AC200006E0FFF7E1FF401B302801D90320E5E72068C0680028F4D14AF6AA202168086044
:20AC40000020DBE701464AF6AA200A681060002070470000034800680349097808440149F2
:20AC600008607047500000205800002010B50848006840F0100006490860032000F0C2F88C
:20AC8000002000F007F800F02BF8002010BD00000020024070B504460E4800784FF47A71D8
:20ACA000B1FBF0F00C490968B1FBF0F5284600F083FE08B1012070BD102C07D2002221462D
:20ACC000501E00F060F80548046001E00120F2E70020F0E75800002000000020540000202F
:20ACE00008B500BF1F48806940F001001D4988610846806900F00100009000BF00BF0320AF
:20AD000000F080F8002211466FF00B0000F03BF8002211466FF00A0000F035F8002211464D
:20AD20006FF0090000F02FF800221146501F00F02AF800221146101F00F025F8002211466C
:20AD4000901E00F020F800221146501E00F01BF800BF0549486820F0E06040F000704860FE
:20AD600000BF08BD001002400000014000BF00F01F02012191404209920002F1E022C2F86D
:20AD8000001100BF70472DE9F05F80460D461646002707F07BF8074639462A46334601F01B
:20ADA0000700C0F1070ABAF1040F02D94FF0040A01E0C0F1070AD14600F1040ABAF1070F6A
:20ADC00002D24FF0000A01E0A0F1030AD4464FF0010A0AFA09FAAAF1010A0AEA020A0AFAC2
:20ADE0000CFA4FF0010B0BFA0CFBABF1010B0BEA030B4AEA0B042146404607F04FF8BDE838
:20AE0000F09F000000BF00F00702064B19684FF6FF031940044B0B4343EA0221014B1960C7
:20AE200000BF70470CED00E00000FA0500BF00BF00BF00BF00BFBFF34F8F00BF00BF00BF3C
:20AE40000948006800F4E06008490843001D0649086000BF00BF00BFBFF34F8F00BF00BF4A
:20AE600000BF00BF00BFFDE70CED00E00000FA052DE9F04385B006463DA30FCB01AC0FC4D5
:20AE80003FA0006800904FF00008002500270024A146012E30D0022E58D0102E61D13948C5
:20AEA0004468006800F0807000B301A8C4F38341475C04F4803070B132484068C0F3404006
:20AEC0001DF8008004F4803040B12F48B0FBF8F000FB07F502E02D4807FB00F529484068DC
:20AEE00000F48000B0F5800F01D1A94603E068000321B0FBF1F935E02248046A04F4407050
:20AF0000B0F5807F05D104F0020010B14FF400491BE004F44070B0F5007F07D11948406ACA
:20AF200000F0020010B149F640490EE004F44070B0F5407F07D11348006800F4003010B11C
:20AF40004FF2244901E04FF000090BE000F0A0F90C494968C1F38131491C4900B0FBF1F9F7
:20AF600000E000BF00BF484605B0BDE8F083000002030405060708090A0B0C0D0E0F101081
:20AF8000010200000010024000127A0000093D00F8B5044600260025207800F00100002897
:20AFA0006BD000274348C06900F0805070B900BF4048C06940F080503E49C8610846C069FB
:20AFC00000F08050009000BF00BF01273A48006800F48070B0B93848006840F480703649B9
:20AFE0000860FFF701FE064606E0FFF7FDFD801B642801D90320F8BD2F48006800F4807036
:20B000000028F2D02B48006A00F440752DB3A08800F44070A84220D02648006A20F4407599
:20B02000012026490860002008602248056205F0010090B1FFF7D8FD064608E0FFF7D4FDC2
:20B04000801B41F28831884201D90320D3E71948006A00F002000028F0D01648006A20F467
:20B0600040706168084313490862012F04D10846C06920F08050C86100BF207800F0020078
:20B08000022807D10B48406820F44040A168084308494860207800F01000102807D10548DD
:20B0A000406820F48000E1680843024948600020A1E700000010024000700040400442425B
:20B0C00070B504460D4600266248006800F00700A8420ED25F48006820F0070028435D497E
:20B0E00008600846006800F00700A84201D0012070BD207800F00200022807D15648406860
:20B1000020F0F000A168084353494860207800F0010000285DD06068012806D14E480068F3
:20B1200000F4003090B90120E2E76068022806D14948006800F0007040B90120D8E746482F
:20B14000006800F0020008B90120D1E74248406820F00300616808433F494860FFF744FD3B
:20B1600006466068012810D108E0FFF73DFD801B41F28831884201D90320B9E73648406885
:20B1800000F00C000428F0D123E06068022810D108E0FFF729FD801B41F28831884201D9C1
:20B1A0000320A5E72C48406800F00C000828F0D10FE008E0FFF718FD801B41F288318842A4
:20B1C00001D9032094E72448406800F00C000028F0D12048006800F00700A8420ED91D4801
:20B1E000006820F0070028431A4908600846006800F00700A84201D0012079E7207800F029
:20B200000400042807D11448406820F4E060E168084311494860207800F00800082808D19F
:20B220000D48406820F46050216940EAC1000A49486000F03DF808494968C1F30311074A9D
:20B24000515CC840064908600020FFF723FD00204EE700000020024000100240A07001082A
:20B260000000002001480068704700000000002000B5FFF7F7FF04494968C1F30221034A63
:20B28000515CC84000BD000000100240B070010800B5FFF7E7FF04494968C1F3C221034A4E
:20B2A000515CC84000BD000000100240B0700108F0B585B00FF26C0C9CE8E01001A8A0E8A9
:20B2C000E0101CA52D68009500210022002300240020194D696801F00C05F5B1042D02D007
:20B2E000082D19D101E0154819E001ADC1F38346AC5D01F4803555B10F4D6D68C5F34045A6
:20B300001DF805200D4D6543B5FBF2F302E00C4D04FB05F3184602E000BF084800BF00BF5D
:20B3200005B0F0BD02030405060708090A0B0C0D0E0F1010010200000010024000127A0033
:20B3400000093D00F8B504460025207800F00100002878D0F848406800F00C0004280CD0A6
:20B36000F548406800F00C00082811D1F248406800F48030B0F5803F0AD1EF48006800F482
:20B38000003000285FD0606800285CD10120F8BD00BF6068B0F5803F06D1E748006840F4A6
:20B3A0008030E549086028E0606858B9E248006820F48030E04908600846006820F4802015
:20B3C00008601AE06068B0F5A02F0BD1DA48006840F48020D84908600846006840F4803072
:20B3E00008600AE0D448006820F48030D24908600846006820F48020086000BF606888B19E
:20B40000FFF7F2FB054606E0FFF7EEFB401B642801D90320BBE7C848006800F400300028EF
:20B42000F2D010E0FFF7E0FB054606E0FFF7DCFB401B642801D90320A9E7BF48006800F4B4
:20B4400000300028F2D1207800F00200022857D1B948406800F00C0050B1B748406800F0B8
:20B460000C00082818D1B448406800F4803098B9B148006800F0020020B12069012801D067
:20B48000012084E7AC48006820F0F800616940EAC100A949086033E02069E8B10120A74967
:20B4A0000860FFF7A1FB054606E0FFF79DFB401B022801D903206AE79F48006800F00200BF
:20B4C0000028F2D09C48006820F0F800616940EAC1009949086013E0002098490860FFF7DD
:20B4E00083FB054606E0FFF77FFB401B022801D903204CE79048006800F002000028F2D15B
:20B50000207800F0080008282DD1A069B8B101208B490860FFF768FB054606E0FFF764FBBF
:20B52000401B022801D9032031E78348406A00F002000028F2D0012007F022F813E00020DB
:20B540007F490860FFF750FB054606E0FFF74CFB401B022801D9032019E77748406A00F031
:20B5600002000028F2D1207800F00400042873D100267148C06900F0805070B900BF6E487C
:20B58000C06940F080506C49C8610846C06900F08050009000BF00BF01266A48006800F42A
:20B5A0008070B0B96748006840F4807065490860FFF71AFB054606E0FFF716FB401B6428B7
:20B5C00001D90320E3E65F48006800F480700028F2D000BFE068012806D15748006A40F088
:20B5E00001005549086227E0E06858B95248006A20F00100504908620846006A20F00400FE
:20B60000086219E0E06805280BD14B48006A40F00400494908620846006A40F001000862F6
:20B620000AE04548006A20F00100434908620846006A20F00400086200BFE068A0B1FFF79E
:20B64000D3FA054609E0FFF7CFFA401B41F28831884202D903209AE622E03748006A00F0C0
:20B6600002000028EFD012E0FFF7BEFA054608E0FFF7BAFA401B41F28831884201D9032056
:20B6800085E62D48006A00F002000028F0D1012E05D12948C06920F080502749C86100BFAE
:20B6A000E069C8B32448406800F00C00082860D0E069022848D1002020490866FFF794FA4F
:20B6C000054606E0FFF790FA401B022801D903205DE61948006800F000700028F2D1206A56
:20B6E000B0F5803F07D11448406820F40030A168084311494860D4E9080108430E49496857
:20B7000021F4741108430C49486001200B490866FFF76AFA054607E02DE0FFF765FA401B1B
:20B72000022801D9032032E60348006800F000700028F2D01FE000000010024000004242F8
:20B74000800442420070004000200C490866FFF74BFA054606E0FFF747FA401B022801D94C
:20B76000032014E60648006800F000700028F2D101E001200BE6002009E600000000424225
:20B7800000100240042808D14FF0E021096941F004014FF0E022116107E04FF0E02109691E
:20B7A00021F004014FF0E022116170470EB563480078012800D10EBD6148407E08B9022014
:20B7C00001E05F48407E02465D48418801235D48F9F72CFD5C48007830B95C4A11885C4AA1
:20B7E00010885C4A03F01AFD5B485C490978CDE900105B48027856480068029059480378A1
:20B8000051480078029903F03BFA53480078C0435549087050488079C04388714E48B0F95C
:20B820000200C04348804C48B0F90400C04388804E480078D0B94E48027E4E480189454B92
:20B840004B48163009F0F0FB4B48027E49484189404B4948163009F049FC4848027E454880
:20B8600081893C4B4548163009F0A2FC4448007828B94048018A374A4248FCF7FFF9424954
:20B880004248F8F7CFFD424805F0B6FD41480088401C4049088008460088052801DB0020B4
:20B8A00008803D480088401C3B490880084600880A2809DB00200880244B1A88997A5B88F0
:20B8C00098B2364BF9F7B6F835480088401C3449088008460088322804DB00200880314869
:20B8E000F9F7BEFD30480088401C2F49088008460088642809DB00200880124908780A224C
:20B900002A4906F0A7FA1149887229480088401C2749088008460088C82801DB0020088032
:20B9200024480088401C2349088008460088B0F57A7F01DB0020088000BF3CE75C0000206D
:20B94000E80900208C030020D0000020140800200A05002084010020D600002029040020E4
:20B96000D200002028040020DE000020EC030020C4150020C41E0020DE150020F815002041
:20B98000620400206004002002050020DA1E0020080B00205E00002060000020DC01002030
:20B9A00062000020A40100206400002038150020660000206800002070B504462546681EE1
:20B9C000B0F1807F01D301200FE0681E4FF0E02148610F214FF0FF3006F060FA00204FF027
:20B9E000E021886107200861002070BD10B5FFF7DDFE10BD7047704710B50346002200BFC0
:20BA000093F83C00012801D1022010BD012083F83C0000BF22F0FF00CC6840EA040222F453
:20BA200040708C6840EA040222F480604C6840EA040222F400600C6840EA040222F4805058
:20BA40000C6940EA040222F400504C6940EA040222F480408C6940EA040222F400408C69B0
:20BA600040EA04021868426400BF002083F83C0000BF00BFC9E7024600BF92F83C000128B6
:20BA800001D102207047012082F83C0000BF022082F83D001068406820F0700013685860B9
:20BAA000106840680B681843136858601068806820F0800013689860106880684B68184394
:20BAC00013689860012082F83D0000BF002082F83C0000BF00BFD5E770B504460D46042264
:20BAE0002946206809F00AF82068406C40F40040216848642068006840F001002168086065
:20BB0000002070BD70B504460D4600222946206808F0F4FF00BF2068006A41F211110840C4
:20BB200050B92068006A8910084028B92068406C20F400402168486400BF00BF2068006A1B
:20BB400041F21111084050B92068006A8910084028B92068006820F001002168086000BFDA
:20BB6000002070BD10B504460CB9012010BD94F83D0028B9002084F83C00204600F00CF8DA
:20BB8000022084F83D00211D206808F06FFF012084F83D000020E9E710B586B00446324914
:20BBA0002068884233D100BF3048806940F400602E4988610846806900F40060019000BF40
:20BBC00000BF8814029000200390049002A92848FEF76AFE4FF460400290022003900590FA
:20BBE00002A92348FEF760FE4FF47060029002200390059002A91F48FEF756FE0122114618
:20BC00001920FFF7C0F81920FFF7B0F829E02068B0F1804F25D100BF1448C06940F00100FA
:20BC20001249C8610846C06900F00100019000BF00BF00BF0846806940F0040088610846A8
:20BC4000806900F00400019000BF00BF012002900020039004900220059002A90548FEF75A
:20BC600023FE06B010BD0000002C014000100240000C0140000801400146022081F83D00AC
:20BC80000868006840F001000A681060012081F83D000020704701460868C06840F00100FB
:20BCA0000A68D0600868006840F001000A681060002070472DE9F04104460D46002600BF57
:20BCC00094F83C00012802D10220BDE8F081012084F83C0000BF022084F83D00206886687F
:20BCE00026F0770626F47F4620688660286850283BD00CDC202860D004DC002853D010288E
:20BD000065D155E030285DD0402860D141E0602835D070280DD0B0F5805F03D0B0F5005F1C
:20BD200055D115E02068806820F00700216888604EE0D5E902136A68206808F0EDFE20682A
:20BD4000866826F0770646F07706206886603FE0D5E902136A68206808F0DEFE20688068B1
:20BD600040F480402168886032E0EA686968206808F0B0FF5021206808F0DAFE28E0EA68D7
:20BD80006968206808F0BBFF6021206808F0D0FE1EE0EA686968206808F09CFF40212068A4
:20BDA00008F0C6FE14E00021206808F0C1FE0FE01021206808F0BCFE0AE02021206808F06E
:20BDC000B7FE05E03021206808F0B2FE00E000BF00BF012084F83D0000BF002084F83C0079
:20BDE00000BF00BF71E7704710B5044620680069C0F34000D8B12068C068C0F34000B0B136
:20BE00006FF0020021680861012020772068806900F0030018B12046FFF7E5FF05E020465F
:20BE200000F0D6F8204600F0ABF90020207720680069C0F38000D8B12068C068C0F3800003
:20BE4000B0B16FF0040021680861022020772068806900F4407018B12046FFF7C4FF05E091
:20BE6000204600F0B5F8204600F08AF90020207720680069C0F3C000D8B12068C068C0F3DF
:20BE8000C000B0B16FF0080021680861042020772068C06900F0030018B12046FFF7A3FF02
:20BEA00005E0204600F094F8204600F069F90020207720680069C0F30010D8B12068C0685F
:20BEC000C0F30010B0B16FF0100021680861082020772068C06900F4407018B12046FFF7A4
:20BEE00082FF05E0204600F073F8204600F048F9002020772068006900F0010058B120685A
:20BF0000C06800F0010030B16FF0010021680861204600F095F920680069C0F3C01058B174
:20BF20002068C068C0F3C01030B16FF08000216808612046FFF75EFD20680069C0F3801031
:20BF400058B12068C068C0F3801030B16FF0400021680861204600F077FA20680069C0F308
:20BF6000401058B12068C068C0F3401030B16FF02000216808612046FFF73DFD10BD000000
:20BF80001FB504460E492068884218D140200090022001900320039069460A48FEF784FC22
:20BFA00000BF0949486820F4406040F0E06040F44060486000BF0021044800F00BF81FBD25
:20BFC000000400400010014000000140841E00207047000030B504460D4601222946206876
:20BFE00008F07EFD0A492068884201D1012000E0002028B12068406C40F400402168486480
:20C000002068006840F0010021680860002030BD002C014070B504460D46164600BF94F82B
:20C020003C00012801D1022070BD012084F83C0000BF022084F83D0036B1042E1BD0082ECD
:20C0400031D00C2E5ED145E02946206808F07AFD2068806940F0080021688861206880695F
:20C0600020F004002168886120688069296908432168886147E02946206808F095FD20684A
:20C08000806940F40060216888612068806920F480602168886120688069296940EA01208C
:20C0A000216888612FE02946206808F0B5FD2068C06940F008002168C8612068C06920F002
:20C0C00004002168C8612068C069296908432168C86118E02946206808F0D4FD2068C06901
:20C0E00040F400602168C8612068C06920F480602168C8612068C069296940EA012021688C
:20C10000C86100E000BF00BF012084F83D0000BF002084F83C0000BF00BF85E710B504462E
:20C120000CB9012010BD94F83D0028B9002084F83C00204600F00CF8022084F83D00211D57
:20C14000206808F093FC012084F83D000020E9E708B5094A016891420DD100BF0749C9699B
:20C1600041F00201054AD1611146C96901F00201009100BF00BF08BD000400400010024023
:20C180007047000030B504460D4601222946206808F0A6FC0A492068884201D1012000E03A
:20C1A000002028B12068406C40F40040216848642068006840F0010021680860002030BD8A
:20C1C000002C014030B504460D4600222946206808F086FC19492068884201D1012000E056
:20C1E000002090B100BF2068006A41F21111084050B92068006A8910084028B92068406C9F
:20C2000020F400402168486400BF00BF2068006A41F21111084050B92068006A89100840AC
:20C2200028B92068006820F001002168086000BF012084F83D00002030BD0000002C014018
:20C2400038B5044670480088401C6F49088008460088B0F5967F01DB002008806B4840784C
:20C260006B4B0090DA79997958796A4B1B7800F04DFE69480078401C67490870084600784C
:20C2800005280ADB65480068806840F0010063490968886000206049087061480068401CAB
:20C2A0005F49086000F04CFA5D48C08842F6FF7188420CDA5A480089594989880844584928
:20C2C00008810846C088898808445549C880544A917A108905F05AFD5249488052495348D5
:20C2E00004F0BEFA52480078524909784840FF281AD14F4880794F4989794840FF2813D10D
:20C300004B4880884B498988484080B24FF6FF71884209D14648408846494988484080B25A
:20C320004FF6FF7188420AD0FEF75EFC42490968401AC82807D902204049087003E0FEF734
:20C3400053FC3D4908603D480078012802D0022856D151E03648807901284CD13848007871
:20C36000012804D1FBF7A6F800203549087030480078012811D0022804D003280ED00428EC
:20C3800037D116E0264B1A89264BB3F90210284BB3F90200FBF74AFA2CE000BF204B1A892C
:20C3A000204BB3F90210224BB3F90400FBF73EFA20E02448007800F0010050B9184B1A8929
:20C3C000184BB3F902101A4BB3F90400FBF72EFA0EE01C48007800F0010048B1104B1A895B
:20C3E000104BB3F90210124BB3F90200FBF71EFA00E000BF00BF04E001201149087000E0FA
:20C4000000BF00BF38BD0000F8040020D2000020080A002028040020F0040020F01E0020DB
:20C42000241500201408002084010020A4020020D6000020DE000020F404002030000020A0
:20C44000F104002091010020704770472DE9F0470446206805682068C668206847694FF0EE
:20C460000008C14605F00F08B8F1000F0AD105F0200038B106F0200020B1204609F0E4F8EE
:20C48000BDE8F087B8F1000F6DD007F0010018B906F49070002866D005F0010030B106F499
:20C4A000807018B1E06B40F00100E06305F0040030B107F0010018B1E06B40F00200E063A9
:20C4C00005F0020030B107F0010018B1E06B40F00400E06305F0080030B107F0010018B162
:20C4E000E06B40F00800E063E06B68B305F0200028B106F0200010B1204609F0A5F82068C7
:20C500004069C0F38019E06B00F0080010B9B9F1000F22D0204609F028F82068406900F0CF
:20C520004000B0B12068406920F0400021684861606B50B11748616B4863606BFDF7C2FE86
:20C5400010B1606B416B88470CE02046FFF77DFF08E02046FFF779FF04E02046FFF775FFA0
:20C560000020E0638CE705F0800030B106F0800018B1204609F0AEF982E705F0400030B1CB
:20C5800006F0400018B1204608F0FFFF78E700BF76E700001954010810B504460CB901205A
:20C5A00010BDA06900B100E000BF94F8390028B9002084F83800204600F028F8242084F8A5
:20C5C00039002068C06820F400502168C860204609F09CF82068006920F4904021680861A3
:20C5E0002068406920F02A00216848612068C06840F400502168C8600020E063202084F89A
:20C60000390084F83A000020CAE7000010B586B004462B49206888424FD100BF2948C069D6
:20C6200040F480202749C8610846C06900F48020019000BF00BF08150290022003900120EE
:20C6400004900320059002A91F48FEF72DF94FF400600290002003900120049002A91A48B7
:20C66000FEF722F900BF1949486820F0300040F0E06040F01000486000BF012211462720C1
:20C68000FEF781FB2720FEF771FB11480068C06840F480700E490968C8600D48006840691E
:20C6A00040F001000A490968486109480068C06840F0200006490968C86006B010BD000040
:20C6C00000480040001002400010014000000140702600207047704710B500F011F90549BD
:20C6E00031F8100041F255510844034908810020086010BD508301082415002000B585B093
:20C7000000BF0D48806940F010000B4988610846806900F01000009000BF00BF4FF4607047
:20C720000190002002900120039001A90348FEF7BBF805B000BD0000001002400010014050
:20C74000F8B500F0DDF8064600F0DAF8044600F0D7F80546A64203D1AC4201D15E4805706E
:20C760005E48007830B95C4800785B49487001205A4908705848007857494978884210D0DB
:20C78000FEF732FA564908605648007828B155480078401C5349087017E001205249887250
:20C7A00013E0FEF721FA4E490968401AC8280CD900204D4988724B4908704B498881C8819D
:20C7C0004A4908700120484908744748807A10B9002047490870404800783F494978454ACE
:20C7E000515C884245D14048006840B13E48006842F6AA21B1FBF0F03B49888002E00120BF
:20C80000394988803A480078401C394908700846007802280DDD3448006844F63E11B1FB4B
:20C82000F0F03149888100203049087001202E4908742F4800780F280CDA274800782E4906
:20C8400031F8100041F255510844274908810020888009E00F20264908701F48007826490C
:20C8600031F810002049088100201F490860C88026E019484078184909781E4A515C884275
:20C880001ED100201A4908701749888012480078194931F8100041F25551084412490881D0
:20C8A0004FF6FF70086011480078401CC0B20F490870052804DD0620087000200A49087452
:20C8C000054800680D49009003F05EF80248007801494870F8BD00007003002072030020D3
:20C8E00074030020730300202415002078030020790300204083010850830108840100202E
:20C9000010B51E48C07AA8B94FF400711C48FEF759F904464FF480711948FEF753F944EAA4
:20C920004000C4B280211648FEF74CF944EA8000C4B220E04FF400711148FEF743F908B9E5
:20C94000012000E0002004464FF480710C48FEF739F908B9012000E0002044EA4000C4B2F7
:20C9600080210748FEF72EF908B9012000E0002044EA8000C4B204F0070010BD2415002084
:20C980000010014007E0044803F09FFE002005F0EDFCFAF7B1FAF6E7F800002070B5044685
:20C9A000204609F006FFA1890122A068FEF716F90120FAF77CFAA1882068FEF703F9054645
:20C9C000A1890022A068FEF709F90120FAF76FFA012D01D1012070BD0020FCE71FB5044622
:20C9E000A06809F063FE206809F060FEA089009001200390112001906946A068FDF754FFC9
:20CA0000A0880090012003901120019069462068FDF74AFF1FBD2DE9F04704460F464FF06D
:20CA200000084FF08009204609F0C3FE00251CE0A1890122A068FEF7D1F83220FAF737FA5E
:20CA4000A1882068FEF7BEF80646012E03D149FA05F040EA0808A1890022A068FEF7BEF8BA
:20CA60003220FAF724FA681CC5B2082DE0DB87F800800120FAF71BFABDE8F08710B5044619
:20CA8000204609F09EFEA18801222068FEF7A6F80120FAF70CFAA1890122A068FEF79EF83C
:20CAA0003220FAF704FAA1890022A068FEF796F8A18800222068FEF791F80120FAF7F7F90B
:20CAC00010BD10B50446204609F07BFEA1890122A068FEF783F8A18801222068FEF77EF89E
:20CAE0003220FAF7E4F9A18800222068FEF776F83220FAF7DCF9A1890022A068FEF76EF819
:20CB000010BD10B50446204609F05BFEA18800222068FEF763F8A1890122A068FEF75EF8BE
:20CB20003220FAF7C4F9A18801222068FEF756F83220FAF7BCF9A18800222068FEF74EF8D8
:20CB4000A1890022A068FEF749F810BD2DE9F04104460D46A8468026204609F032FE002750
:20CB600036E006EA0800C0B1A18801222068FEF735F83220FAF79BF9A1890122A068FEF71F
:20CB80002DF83220FAF793F9A1890022A068FEF725F83120FAF78BF917E0A18800222068AB
:20CBA000FEF71CF83220FAF782F9A1890122A068FEF714F83220FAF77AF9A1890022A0684E
:20CBC000FEF70CF83120FAF772F97610781CC7B2082FC6DBA18801222068FDF7FFFF01205D
:20CBE000FAF765F9BDE8F08101480249086070470030000808ED00E00120234909780529D4
:20CC000010D12149103109789B290BD11E4914310978522906D11C4918310978052901D1B9
:20CC2000032030E018490978042910D1164910310978C3290BD1144914310978B42906D111
:20CC40001149183109780B2901D102201BE00E49097881B90C491031097810290BD10A49FC
:20CC600014310978042906D10749183109780A2901D1012007E005490968054A914201D110
:20CC8000042000E000207047D0FF0FE0002004E01004031300B585B000BF2B48806940F098
:20CCA0001000294988610846806900F01000009000BF00BF254826490860401488800846D6
:20CCC000808801900020029001200390086801A9FDF7EAFD00201E4988714872C860C871C5
:20CCE00008721A481B4908604FF4804088800846808801900020029001200390086801A91A
:20CD0000FDF7D2FD0020134988714872C860C87108720E48104908604FF400408880084656
:20CD2000808801900020029001200390086801A9FDF7BAFD0020084988714872C860C871AA
:20CD4000087205B000BD00000010024000100140501D0020641D0020781D00202DE9F0411A
:20CD600004460F4616469846069DB8F1000F04D10121204609F0FEFC03E00221204609F0CA
:20CD8000F9FCE07900F0010020B101206072FDF72BFFE060607A01281BD1207A50B9FDF7AC
:20CDA00023FFE060FDF720FF206100206072012028700EE0FDF718FFE168401AB84208D95B
:20CDC000FDF712FFE060002060722870FDF70CFF2061287868B966B1FDF706FF2169401A4F
:20CDE000B04206D9FDF700FF20610020607201202870BDE8F0812DE9F04105460E461746EA
:20CE00009846B8F1F10F13D100240EE0BC4201D1012300E000231A4605EBC403998855F819
:20CE20003400FDF7DBFE601CC4B2B442EEDB0DE0002409E005EBC402918855F834000022D4
:20CE4000FDF7CCFE601CC4B2B442F3DBBDE8F08110B586B000BF2A48806940F0040028498E
:20CE600088610846806900F00400019000BF00BF00BF0846806940F0080088610846806941
:20CE800000F00800019000BF00BF002433E01D4A02EBC40291881B4A52F834000022FDF728
:20CEA0009DFE184800EBC400808802900120039002200590134951F8340002A9FDF7F4FC5B
:20CEC000114A02EBC40291880F4A52F834000022FDF784FE0C4800EBC400808802900120FE
:20CEE000039002200590084951F8340002A9FDF7DBFC601CC4B2032CC9DB06B010BD00005C
:20CF0000001002402C040020440400202DE9F0470746894692461C46DDF82080B9F1060F30
:20CF200006D0B9F10C0F05D0B9F1FF0F06D103E0002505E0012503E0022501E0002500BF10
:20CF400000BFBAF1060F06D0BAF10C0F05D0BAF1FF0F06D103E0002605E0012603E0022631
:20CF600001E0022600BF00BF43462A4603217548FFF741FF072F43D2DFE807F04204436F19
:20CF80007AA6AD004CB9F123324603216E48FFF732FF00206D49088031E0B8F1F10F22D127
:20CFA0006B48408969490988884206DDF123324603216548FFF71FFF0FE065488089634943
:20CFC0000988884206DDF023324603215E48FFF712FF02E000205D4908805C480088401CFF
:20CFE0005A4908800BE0B8F1F00F08D1F023324603215548FFF7FFFE0020544908809DE099
:20D0000000BF04BB51480088B0F5167F06DAF123324603214C48FFF7EEFE0EE04B48008828
:20D02000B0F5966F06DAF023324603214648FFF7E2FE02E000204549088044480088401CCB
:20D040004249088008E04346324603213E48FFF7D2FE00203D49088070E00CB9F12000E030
:20D06000F0200346324603213748FFF7C4FE65E004BB36480088B0F5167F06DAF1233246D4
:20D0800003213148FFF7B7FE0EE030480088B0F5966F06DAF023324603212B48FFF7ABFE0F
:20D0A00002E000202949088028480088401C2749088008E0F023324603212348FFF79BFE97
:20D0C00000202249088039E0F123324603211E48FFF791FE32E01F4800881D4909898842C6
:20D0E00022DB1B48408919490988884206DDF123324603211448FFF77EFE0FE01448808995
:20D1000012490988884206DDF023324603210E48FFF771FE02E000200C4908800B48008852
:20D12000401C0A49088008E0002008490880F023324603210448FFF75EFE00BF00BFBDE867
:20D14000F08700002C040020440400205C040020080A0020BC0300207CB504460D460949EF
:20D1600003C9CDE90001084803F0A2FA01208DF8060003208DF80000009820600198606088
:20D180007CBD0000C0760108F80000202DE9FF4F85B0804691461D464FF0000AFE4903C90A
:20D1A000CDE90301FD48008800B2FD490880FD48B0F9020064286DDD0846B0F90000002883
:20D1C00068DDF848B0F9020064214843F449B1F90010B0FBF1F000B2F34908800846B0F91F
:20D1E0000040F2480068C0EB0420F049096801EBA010EE49086008460068001200B2EC49EA
:20D200000880E748B0F90000EA49B1F90010401A052811DDE348B0F90200E749B1F900108C
:20D22000401A002804DDE048B0F90000E3490880DC484088E0490880D948B0F90000DD4979
:20D240000880DF48007820BBDE48B0F90400192829DDDD480088401CDB4908800846008827
:20D26000282820DB00200880D1480088D749D84A128821F81200D6480088401CD44908806C
:20D280000846008832280EDB002008800120CC49087008E0C248B0F90000C6490880C148E4
:20D2A0004088C5490880CB48408800B2CA490880A9F16404B4F5006F02DD4FF4006000E06C
:20D2C0002046044604FB04F0C11700EB5151CC12C24800780521B1EBD00F17DBB14AD17B0C
:20D2E000BF4A1279012383EAD21003F0B3F9BC490979BC4A92F910201144B84A127801EB73
:20D30000D2010A314843C0F3872A16E0A54AD17BB34A1279012383EAD21003F09BF9B04964
:20D320000979B04A92F910201144AC4A127801EBD20115394843C0F3872A0AF10100604346
:20D3400032214843A849C98990FBF1F000B2A74908800AEB8A00162101EB40009049B1F9B1
:20D360000010884202DA0020A04908809B480078C0F3800038B18A48B0F900003C2802DC32
:20D3800000209A4908809948B0F90000002803DD9648B0F9000000E0002094490880084636
:20D3A000B0F900008C49B1F90010884203DA8F48B0F9000002E08848B0F900008B49088057
:20D3C0009DF81800C0F34000B0B305F00F00012806D002280FD0032818D004282DD120E001
:20D3E0004FF4FA6201217C48B0F9000007F09AFA7F4908602CE040F2DC5201217648B0F94F
:20D40000000007F08FFA7A49086021E04FF47A7201217148B0F9000007F084FA7449086013
:20D4200016E04FF4FA7201216B48B0F9000007F079FA6F4908600BE00BE04FF47A72012118
:20D440006548B0F9000007F06DFA6949086000BF09E04FF4FA7201215F48B0F9000007F03E
:20D4600061FA634908604FF47A7201215A48B0F9000007F057FA5F4908605248807968B995
:20D480004848B0F90200642808DD464840885A490880084600880004584908609DF81800CF
:20D4A000C0F34000F0B305F00F00012806D0022814D0032824D0042842D134E04B49B1F915
:20D4C000001001EBC10108114C4B4A490A684849096809F093F9484908803EE04349B1F9E5
:20D4E000001001EB410202EBC1010811434B41490A683F49096809F081F93F4908802CE013
:20D500003A49B1F9001001EB810202EBC10108113A4B38490A683649096809F06FF936494F
:20D5200008801AE01AE0354B32480268304801682E48B0F9000009F061F92F4908800CE0CC
:20D540002E4B2C4802682A4801682848B0F9000009F054F92849088000BF0BE0274B2548B8
:20D560000268234801682148B0F9000009F046F9214908806FF0C7002149086140F63400CE
:20D5800048612048C08901B21D4A1B48B0F9000004F0A6FD1C4939E0A8760108BC030020F0
:20D5A0001E010020140800202401002000010020260100202201002020010020040100209A
:20D5C00008010020D60000200A0100202807002006010020280A002028010020910100203E
:20D5E000E8090020080A0020DC0100202A0100202C01002030010020340100201801002074
:20D60000BC060020241500203E01002008806FF063005849086140F21A404861564AD17BFB
:20D62000564A127A012383EAD21002F0E5FF5349097A4FF47A7251434843401400904E488E
:20D640000089C1114E4A009804F04AFD4D4908804D4A117B484AD0884C4A128801F0F4FBC9
:20D6600007464A48078001231A4649480188384601F042FD46490880404A517A3E4A907DF7
:20D6800001F0D0FB83463D4A527A0F3A91B23A4A507D01F0C7FB019001980BFB00F0810A77
:20D6A0000291029988B201231A463A49098801F023FD384908803848B0F900003449098819
:20D6C00048438612334800887043861233480078B0B933480068301A022805DD3048006864
:20D6E000801C2F49086018E02D480068301A10F1030F12DA2A480068C01E294908600CE012
:20D7000027480068132805DD2548006810382449086002E00020214908702148006810F16D
:20D72000C80F03DA6FF0C7001D4908601D48008818B91D4802F0C9FF02E01B4802F0B8FF76
:20D74000174800680F49B1F900100844401000B2ADF8100001208DF8120004208DF80C0080
:20D760000398C8F800000498C8F8040009B0BDE8F08F0000BC06002014080020E8090020E2
:20D780009806002040010020280A00204201002044010020460100203E0100203C0100202D
:20D7A0003801002034010020F80000202DE9FF4F87B0824616461F46FE4903C9CDE90501B0
:20D7C000002004900390BE4203DA07FB07F0C01202E006FB06F0C012F74948800846408891
:20D7E000B0F5006F02DD4FF4006001E0F2484088F14948809DF82000C0F3400000287CD092
:20D80000149803287AD004DC012807D0022876D149E0042874D03328F9D1D7E0E748007A78
:20D82000002801DC012001E0E448007A0490E348407A0390E0484088E049C9884843C00A70
:20D8400004B2DE48C088A04202DADC48C08800E0204604B2D9484089D949097A48434FF421
:20D860007A714843401400EBC00101EB00104FF6FF7101EA800501230522D24801882846B5
:20D8800001F03AFCCF490880CC48C0884042CE49086100204861C948C08880024042886154
:20D8A0000020C861DFE0C548007D002801DC012001E0C248007D0490C048407D0390BE4856
:20D8C0004088BE49498A4843C00A04B2BB48408AA04202DAB948408A00E0204604B2B7484A
:20D8E000C08AB749097A48434FF47A714843401400EBC00101EB001003E0B5E01DE0ADE019
:20D9000063E04FF6FF7101EA800501230522AD480188284601F0F0FBAA490880A748408A58
:20D920004042A949086100204861A448408A8002404288610020C86195E0A04890F8200050
:20D94000002801DC012002E09C4890F8200004909A4890F821000390974840889749C98BA6
:20D960004843C00A04B29548C08BA04202DA9348C08B00E0204604B29048408C9049097A94
:20D9800048434FF47A714843401400EBC00101EB00104FF6FF7101EA800501230522894806
:20D9A0000188284601F0A8FB864908808348C08B404285490861002048618048C08B800258
:20D9C000404288610020C8614DE000BF7B4890F82C00002801DC012002E0784890F82C00B4
:20D9E0000490764890F82D000390734840887349498D4843C00A04B27048408DA04202DA2A
:20DA00006E48408D00E0204604B26C48C08D6C49097A48434FF47A714843401400EBC0010A
:20DA200001EB00104FF6FF7101EA80050123052264480188284601F05FFB624908805F48B2
:20DA4000408D404260490861002048615B48408D8002404288610020C86104E0002004905E
:20DA60000390002400BF4DE09DF82000C0F34000F0BB524890F83800002801DC012002E04E
:20DA80004E4890F8380004904C4890F82D000390494840884949498D4843C00A04B2474865
:20DAA000408DA04202DA4548408D00E0204604B24248C08D4249097A48434FF47A7148435C
:20DAC000401400EBC00101EB00104FF6FF7101EA8005012305223B480188284601F00CFB68
:20DAE000384908803548408D40423749086100E008E0002048613148408D800240428861A4
:20DB00000020C861314890F90E00322805DC2F4890F90E0010F1320F02DA00202B498873B6
:20DB20002A4890F90F00322805DC284890F90F0010F1320F02DA00202449C87324480078CE
:20DB40000521B1EBD00F63DB224AD17B1C4A1279012383EAD21002F07DFD194909791B4A15
:20DB600092F9102011449DF8202001EBD201083101EB8101154A92F90E2002EB4101484388
:20DB8000C0F38F2014490880124AD17B0C4A1279012383EAD21002F05DFD094909790B4ACD
:20DBA00092F9102011449DF8202001EBD2010A3114E00000B0760108E80000201C0B002014
:20DBC000E80900204A010020E0060020080A002091010020140800204E01002001EB8101C6
:20DBE000BA4A92F90F2002EB410116314843C0F38F20B749088008460088B6490988401ABC
:20DC0000C01E4FF4806191FBF0F0B34908804CE0B24AD17BB24A1279012383EAD21002F0B2
:20DC200019FDAF490979A94A92F9102011449DF8202001EBD201173901EB8101A34A92F987
:20DC40000E2002EB41014843C0F38F20A1490880A24AD17BA24A1279012383EAD21002F0F4
:20DC6000F9FC9F490979994A92F9102011449DF8202001EBD201153901EB8101934A92F99A
:20DC80000F2002EB410116314843C0F38F2090490880084600888F490988401AC01E4FF4D7
:20DCA000806191FBF0F08C4908808E480078C0F3800078B98C48008800908748008803B210
:20DCC0008448028800210846F9F732FF6043800A04B20EE08448008800907F48008803B2A5
:20DCE0007C480288FF213C20F9F722FF6043800A04B27E488480B0F90400002802DC0020C9
:20DD00007A4988807848008872490988884220DD7648B0F904007549B1F90610401A022870
:20DD200006DD7248C088401C00B27049C88033E06E48B0F904006D49B1F90610401AB0F108
:20DD4000FF3F29DA6948C088401E00B26749C88022E000BF6548B0F904006449B1F90610F9
:20DD6000401A022807DD6148C1880498084400B25E49C88010E05D48B0F904005B49B1F930
:20DD80000610401AB0F1FF3F06DA5848C1880398081A00B25549C8805448B0F9060006289D
:20DDA00001DA062002E05148B0F906004F49C8804D48008846490988884208DD01204B49B7
:20DDC00008700020C8804A4802F07FFC02E0484802F06EFC474A117B404AD088464A12886D
:20DDE00001F032F881464448A0F8009001231A4642480188484601F07FF940490880384A6C
:20DE0000517A364A907D01F00DF80290344A527A0F3A91B2314A507D01F004F80190DDE9C0
:20DE2000011048434FEA902B1FFA8BF001231A463349098801F060F931490880274AD17B24
:20DE4000274A127A012383EAD21002F0D5FB2D4909884843642190FBF1F0801200B2009039
:20DE60001E480089C111284A009804F039F9274908801E48B0F906002049098848434FEAE6
:20DE8000A0281F48008808FB00F04FEAA0281F48B0F9000040444FEA6008B8F1000F01DA0F
:20DEA000002000E0404600B2ADF8160001208DF81A0004208DF814000598CAF800000698F5
:20DEC000CAF804000BB0BDE8F08F0000080A0020500100204E0100205201002014080020DC
:20DEE000E809002091010020BC030020E8000020F8000020280A0020540100205601002022
:20DF0000580100204A010020E0060020480100202DE9FF4F8BB081468A46FE4903C9CDE9AF
:20DF200009014FF0000B0020089005900490FA48A0F802A0F9480088C82801DA642002E036
:20DF4000F648008840100690F34841880698814204DBFCF749FEF249086020E0F148B0F912
:20DF60000200C82807DDEF48B0F90200EE4991FBF0F086B201E04FF49666B6F5FA7F02DAEE
:20DF80004FF4FA7000E030460646FCF72DFEE4490968401AB04202D90120DF490870E14865
:20DFA00000883C2814DDDD480088C82801DA96200CE0DA480088B0F52F7F02DD40F20D202F
:20DFC00004E0D648008800EB40008010079010E0D2480088C82801DA962009E0CF480088CA
:20DFE000B0F52F7F02DD40F20D2001E0CB4800880790C94841880798814202DB0020C64935
:20E000000870CA484078012802D0C848807810B90120C1490870C048007801283ED1BE4891
:20E02000B0F90610C2484079002801DA032007E0BF484079052801DD032001E0BC484079C5
:20E04000401EBC4A105C81420CDC0020B249C880B94802F03AFB0120B84908700020B849FF
:20E060000880B6E3AC48B0F90610B1484079002801DA032007E0AE484079052801DD032030
:20E0800001E0AB484079401EAA4A105C081A00B2A149C880A84802F00BFB9AE39E490E983D
:20E0A0004880A048B0F90200B0F5FA7F23DD9F4800780F281FDB08464088C8281BDD994878
:20E0C000B0F90200642148439849097890FBF1F09C4908609C4800680968C0EB01309A49EE
:20E0E000096801EBA0209849086008460068C0F30F30964908800D9803287DD004DC012885
:20E1000007D0022879D160E0042877D03328F9D198E18F48007A002801DC012001E08C4837
:20E12000007A83468A48407A0890DFF8ECC1BCF80230DFF81CC2BCF80220BCF80010BCF80B
:20E1400000C04FEA6C00F7F763FA734949884843800A04B27E488088A04202DD7C4880885C
:20E1600000E0204604B27A48C088A04202DA7848C08800E0204604B2754840896C49097A19
:20E1800048434FF47A714843401400EBC00101EB00104FF6FF7101EA8005012305226D481A
:20E1A0000188284600F0A8FF6A4908806848C088404269490861002048616548C0888002C1
:20E1C000404288610020C861ABE16148007D002801DC012001E05E48007D83465C48407D85
:20E1E0000890DFF834C1BCF80230DFF864C1BCF80E20BCF80C1002E047E08CE1C7E0BCF856
:20E200000CC04FEA6C00F7F703FA434949884843800A04B24E48008AA04202DD4C48008A7B
:20E2200000E0204604B24A48408AA04202DA4848408A00E0204604B24548C08A3C49097A93
:20E2400048434FF47A714843401400EBC00101EB00104FF6FF7101EA8005012305223D4889
:20E260000188284600F048FF3A4908803848408A404239490861002048613548408A80021C
:20E28000404288610020C8614BE1314890F82000002801DC012002E02D4890F8200083468F
:20E2A0002B4890F821000890DFF86CC0BCF80230DFF89CC0BCF81A20BCF81810BCF818C038
:20E2C0004FEA6C00F7F7A4F9134949884843800A04B21F48808BA04202DD1D48808B00E093
:20E2E000204604B21A48C08BA04202DA1848C08B00E0204604B21648408C0D49097A484362
:20E300004FF47A714843401414490978484385B2012325E0C8760108E8000020EA030020CB
:20E320006001002014080020205503008C030020E8090020F9000020F8000020690100202D
:20E340006A0100207401002078010020D20100201C0B002066010020E0060020E600002037
:20E360000522FE480188284600F0C6FEFB490880FB48C08B4042FB49086100204861F848F3
:20E38000C08B8002404288610020C861C9E0F44890F82C00002801DC012002E0F04890F89B
:20E3A0002C008346EE4890F82D000890DFF8B8C3BCF80230DFF8A8C3BCF82620BCF8241089
:20E3C000BCF824C04FEA6C00F7F722F9E64949884843800A04B2E248008DA04202DDE0488C
:20E3E000008D00E0204604B2DD48408DA04202DADB48408D00E0204604B2D948C08DDB4966
:20E40000097A48434FF47A7148434014D8490978484385B201230522D0480188284600F033
:20E420006BFECE490880CE48408D4042CD49086100204861CA48408D80024042886100203B
:20E44000C8616EE0C64890F83800002801DC012002E0C34890F838008346C14890F8390011
:20E460000890C1484088B0F5FF7F15DADFF8F8C2BCF80230DFF8E8C2BCF80E20BCF80C1077
:20E48000BCF80CC04FEA6C00F7F7C2F8B64949884843800A04B207E0B34840884043B049EE
:20E4A000498EB0FBF1F004B2AD48808EA04202DDAB48808E00E0204604B2A948C08EA04261
:20E4C00002DAA748C08E00E0204604B2A448408FA649097A48434FF47A7148434014A44975
:20E4E0000978484385B2012305229C480188284600F002FE994908809948C08E40429949C6
:20E500000861002048619648C08E8002404288610020C86105E04FF0000B0020089000245C
:20E5200000BF00BF934890F90E00322805DC914890F90E0010F1320F02DA00208D49887331
:20E540008C4890F90F00322805DC8A4890F90F0010F1320F02DA00208649C873864AD17B46
:20E56000824A1279012383EAD21002F073F87F490979804A92F91020114401EB81017D4A1B
:20E5800092F90E2002EB41014843C0F38F207B490880794AD17B754A1279012383EAD2108E
:20E5A00002F058F871490979724A92F91020114401EB81016F4A92F90F2002EB41011631BA
:20E5C0004843C0F38F206E490880084600886B490988401AC01E4FF4806191FBF0F069497A
:20E5E00008806948008800900846008803B26348028800210088F9F79BFA6043800A04B2F9
:20E6000059488480B0F90400002802DC0020564988805D48008859490988884220DD52481A
:20E62000B0F904005049B1F90610401A022806DD4D48C088401C00B24B49C880ABE04A4889
:20E64000B0F904004849B1F90610401AB0F1FF3F05DA4548C088401E00B24349C8809AE071
:20E6600000BF4A480078012857D140484078032805D1002046490880444908708BE03B4815
:20E680004078012805D14FF4967005901E20049003E0642005900A2004903D480088401CF0
:20E6A0003B49088008460188059881422FDC2E48B0F904002C49B1F90610401A022814DD3F
:20E6C00033480188049891FBF0F0C0F10A003049098891FBF0F200FB121068BB2248C08809
:20E6E000584400B22049C88055E01F48B0F904001D49B1F90610401AB0F1FF3F4BDA1A48EC
:20E70000C1880898081A00B21749C88043E000201F4908801D4908703DE01348B0F904005E
:20E720001149B1F90610401A022806DD0E48C088584400B20C49C8802DE00B48B0F90400C2
:20E740000949B1F90610401AB0F1FF3F23DA0648C1880898081A00B203491BE06601002098
:20E760001C0B0020E0060020E8000020E8090020E6000020080A0020140800207C01002022
:20E780007E01002080010020BC030020690100206A010020C8804A48B0F90600062801DAB3
:20E7A000062002E04648B0F906004549C8804548008845490988884208DD01204049087039
:20E7C0000020C880414801F080FF02E03F4801F06FFF3F4A117B3F4AD0883F4A128800F007
:20E7E00033FB80463C48A0F8008001231A463B480188404600F080FC38490880384A517AB1
:20E80000344A907D00F00EFB0290354A527A0F3A91B2304A507D00F005FB0190DDE901106C
:20E820004843810A0391039988B201231A462D49098800F061FC2B490880264AD17B284A56
:20E84000127A012383EAD21001F0D6FE264909884843642190FBF1F0801200B200901D483F
:20E860000089C111214A009803F03AFC204908801348B0F90600194909884843871219489E
:20E880000088784387121A48B0F9000038444710002F01DA002000E0384600B2ADF82600B9
:20E8A00001208DF82A0002208DF824000998C9F800000A98C9F804000FB0BDE8F08F000011
:20E8C000E8000020BC0300207E010020F8000020280A0020140800206C0100206E010020F0
:20E8E000E80900207001002066010020E0060020640100202DE9FF5F82460E468C4903C933
:20E90000CDE90201002700BF0025002E40D1A9468848C07F08B9872001E08648C07F8146D9
:20E92000854840680A21C1EB4911884205D282484068401C8049486010E07F4840680A21C7
:20E9400001EB4911884205D97B484068401E7A49486003E04FEA491077494860774AD17BAB
:20E96000744A127A012383EAD21001F045FE7149097A4FF4FA7251434843401400906F4800
:20E980000089C1116E4A009803F0AAFB044655E06C484088400141F2883190FBF1F0C5B229
:20E9A000012D01DA012000E028460546654840884001654909784843642190FBF1F00A38F1
:20E9C0005D494968884205D95B48406828445A49486026E05B48408840015B4909784843D4
:20E9E000642190FBF1F00A305349496888420DD251484068A84205D94F484068401B4E49BC
:20EA000048600EE000204C4948600AE04D48408840014D4909784843642190FBF1F0464959
:20EA20004860464A1289D111424A127A4FF47A735A43D011424A03F053FB04463F4AB2F910
:20EA400002103D4A5268520910B2404A03F048FB0746381907B236BB4FF000093548807F7A
:20EA600008B93C2001E03348807F814633480088A9F105018AB2009088B280230021F9F7FA
:20EA800057F87843800A07B22C480088484506DD0020294948602E4801F017FE02E02C48B1
:20EAA00001F006FE02E02A4801F002FE254A117B224AD088274A128800F0C6F98046254870
:20EAC000A0F8008001231A4623480188404600F013FB21490880174A517A184A907D00F0A5
:20EAE000A1F9019001231A461C480188019800F003FB1A4908801848008878434FEAA02B61
:20EB0000084600880BFB00F04FEAA02B0FFA8BF0ADF80C0001208DF80E008DF80800029815
:20EB2000CAF800000398CAF80400BDE8FF9F0000B8760108E8090020F000002014080020DB
:20EB400098060020280A0020A7010020BC060020F80000205A0100205C0100205E0100206C
:20EB600070B504460D461646FCF73EF83C490968401A642870D3FCF737F8394908603948A2
:20EB8000006828443749086037480078401C364908700846007808280ADB32480068C0F3FF
:20EBA000CF003249088000202F4908702D490860462C0BDA2D48008841F27071884205DD81
:20EBC0002B480088401C2A49088002E0002028490880462C05DC2548008841F288318842EA
:20EBE00007DA962E05DA23480088401C2149088002E000201F4908801D480088B0F5967FB7
:20EC000005DD00201A49088001201B49087019480088642804DD00201649088016490870D6
:20EC200015480078012814D1462C0EDA04F11E001249087008460078642801DD642001E01C
:20EC40000E4800780D49087006E064200B49087002E06420094908700848007870BD0000BD
:20EC6000A4000020A8000020AC000020AE000020B0000020B2000020B4000020B500002023
:20EC80002DE9FF4385B0074615469846DDE9109408EA090000F00103BDF81A105548007814
:20ECA0002A46049001F062FC06462078B04223D05148007800BB052601204F490870207878
:20ECC000042819D14D480068142806DD04260020087001204A4908700EE00020494908600C
:20ECE000494908604949088044490860444908700526012040490870062E68D2DFE806F08E
:20ED00006733574B03683B48007800F0010078B905F00F03BDF81A2036480078014602906A
:20ED200003A8FEF733FA039820600498606016E03048007800F0010088B105F00F000090EB
:20ED4000BDF81830BDF81A202A4800780146029003A8FEF72BFD03982060049860600020A5
:20ED60002549087041E02A480078012807D12948B0F9020040012649486000200870394616
:20ED800003A8FFF7B7FD039820600498606000201949087029E0294603A8FEF7DDF9039824
:20EDA0002060049860600020134908701DE01A480389BDF818102A4603A8FFF7A9F803986E
:20EDC00020600498606000200B4908700DE000BF124801F07AFC1248F6F7AEFE0520207056
:20EDE0000020A0716080A08000BF00BF09B0BDE8F0830000910100208201002038010020E5
:20EE00003C010020000100201801002034010020F0000020140800208C030020F8000020D3
:20EE20008401002010B502464FF480608A4208DD01FB01F4A302B3FBF2F4B4FBF2F4A0B23B
:20EE400001E04FF4806010BDF0B503460E461546002100244FF48060182E04D0242E12D08E
:20EE6000302E34D121E0E721FC2401EBC10707EB0117B3EB870F02DD4FF4806701E0B3FB7C
:20EE8000F1F73A4625E04FF4A5714FF4B47401EBC10707EB0117B3EB870F02DD4FF4806746
:20EEA00001E0B3FBF1F73A4613E040F2AD114FF4EA7401EBC10707EB0117B3EB870F02DD06
:20EEC0004FF4806701E0B3FBF1F73A4601E0642200BF00BF02FB02F74FF0640CB7FBFCF7E2
:20EEE0005743B7FBFCF75743BF0242F2107CB7FBFCF2B2F54D7F02D24FF44D7700E017468D
:20EF00003A46AA4201D290B200E0284604EBC40707EB0417B3EB870F01DD4FF48060F0BD79
:20EF20002DE9F04105460E4617461C46002F7DD1552D66D14748007820BBFBF755FE454941
:20EF40004968401AB0F57A7F15D90120414908700020207040480078C043404908703E48BD
:20EF60004078C04348703E48007820F00200801C3B49087018E03A48007820F002003849F1
:20EF8000087011E00020207033480078C0433349087031484078C04348703148007820F081
:20EFA0000200801C2E490870AA2E06D12C48007820F004002A49087023E02A480078C8B9BC
:20EFC000FBF712FE27494968401AB0F57A7F0AD90120244908702248007820F00400001D1A
:20EFE0001F4908700DE01E48007820F004001C49087006E01A48007820F00400001D184923
:20F00000087019480078E0B9FBF7EEFD16494968401A41F2883188420CD901201249087030
:20F020000F48007820F00100401C00E010E00C4908700DE00A48007820F001000849087066
:20F0400006E00748007820F00100401C04490870BDE8F081B0010020D2000020D400002004
:20F0600088010020B8010020C0010020012013490870002048600120114908700020488095
:20F080008880C8800F4908600F4908600F4908600F4908600F4908600F4908600F490860E0
:20F0A0000F4908620F4908620F4908620F4908620F4908620F49086270470000F0000020FD
:20F0C000E800002004000020080000200C0000201000002014000020180000201C000020D8
:20F0E000500600202C06002074060020E0060020BC0600209806002070B504461546661ABE
:20F1000032B2002A06DDAA4202DB4E19B0B20CE020460AE0002A07DA56429E4202DBCE1AE8
:20F12000B0B202E0204600E0204670BD10B5FBF75BFD2E490968401A642855D3FBF754FD6A
:20F140002A4908602A4800782A4908702A480078487000208870C8702848008800B288805B
:20F160002748008800B2C88026484088088125480088488124480088888123484088C881A8
:20F1800022480089088222480068801200B2488220480068801200B28882154800780228F5
:20F1A00003D113484088C8821EE011480078012804D10F4880880F49C88215E00C4800787F
:20F1C00004280ED11448007800F0010020B9084880880849C88207E0054840880549C882FF
:20F1E00002E000200349C88210BD000084000020D600002034080020300000200400002040
:20F20000080000202C0000200A0500208C030020100000200C0000209101002070B505461E
:20F220000E46144608216748FBF7CCFC664908704FF400416548FBF7C5FC654908706248B3
:20F240000078644909784840634908705E480078604908705E4800786049097848406049A4
:20F2600008705B4800785D490870574800785849097848405B490870FBF7B6FCB0F57A7FBE
:20F280000CD2FBF7B1FC58490860FBF7ADFC57490860FBF7A9FC5649086070BD2088C0F31F
:20F2A0008030002878D1B5F5966F7CDD462E7ADD4948007800BBFBF797FC4B490968401AB2
:20F2C00042F2107188421BD9206820F4804000F5804020600120474948800846F8F766F915
:20F2E00000204549087045484088401C43494880022043490870D0E7FBF776FC3A490860B7
:20F300003748007800BBFBF76FFC38490968401A41F2883188421BD9206820F4804000F597
:20F32000804020600220334948800846F8F73EF900203149087031484088401C2F494880C4
:20F3400002202F490870A8E7FBF74EFC274908602448007810BBFBF747FC25490968401ADB
:20F3600041F2883188422AD9206820F4804000F58040206003201F4948800846F8F716F9A4
:20F3800000201D4908701D484088401C1B49488002201B49087080E711E004E0FBF724FC6E
:20F3A000134908600BE0FBF71FFC0F490860FBF71BFC0E490860FBF717FC0D49086000BF87
:20F3C0006BE70000000C0140A002002000080140A1020020890200208802002091020020B8
:20F3E00090020020980200208C020020940200209C020020E414002069030020680A002049
:20F40000920100201FB53948007890B93848807E55280ED1374A384800783849498889B243
:20F42000CDE9010200913649887836490EC900F0ABFE3049344A30480078CDE902210190C3
:20F44000304880680090314801782E480CC8304800F032FF274801902E488088ADF80000C4
:20F46000264B5B889AB2254B1989234B9879294B1C6802949B88ADF80C30234600F0A4FDCF
:20F480001E4A917D507D1B4A00F020FD20490839088A184900F076FA1E4801680291808850
:20F4A000ADF80C00134ADDE9020100F0D3FB114800F03EF80F48134A009011780F4A528838
:20F4C00090B2154A12680392144A1388039A00F095FC084812490090CA8912490878124B9F
:20F4E0001249098800F010FB1FBD0000D0000020E809002084010020D60000201408002071
:20F50000BC0300208C030020E8030020D2000020CC1E00201A0500200A050020D2010020F5
:20F52000DA1E0020A80100202F150020A401002010B50446FBF758FB41F2883188420CD2D9
:20F54000FBF752FBEE490860FBF74EFBED490860FBF74AFBEC49086010BD2068C0F3804058
:20F5600000286FD14FF40041E848FBF72BFB00BBFBF73AFBE3490968401A41F288318842C8
:20F580001BD9206820F4802000F5802020600120DF4948800846F8F709F80020DD49087019
:20F5A000DD484089401CDC4948810220DB49087003E0FBF719FBD3490860D9480088002817
:20F5C00047D1D8480078012843D1D748007805283FD0D548807901283BD1D348B0F9040058
:20F5E000C82804DCD048B0F90200C82831DDCF48807A40BBCE480089C82825DAFBF7F4FA00
:20F60000C1490968401A41F28831884225D9206820F4802000F5802020600220BC49488021
:20F62000BF48008888800846F7F7C0FF0020B9490870B9484089401CB74948810220B7498D
:20F6400008700AE08DE0FFE7FBF7CEFAAE49086003E0FBF7C9FAAC490860FBF7C5FAA84945
:20F660000968401A14287CD3FBF7BEFAA4490860B048C088B04909680844AF490860AF48E8
:20F680000088AF4909680844AD490860AB484088AC4909680844AB490860A8488088AA491B
:20F6A00009680844A8490860A8480078401CA74908700846007820287EDB002008709E4823
:20F6C00000684FF4FA71B1EB501F2FD89A480068C900B1EB501F29D39948006841F28831B3
:20F6E000B1EB501F22D8964800684EF66021B1EB501F1BD39348006841F28831B1EB501FC7
:20F7000014D8904800684EF66021B1EB501F0DD38D48006841F28831B1EB501F06D88A4829
:20F7200000684EF66021B1EB501F16D2206820F4802000F580202060032075494880084661
:20F74000F7F734FF00207349087073484089401C714948810220714908707D480068C82167
:20F7600000E0C2E0B1EBA02F36DA7A48008872490968C0EB511019282AD277480078401C3A
:20F7800075490870084600780A2828DD206820F4802000F58020206004205D4948806648A5
:20F7A0000068C0F34F1088800846F7F7FFFE002058490870584800E01AE04089401C564917
:20F7C000488102205549087000206349087006E000206149087002E000205F49087000207A
:20F7E000554908605649086056490860564908604F48407B00287AD14D484088002876D15D
:20F80000FBF7F2F955490968401A41F28831884274D94848C0885249524A127821F81200DB
:20F820004648008850494F4A127821F81200434841884E484B4A127820F812103F488188F8
:20F840004B48484A127820F8121046480078401C444908700846007832284FDB0020087076
:20F8600032213F48F8F778FE4249086032213E48F8F772FE4049086032213C48F8F76CFEFD
:20F880003E49086032213A48F8F766FE3C49086038480068B0F5FA7F0DD83748006842F65A
:20F8A000E061884207D835480068884203D834480068884222D9206820F4802000F580205A
:20F8C00020600520124948802A48008888800846F7F76CFE00200F4908700F484089401C4C
:20F8E0000D49488102200D49087007E0FFE700201C490870FBF778F91849086000BF2BE633
:20F900002C020020300200203402002000100140E414002069030020680A002092010020B7
:20F920009C01002030000020D60000202415002014080020DA1E00203C0200200205002092
:20F94000400200204402002048020020380200200C000020200500203902002060020020CD
:20F960008C1200204C020020F012002054130020B813002050020020540200205802002065
:20F980005C0200207047000013B50C465448007860B9FBF729F9534908609DF801200621F6
:20F9A0005148F4F78EF801204D4908702078C0F3C01000287ED19DF8000018B19DF8000089
:20F9C000072821D1FBF710F946490968401AB0F57A7F1DD9206820F08000803020600120B4
:20F9E000424948809DF8000088800846F7F7DEFD00203F4908703F48C08A401C3D49C882E3
:20FA000001203D4908701CBDFBF7EEF8354908609DF800009DF8011088425FD09DF8001057
:20FA2000364802780078401C344B18702E48815418460078062851DB00201946087006215A
:20FA40002948F5F7AFFD28B92D480068401C2C49086006E000202A490860FBF7C5F82949A4
:20FA6000086027480068322838D9FBF7BDF82549096801F5FA71884230D9206820F080000A
:20FA8000803020600220194948801748007800021549497800EB01101349897808441349F1
:20FAA00088801148C07800020F49097900EB01100D4900E012E0497908440C49C8800846B4
:20FAC000F7F774FD00200A4908700A48C08A401C0849C88201200849087094E700BF92E7AC
:20FAE00072020020740200207C020020E414002069030020380A00209201002082020020E1
:20FB000084020020780200202DE9F04105460E4614469846069FFBF767F8B0F57A6F01D230
:20FB2000BDE8F081FBF760F842F21071884220D23868C0F3804000287CD1FBF755F83E49A6
:20FB40000968401A142875D3FBF74EF83A49086098F80000A8BB0DB1C82E0BDD40F2C27040
:20FB6000844207DD40F63E00844203DA0020334908705FE031480078401C304908700846E5
:20FB80000078FA2856DB00200870386820F4802000F58020386008202949488005EB8600A9
:20FBA00088800846C480F7F701FD00202549087025484089401C24494881022023490870EB
:20FBC00038E0FFE70DB1C82E03DD002088F8000030E040F68B60844202DCB4F5BA7F26DA3C
:20FBE0001B480078401C1A49087008460078FA2820DB00200870386820F4802000F580208F
:20FC0000386009200E49488005EB860088800846C480F7F7CBFC00200A4908700A48408939
:20FC2000401C0949488102200849087002E000200749087000BF73E76C020020700200205F
:20FC4000E414002069030020680A0020920100207102002037B514466048007801280CD0BD
:20FC6000FAF7C2FF5E490860FAF7BEFF5D490860FAF7BAFF5C4908603EBD2068C0F30040DA
:20FC8000002875D1BDF90000002801DB014600E0414244F62062914228DDFAF7A5FF5049D0
:20FCA0000968401AB0F57A7F24D9206820F4803000F58030206001204C494880BDF9000039
:20FCC000002801DB014600E04142484A91801046F7F76CFC0020464908704648C088401CCE
:20FCE0004449C880022044490870C5E7FAF77CFF3B490860BDF90200002801DB014600E021
:20FD0000414244F62062914228DDFAF76DFF35490968401AB0F57A7F24D9206820F480303F
:20FD200000F580302060022030494880BDF90200002801DB014600E041422C4A91801046F8
:20FD4000F7F734FC00202A4908702A48C088401C2849C8800220284908708DE7FAF744FFF8
:20FD600020490860BDF90400002802DB014601E031E0414244F62062914228DDFAF734FF7F
:20FD800019490968401AB0F57A7F24D9206820F4803000F580302060032014494880BDF92C
:20FDA0000400002801DB014600E041420F4A91801046F7F7FBFB00200D4908700D48C08862
:20FDC000401C0C49C88002200B49087054E7FAF70BFF0549086000BF4EE70000300000200C
:20FDE00014020020180200201C020020E414002069030020680A0020920100202DE9FF4116
:20FE000005460E461F460A9C2068C0F3805000284DD1FAF7E9FE27490968401A142846D37F
:20FE2000FAF7E2FE23490860B5F5FA7F3CDD0F2E3ADBBDF80800C82836DDBDF80A003228B6
:20FE400032DA40F2DC5087422ADD1B480088401C1949088008460088FA2828DB0020088094
:20FE6000206820F4800000F580002060012013494880BDF808008880BDF80A00C880084612
:20FE8000F7F794FB00200E4908700E4890F82400401C0C4981F8240001200B49087006E0D3
:20FEA00000200549088002E0002003490880BDE8FF8100006402002068020020E414002029
:20FEC00069030020380A00209201002070B504460E461546FAF788FE41F28831884201D362
:20FEE0005A2C08DDFAF780FE31490860FAF77CFE2F49086070BD2888C0F34020002855D1BD
:20FF0000052C01DBBE2C22DDFAF76EFE28490968401A41F2883188421DD9286820F4007092
:20FF200000F50070286001202249488008468480C680F7F73BFB00201F4908701F48408B92
:20FF4000401C1E49488301201D490870D2E7FAF74BFE17490860052E01DBBE2E22DDFAF76E
:20FF600043FE18490968401A41F2883188421DD9286820F4007000F50070286002200D49EF
:20FF8000488008468480C680F7F710FB00200A4908700A48408B401C084948830120084916
:20FFA0000870A7E7FAF720FE0649086000BFA1E70C020020E414002069030020380A0020FA
:20FFC00092010020100200200FB42DE9F04105460E4617460B9C2088C0F30020002877D1A4
:20FFE000012D76D141F28830864272DDB7F5FA7FFBDDBDF92400002801DB014600E0414205
:020000040801F1
:20000000B1F5967F2CDAFAF7EFFD58490968401A41F28831884227D9206820F4807000F59F
:2000200080702060012052494880BDF92400002801DB014600E041424D4A91801046F7F758
:20004000B5FA00204B4908704B48008B401C4A490883012049490870BDE8F0015DF814FB08
:20006000FAF7C2FD41490860BDF92600002801DB014600E04142B1F5967F2BDAFAF7B4FDF2
:200080003F490968401A41F28831884226D9206820F4807000F58070206002203449488000
:2000A000BDF92600002801DB014600E04142304A91801046F7F77AFA00202E4908702E48EE
:2000C000008B401C2C49088301202C490870C3E73CE03CE0FAF788FD29490860BDF928001B
:2000E000002801DB014600E04142B1F5967F29DAFAF77AFD23490968401A41F2883188423F
:2001000031D9206820F4807000F580702060032017494880BDF92800002801DB014600E090
:200120004142134A91801046F7F740FA0020114908701148008B401C0F49088301200F49C2
:20014000087089E7FAF750FD0E4908600BE0FAF74BFD06490860FAF747FD09490860FAF7FF
:2001600043FD0849086000BF76E7000000020020E414002069030020380A0020920100208F
:2001800004020020080200202DE9FF410646DDE90A870C9C00252078C0F34010002878D13D
:2001A000052F08D1FAF720FD3B490860FAF71CFD3A4908606DE0012F01D0042F32D1B8F116
:2001C000320F2ADD4EBB364890FBF8F085B242F21070854200DA00E028460546FAF704FDC6
:2001E0002D490968401AA84253D9206820F020002030206001202B4948800846F7F7D6F9B8
:200200000020294908702948408A401C27494882012027490870BDE8FF81FAF7E5FC1E499C
:20022000086036E09DF8040005282EDB9DF8050058BB56BB9DF804001E4991FBF0F085B210
:2002400042F21070854200DA00E028460546FAF7CBFC12490968401AA8421AD9206820F05D
:2002600020002030206002200E4948800846F7F79DF900200C4908700C48408A401C0B49C0
:20028000488201200A490870C5E7FAF7ADFC0349086000BFBFE70000F4010020F80100201B
:2002A00048F13E00E414002069030020380A002092010020D8B805000FB42DE9F84305461A
:2002C0000E46DDE90D840F9FFAF78EFC41F28831884207D35E480078012803D05C48007884
:2002E000022819D1FAF780FC5A490860FAF77CFC58494860FAF778FC56490864FAF774FCEF
:2003000054494864FAF770FC5249C1F88000FAF76BFC5049C1F88400FAF766FC4E490968DA
:20032000401A142847D3FAF75FFC4B490860222E27D006F00F0020B39DF828001E2820DDA6
:200340009DF82900E8B9B8F1020F1AD100949DF8283028883F4A012100F088F800949DF824
:20036000283068883B4A4032022100F07FF800949DF82830A888374A8032032100F076F84E
:2003800019E0FAF731FC33490860FAF72DFC31494860FAF729FC2F490864FAF725FC2D49A4
:2003A0004864FAF721FC2B49C1F88000FAF71CFC2849C1F884003878C0F38010F0BB2078E9
:2003C00000F001002178C1F3400108442178C1F380010844022838DD386820F04000403099
:2003E0003860207800021D4948801A48418FB0F87A0001EB80011748B0F8BA0001EB00101F
:20040000164949880843154948801248818F90F87C0001EB0020114988800E48B0F8BC00A5
:20042000C8800846F7F7C2F800200D4908700D48808A401C0B498882012000E005E00A493E
:200440000870BDE8F8035DF814FB00BFF9E70000D0000020CC110020FC010020E41400205F
:2004600069030020380A0020920100202DE9F0470546884614469946089E002708E004F192
:200480000800791C30F8111020F81710781C87B2182FF4D32587192104F10800F8F75CF836
:2004A000E063E06B0A2812D2FAF79EFB2168401A43F6982188420DD93078A8F10101012223
:2004C0008A401043307001206087BDE8F087FAF78BFB2060322D03DB40F6D270854210DDDB
:2004E000FAF782FB6168401AB0F57A7F0CD93078A8F1010101228A401043307002206087BC
:20050000E3E7FAF771FB606000BFDEE710B51149487B01F0FFFC0F49487B05F083FB0E48BE
:2005200003F088FC0C48F5F707FB0C4801890C4804F0A0FE094841890A4804F09BFE0748F5
:200540008189094804F096FE01F0E4FE012001F00DFF10BDE809002084010020C41E002042
:20056000C4150020DE150020F81500202DE9FF410E4615461F461D48006850BB25B3012FF8
:2005800022D1FAF731FB40F6B83188421CD9C82E0BDD9DF80000552807D09DF80000F828F1
:2005A00001D1012411E004240FE0642E0DDA222D01D1012409E005F0F00018B1332D01D0B5
:2005C000032402E0022400E00524012001F0CEFE08E0052400200649087008460078C04344
:2005E00004490870204604B0BDE8F08184010020D2000020D400002010B502464FF4806348
:200600000AB9184610BD022902DC4FF480731FE0062906DC881E4FF4807404EB801083B20C
:2006200016E0162908DC881F00EB40004FF4007404EBC00083B20BE01E2907DCA1F1160077
:200640004FF4607404EB001083B201E04FF480631846D7E710B502464FF480630AB91846D8
:2006600010BD022902DC4FF400731FE0062906DC881E4FF4007404EB401083B216E01629D8
:2006800008DC881F00EB80004FF4207404EB800083B20BE01E2907DCA1F116004FF4707405
:2006A00004EBC00083B201E04FF480631846D7E710B50446207838B9F6F716FFFCF70CF8A2
:2006C000F7F7AEF80120207010BD10B5044601F03BFFF7F793F8FEF7C9FC0020207010BD1E
:2006E0002DE9F04107460D46144605EB4500C0F34F06207800F0010050BBB74203DAFAF721
:2007000073FA1C490860FAF76FFA1A490968401A41F2883188422AD9206820F00100401C69
:20072000206002201449488008468680F6F73EFF00201249087012480089401C1049088160
:20074000012010490870FAF74FFA0F4908600EE0FAF74AFA0C490968401A41F288318842B4
:2007600005D90A48006820F0010008490860BDE8F0810000D4020020E41400206903002067
:20078000380A002092010020D8020020840100201CB52C492C48808BC0F30B0010B940F623
:2007A000B83001E02848808B284CCDE90001237B274C247814B9274C248801E0264CE48872
:2007C0002246254CE17B224C207800F0FFF92248008941F2883188420DDA1C4A117B22460C
:2007E000127812B91B4A128801E01B4AD2881046144A00F0FFF8194A917A174A1089114AA7
:2008000000F060F90F48104C0090A37A124CA27D617DE07D00F04EF822461189D088094A94
:2008200000F0ACFA084A127A02EB4203C3EBC2124FF6FF7303EAC20122461089014AFFF7E7
:200840004FFF1CBD84010020E8090020280A0020C0010020B4080020140800202415002017
:2008600070B504460D46207868B900200F4908700F480078C0B90E480078401C0C490870CE
:20088000F6F718FE10E000200949087007480078012802DB0020207001E0F6F72DFB0348BD
:2008A0000078401C0149087070BD0000DC020020DD0200202DE9F04180460E4617461C4658
:2008C000069DFAF791F940F6B831884207D2FAF78BF940490860FAF787F93F4908602878D1
:2008E000C0F3001000283DD13C48C07A58B9A4F11900B04215DD2330874212DAFAF774F938
:20090000344908600DE0A4F11900B04209DD2330874206DA1E38404503DDFAF765F92D4903
:200920000860FAF761F92B490968401A41F2883188424CD9FAF758F927490860286820F030
:200940001000103028602648F6F730FE0020254908702548008A401C23490882012023495A
:20096000087034E01D48C07AB8B9A4F12300B0422DDD0F30B8422ADDFAF736F916490968F7
:20098000401A1B49884222D9286820F010002860FAF72AF90F49086019E0A4F12D00B0421B
:2009A00015DD1930B84212DD0A3840450FDDFAF71BF909490968401A0D49884207D92868AE
:2009C00020F010002860FAF70FF902490860BDE8F0810000C4020020C80200202415002084
:2009E000E414002069030020380A002092010020E09304002DE9F04105460E461446002760
:200A0000182E04D0242E05D0302E09D105E047F60C3707E04AF6C87704E04EF2844701E0C2
:200A20002F4600BF00BF2078C0F3800030BBBD4203DCFAF7D9F81D490860FAF7D5F81B497D
:200A40000968401A41F28831884212D9206820F00400001D20601648F6F7A8FD0020154983
:200A6000087015488089401C13498881012013490870FAF7B9F81249086014E0A7F5FA7083
:200A8000A84203DAFAF7B0F80D490860FAF7ACF80B490968401A41F28831884203D920686A
:200AA00020F004002060BDE8F0810000B0020020E414002069030020380A00209201002001
:200AC000B402002070B505460E4614462078C0F3C000002849D1012E08D1FAF785F83149E5
:200AE0000860FAF781F83049086014E040F6C410854208DAFAF778F82A490860FAF774F803
:200B00002949086007E041F64C50854203DAFAF76BF825490860FAF767F822490968401AED
:200B200041F28831884208D8FAF75EF81E490968401A40F6B831884232D9206820F0080012
:200B4000083020601948F6F731FD0020184908701848C089401C1749C881012016490870C2
:200B6000FAF742F8154908601AE0FAF73DF813490968401A41F28831884211D910480078CD
:200B800070B9104800880A280ADA0E4840880A2806DA0D48807818B9206820F008002060C8
:200BA00070BD0000B8020020BC020020E414002069030020380A002092010020C0020020B5
:200BC000D20000200A0500208C0300202DE9F0478046894615469A46DDE9086400270120AE
:200BE000B0EBE63F4ED12078C0F34000A0BBB9F1010F03DBF9F7F8FF5A490860F9F7F4FFC3
:200C000058490968401AC6F3023101EB8101052202EB410101EB4102C2EBC111B0EBC10F9F
:200C200015D9206820F00200801C20604E484580A0F80480F6F7BAFC00204C4908704C4835
:200C40004089401C4A49488101204A490870F9F7CBFF4949086082E0FFE7B9F1050F03DA50
:200C6000F9F7C2FF44490860F9F7BEFF42490968401A41F28831884271D9206820F0020031
:200C800020606CE0BAF1180F06D0BAF1240F08D0BAF1300F12D10AE0C6F30B00C0EBC0073D
:200CA0000EE0C6F30B0000EB8000470008E0C6F30B0000EB800101EBC00701E02F4600BFF0
:200CC00000BF2078C0F3400098BBBD4203DBF9F78BFF24490860F9F787FF22490968401A9F
:200CE000C6F3023101EB8101052202EB410101EB4102C2EBC111B0EBC10F15D9206820F0A5
:200D00000200801C206018484580A0F80480F6F74DFC00201549087015484089401C144969
:200D20004881012013490870F9F75EFF1249086015E0FFE707F57A70854203DAF9F754FF3D
:200D40000D490860F9F750FF0B490968401A41F28831884203D9206820F002002060BDE826
:200D6000F0870000A8020020E414002069030020380A002092010020AC0200202DE9F04164
:200D80000746884614460026F9F72EFF2B490968401A642850D3002507E02949681C31F882
:200DA000100021F81500681C85B2092DF5D3244847820A21F7F7D0FB06462068C0F340401C
:200DC00090BBB8F1320F2BDAB6F57A7F28D91D480078322830DD206820F4003000F50030FF
:200DE0002060C6F30F20184948800A211448F7F727FB154988800A211148F7F732FB12496B
:200E0000C8800846F6F7D2FB00201049087010480089401C0E49088102200E4908700BE098
:200E200000200849087007E0FFE7B6F57A7F03D8206820F400302060BDE8F081CC0200202D
:200E40001C140020D0020020E414002069030020680A00209201002010B5F9F7C5FE9C490A
:200E60000968401AC8287DD3F9F7BEFE9849086098480088C01268B997480089FA21484309
:200E80009649097A4FF47A725143B0FBF1F09249888016E08F480088C0F30A008D49098845
:200EA000012202EBE121484340118B49098948438A49097A4FF47A725143B0FBF1F08649DF
:200EC000888085488088142801DA002001E08248808881498880824840780873814800882B
:200EE0001C2190FBF1F07C49C8727F48007848737D48407888737D48007800F0010040B1B9
:200F00007448037B0846C27B79497A48F3F78CFC01E07948407A7049C8737448007800F0A2
:200F2000010010B14EF6EE6001E07448C08A6A4908826A48807EEE2815D1714880780128B3
:200F400023D16F4880684FF44821B1FBF0F06D49096808446B49086008460068000B6849C5
:200F6000C86012E0B3E05D48807EAA280DD15C4840685A49897948435849C979B0FBF1F086
:200F80003221B0FBF1F05E49C8605448007B534991F91B10084442F2107191FBF0F058492D
:200FA000C968594A1268891A884206D80120574908705348C068544908605448007801285A
:200FC00038D100205149087051480068401C5049086008468068401C8860084680684D4932
:200FE000884203D900204A498860C8603A48008B401C39490883464800680A21B0FBF1F065
:201000003549488244480078401C43490870084600781E280EDB414B30226921404803F04C
:201020009CF83B4B1022AD213D4803F096F8002039490870284800881E281ADB394800784A
:20104000401C3849087008460078052814DB0020087035480088401C334908801E48408B2B
:20106000401C1D49488331480078401C2F49087002E000202B4908702C4800783C280BDB82
:2010800000202A49087022484068401C204948600846C068401CC86023480088B0F5167F9F
:2010A0000EDB0020204908801C4B302269211C4803F053F8164B1022AD21194803F04DF857
:2010C0000E48808A0A2190FBF1F00349087510BD6C000020280A002014080020E809002058
:2010E0008C0300200A050020D200002088010020EC08002000030020B4080020E002002062
:20110000BC0300207C0000207000002074000020580B00209F86010080000020380A002085
:201120001804002075000020780000207600002010B50446F9F758FD10490968401A4EF6F4
:201140006021884218D3F9F74FFD0C4908602068401C20600A480078401C094908700846BE
:2011600000780A2808DB074B30226921064802F0F4FF00200249087010BD0000C0000020F1
:20118000C4000020380A00201804002010B50446022C1BD1F9F728FD0F490968401AC8287C
:2011A00018D30E4B4FF481520C214FF4E26003F06BF80B4B4BF620220C2140F2157003F01D
:2011C00063F8F9F711FD0449086003E0F9F70CFD0149086010BD00009000002014080020BA
:2011E0003408002001B511480078022800D108BD0098A0B1F9F7F8FC0D490968401AB0F5B9
:20120000FA7F10D9F9F7F0FC094908606B4641F204120C214FF4E26003F036F803E0F9F736
:20122000E3FC0349086000BFE1E700005D0000208800002010B50446012C13D1F9F7D4FC8F
:201240000B490968401AC82810D30A4B4FF481520C214FF4E26003F017F8F9F7C5FC04497F
:20126000086003E0F9F7C0FC0149086010BD00008C0000201408002010B5FBF73FFAFBF72E
:201280002BFAF3F799FF03F08BF9FBF703FD0A4801890A4804F050F807484189084804F077
:2012A0004BF805488189074804F046F80248018A0548F6F74BFD10BDC41E0020C4150020F4
:2012C000DE150020F8150020600400201CB50446F9F78AFC40490968401AB0F5FA7F7AD3FA
:2012E0003E480088401C3D49088008460088142837DB3B48007800F0010010B900203949FB
:20130000487437480088C0F3002010B900203549087433480078C0F3801010B900203149BB
:2013200008812F480078C0F3C01010B900202D4948812B480078C0F3001010B90020294981
:20134000888127480078C0F3401010B900202549C8814FF480512448F9F73CFC00201F49CA
:2013600008802248007868B900204FF408430C2240F2FF7100901E4802F0D2FF01201B4926
:20138000087024E019480078012820D100200190184801780078401C164A107005290CDC8A
:2013A00001A841F20133162240F2FF710090104802F0B6FF0A20F9F731F941F214030C22F8
:2013C00040F2FF710A48009402F0AAFF00BFF9F70BFC014908601CBD9C000020A00000202D
:2013E0009C010020080B0020001001405D000020D8050020A200002070B504464D480078F4
:2014000080BB08214C48F9F7DDFB4C4908704FF400414B48F9F7D6FB4A49087080214A48E9
:20142000F9F7D0FB494908704FF480714648F9F7C9FB474908704FF400514348F9F7C2FB9D
:201440004449087004214448F9F7BCFB43490870002020816081A081E0812074607401207E
:20146000344908703E48C08860803D488088A0804FF40060E0803A480089208008212E48CF
:20148000F9F7A0FB05462D480078A84202D02089401C2081294805704FF400412848F9F75D
:2014A00091FB054627480078A84202D06089401C60812448057080212348F9F783FB0546E6
:2014C00022480078A84202D0A089401CA0811F4805704FF480711C48F9F774FB05461C4846
:2014E0000078A84202D0E089401CE081184805704FF400511448F9F765FB0546154800785D
:20150000A84202D0207C401C20741248057004211148F9F757FB054610480078A84202D01D
:20152000607C401C60740D4805704FF47A70608270BD00009A000020000C014094000020DE
:20154000000801409500002000100140960000209700002098000020001401409900002009
:20156000DA1E002010B5F9F73FFB42F21071884204D2F9F739FB4149086010BDF9F734FB0D
:201580003E490968401A41F28831884274D3F9F72BFB3A4908603A48407D3A4991F823107D
:2015A000884207DA3648407D364981F823000020354908703248407D324991F822108842DD
:2015C00007DD2F48407D2F4981F8220000202E4908702B48807D2B4991F82910884207DA80
:2015E0002748807D274981F829000020264908702348807D234991F82810884207DD2048BB
:20160000807D204981F8280000201F4908701C48C07D1C4991F82B10884207DA1848C07DB1
:20162000184981F82B000020174908701448C07D144991F82A10884207DD1148C07D114956
:2016400081F82A0000201049087010480088401C0E490880084600880C280DDD0A4800781D
:2016600050B900200880012007490870054B30226921074802F071FD00BF7EE7C8000020E9
:2016800014080020380A0020CE000020CC0000201804002010B50748007850B9F9F7A4FA73
:2016A00004494968401AB0F5FA6F02D901200149087010BDA801002000B587B001200390D0
:2016C0000320049003A90E48F9F7EEF80D480068806820F001000B49096888600020009068
:2016E0000A2001900720029069460648F7F7EAF920B140F2123104A004F09CFF07B000BDBB
:2017000000080140F01E00202E2E5C436F72655C5372635C6164632E630000000EB55F480E
:201720005F49086081155E4881600021C16041614FF46021C1610020594948600B2158487C
:201740000161F7F729FE18B15A2156A004F072FF0A20009001200190072002906946504807
:20176000F7F7B0F918B164214EA004F063FF0B200090022001900720029069464848F7F7EC
:20178000A1F918B16E2147A004F054FF0C200090032001900720029069464148F7F792F94F
:2017A00018B178213FA004F045FF0D200090042001900120029069463948F7F783F918B128
:2017C000822138A004F036FF0520009001900120029069463248F7F775F918B18C2131A0A0
:2017E00004F028FF04200090062001900120029069462B48F7F766F918B1962129A004F004
:2018000019FF0F200090072001900120029069462348F7F757F918B1A02122A004F00AFFE5
:2018200007200090082001900720029069461C48F7F748F918B1AA211AA004F0FBFE0E20D4
:201840000090092001900120029069461448F7F739F918B1B42113A004F0ECFE1020009071
:201860000A2001900220029069460D48F7F72AF918B1BE210BA004F0DDFE112000900B20D6
:2018800001900720029069460548F7F71BF918B1C82104A004F0CEFE0EBD000000240140BA
:2018A000F01E00202E2E5C436F72655C5372635C6164632E6300000000B589B0234824495A
:2018C00008608115224881600021C1604161C16100201F49486001211D480161F7F75CFD59
:2018E00018B1DC211BA004F0A5FE01200190029003200590002003904FF480500890002056
:2019000007900690049001A91148F6F7D1FE18B1EB2110A004F08EFE02200190029001A953
:201920000B48F6F7C5FE18B1F4210AA004F082FE03200190029001A90548F6F7B9FE18B1FE
:20194000FD2104A004F076FE09B000BD00280140201F00202E2E5C436F72655C5372635CFE
:201960006164632E6300000010B50F480F4908602420486000210D488160C1604FF4A0216A
:2019800001610021416181610121C1610021016241628162C162F8F745F918B1582104A0BC
:2019A00004F048FE10BD0000006400402C2400202E2E5C436F72655C5372635C63616E2E8B
:2019C0006300000008B500BF0A48406940F00100084948610846406900F00100009000BFCB
:2019E00000BF022211460B20F9F7CDF90B20F9F7BDF908BD0010024000B585B000BF3A48B9
:201A0000806940F01000384988610846806900F01000009000BF00BF00BF0846806940F0C8
:201A2000200088610846806900F02000009000BF00BF00BF0846806940F0040088610846E7
:201A4000806900F00400009000BF00BF00BF0846806940F0080088610846806900F0080055
:201A6000009000BF00BF002289142048F9F7B6F84FF4634001900320029001A91B48F8F76B
:201A800013FF40F6087001900320029001A91848F8F70AFF4EF6024001900320029001A9C8
:201AA0001448F8F701FF4FF480500190124802900020039001A90F48F8F7F6FE4FF48050A1
:201AC0000190012002900220049001A90748F8F7EBFE002211462820F9F755F92820F9F704
:201AE00045F905B000BD0000001002400010014000080140000C01400000211010B50848B7
:201B0000084908600320486040F2E24105488160F9F770F818B13A2103A004F08BFD10BD56
:201B200000300040F00700202E2E5C436F72655C5372635C697764672E63000000B595B0C7
:201B40003148324908600020486020212F4881604FF41661C1600021016101214161FAF7B5
:201B600001F84FF48050119011A92848FAF7A2F82648FAF7D3FA70200F90802010900FA9B0
:201B80002248F9F778FF4FF4006008904010099000200A9039200B9000200C900D900E90AB
:201BA00008A91A48F9F728FF6FF08000174909680861602001904FF4966002900020039053
:201BC0000490059006900790002201A90F48FAF721FA042201A90D48FAF71CFA082201A980
:201BE0000A48FAF717FA6020019040F65F10029000200390082004900C2201A90348FAF7C6
:201C000009FA15B000BD0000002C0140041E002000B587B0002003900490059006900190A1
:201C200002904FF0804019490860002048600021164881604FF6FF71C16000210161416126
:201C40008161F9F78FFF18B17E2111A004F0F2FC4FF400500390002004900590069003A978
:201C60000A48FAF727F818B1862109A004F0E2FC00200190029001A90448F9F7FCFE18B12B
:201C80008C2103A004F0D6FC07B000BD441E00202E2E5C557365725C5372635C74696D2E89
:201CA0006300000000B589B01C481D4908600020486000211A4881604721C1600021016169
:201CC00080218161FAF72AFA20B14FF48F7115A004F0B0FC00200790089007A91048F9F7BC
:201CE000CAFE20B140F225110EA004F0A3FC602000902420019000200290049000226946A6
:201D00000748FAF787F920B14FF4977105A004F091FC0348FAF734F909B000BD000400409E
:201D2000841E00202E2E5C557365725C5372635C74696D2E6300000010B50C480C490860F9
:201D40004FF416504860002109488160C16001610C21416100218161C161FAF71DFC18B195
:201D6000462104A004F066FC10BD000000480040702600202E2E5C436F72655C5372635CD6
:201D800075736172742E630000BFFEE730B504460A460021002329480078401C274D2870CB
:201DA000284600780F2841DB0020287024480089244D2D88411B002907DA214800894FF67A
:201DC000FF7528441F4D2D88411B44F62060814200DD00211A4800891A4D28804FF47A7004
:201DE000414319480068081A174D2D6805EB2020154D2860284600680314C3EB031040F380
:201E00005C0000B2114D28800D488089104D2D68C5EB80200E4D2D6805EB60100C4D2860DD
:201E200028460068C0F38F20054DE88112B90020064D28800548B0F9000030BD7A03002049
:201E4000241500207C0300208003002088030020840300202DE9F04107460C4615462946E5
:201E60002046F6F76DFA8046002606E0701C34F8100024F81600701C86B2681EB042F5DCCF
:201E800024F810704046BDE8F081704702480068C0F30220704700000CED00E010B500284F
:201EA00007DA0A07140E054A00F00F031B1FD45403E00A07130E024A135410BD18ED00E0E1
:201EC00000E400E010B5F8F78FFE40F6B831884216D90C480078012812D100200949087063
:201EE0000948C07AAA280BD133200849087008460078C0430649087004484078C04348703E
:201F000010BD0000CF000020E8090020D2000020D400002010B50446012C06D0022C23D0DB
:201F2000032C40D0042C7DD15CE024224E494F48F1F7B5FD24224E494E48F1F7B0FD24224C
:201F40004D494E48F1F7ABFD24224D494D48F1F7A6FD24224C494D48F1F7A1FD24224C49F8
:201F60004C48F1F79CFD7CE024224B493F48F1F796FD242249493F48F1F791FD2422484968
:201F80003E48F1F78CFD242246493E48F1F787FD242245493D48F1F782FD242243493D486C
:201FA000F1F77DFD5DE0242241493048F1F777FD242240492F48F1F772FD24223E492F48FD
:201FC000F1F76DFD24223D492E48F1F768FD24223B492E48F1F763FD24223A492D48F1F772
:201FE0005EFD3EE0242238492048F1F758FD242236492048F1F753FD242235491F48F1F784
:202000004EFD242233491F48F1F749FD242232491E48F1F744FD242230491E48F1F73FFD85
:202020001FE0FFE7242210491048F1F738FD24220F491048F1F733FD24220F490F48F1F7BC
:202040002EFD24220E490F48F1F729FD24220E490E48F1F724FD24220D490E48F1F71FFD61
:2020600000BF00BF10BD0000B87001082C060020DC700108500600200071010874060020B3
:20208000247101089806002048710108BC0600206C710108E006002090710108B47101081C
:2020A000D8710108FC7101082072010844720108687201088C720108B0720108D47201089A
:2020C000F87201081C730108407301086473010888730108AC730108D0730108F473010871
:2020E0002DE9F04304460D46601B06B2B2F9000000FB06FC908810B90020106212E0B2F90F
:20210000040000FB06F7106AC319D069984202DAD069106206E09069984202DD90691062D0
:2021200000E0136250889CFBF0F0B2F80690D2F8208098FBF9F800EB0801002906DA106957
:20214000884203DD108A00B2BDE8F083002905DD5069884202DC908A00B2F5E708B2F3E7C9
:202160002DE9F34F83B00C46204603F0F5F800901D4800990160BDF90C001B49B1F900106D
:2021800000FB01F7FF13BDF90E001749B1F9021000FB01F84FEAE8380FFA87FB0FFA88F001
:2021A00001900198ABEB000000B2ADF80800BDF90C000D49B1F9021000FB01F5ED13BDF985
:2021C0000E000949B1F9001000FB01F6F6130FFA85F90FFA86FA09EB0A0000B2ADF80A007B
:2021E000029805B0BDE8F08F4C0000207047000030B50246B2F900303F4CB4F90040A342E4
:2022000002DD13883C4C2380B2F902303B4CB4F90040A34202DD5388384C2380B2F9043023
:20222000374CB4F90040A34202DD9388344C2380344B1B885B1C1BB2324C23802346B3F990
:202240000030B3F5FA7F56DB2B4BB3F900000023294C2380031E01DB1C4600E05C42B525E8
:202260006C43294D2D68C5EB8404274D2D6805EB6414254D2C602B461B689B121BB20B8004
:202280001E4BB3F9000000231C4C2380031E01DB1C4600E05C42B5256C431C4D2D68C5EBE7
:2022A00084041A4D2D6805EB6414184D2C602B461B689B121BB24B80114BB3F900000023DD
:2022C0000F4C2380031E01DB1C4600E05C42B5256C430F4D2D68C5EB84040D4D2D6805EB92
:2022E00064140B4D2C602B461B689B121BB28B800023044C238030BD540500205605002012
:20230000580500205A0500205C050020600500206405002000B585B000BF1148806940F017
:2023200004000F4988610846806900F00400009000BF00BF002289140A48F8F74FFC4FF491
:2023400080500190012002900220049001A90548F8F7AAFA00200449087005B000BD0000D2
:2023600000100240000801405E04002010B50446012C0BD10C480078A8B9012211030B4871
:20238000F8F72CFC0120084908700CE05CB906480078012807D1002201030448F8F71EFCF9
:2023A00000200149087010BD5E0400200008014010B5044619480078012816D1B4F5D16FC2
:2023C0000FDB17480088401C80B21549088047F23051884220DD0020114908800F49087065
:2023E0001AE000200E49088016E0B4F5BC6F10DA0C480088401C80B20A4908803C280BDD9F
:20240000F4F77AFD01200549087000200649087002E000200349088010BD00006C05002058
:20242000680500206A050020D701002038B50446002031490870F020487008460078C043AE
:202440002E4908702C484078C04348702A4840782B4B0090DA79997958792A4B1B78FAF747
:2024600055FD29480078E0B928480068284908602648406848602548806888602348C06849
:20248000C8602448406808612822234801F002FE042222A12048083801F0FCFD01201A49F2
:2024A000087020A341F205320C214FF4E26001F0EBFE04B938BDF8F797FB1C4908600020CB
:2024C0001B49087012E0F8F78FFB18490968401A64280BD9F8F788FB14490860144800780E
:2024E000401C134908701348F8F7ACFB104800780A28E8DB00BFDDE7D2000020D40000208D
:20250000080A002028040020B6000020580B0020C80A0020380A002008F40108464C414771
:20252000000000005245414459000000B8000020BC000020F007002010B50248F9F7ABFBB6
:2025400010BD0000041E002010B500210B48F9F739FE04210948F9F735FE08210748F9F70B
:2025600031FE00210548F9F7CDFA04210348F9F7C9FA08210148F9F7C5FA10BD041E0020B4
:2025800008B508490968C9084FF47A72B1FBF2F14143009100BF00BF00994A1E00920029DE
:2025A000F9D108BD000000202DE9F04705460E4617469846F8F718FB84490968401A05287E
:2025C00001D2BDE8F087F8F70FFB804908600FFA88F07F4948807F480088281AC8810846A9
:2025E000007801287ED1F8F7FFFA7949C969401AB0F5FA6F06D9F8F7F7FA7549C8610120E0
:20260000887601E0744886607148407E01281BD100206F494876002405E000206F4921F81D
:202620001400601CC4B2192CF7DB00206C4908806C4908606C4908706548408A20B16448E2
:20264000408A0002694908606148C0890A2849DB604805605E48807E00286FD15E488660A7
:202660000774C068002869D05B4880895A490989401A00B25E4908800846B0F9000000281B
:2026800003DD0846B0F9000000E00020584908800846B0F900001E2803DA0846B0F9000029
:2026A00000E01E20524908800846008818B94A48007C642842D049484949098830F8110099
:2026C00048490968081A47490860084600684849B1F900100844434908604548008881B255
:2026E0003F4800E06FE002880088401C3C4B18803A4820F8121018460088192807DB0020B2
:2027000019460880012038490870314908763548006840B334480078012810D13148006809
:202720004FF47A7148436421484329498989FA225143B0FBF1F02649088217E03FE0284891
:20274000008800EB80004100214880894143254800684FF47A72504364225043B0FBF1F013
:202760001B49088202E00020194908821C480088A0B91748B0F810901C480068C0EB0920F1
:202780001E2190FBF1F01949096808441749086008460068C0F30F200D4948820C48408AD1
:2027A000002808DD0C4880680949898AB0FBF1F00749C88203E04FF6FF700549C8820648C8
:2027C00080680549C86000BFFBE6000044030020E0020020480300200003002030140020A0
:2027E00034030020380300203C030020400300203E0300202DE9F04104460D4617469846E5
:20280000069E00201349086088601348008848600020C8600DB90846866000200F4908708B
:2028200048800520888000208860084684810020C881088248824FF6FF70C88200200876EF
:20284000487601208876F8F7CFF90449C861BDE8F081000000030020EC080020E00200201F
:202860002DE9F04106460F4606F00F0000287DD0052FFCD001206F4908700846007E0128B0
:2028800064D1002008760846408A6B49098888425CD06848408A002854D06648408A674924
:2028A0000988401A642100FB01F56448008895FBF0F004B214F11E0F44DBB4F5E47F41DAE5
:2028C00004F164005D4909884843642190FBF1F0584988825A48058804F164006843642189
:2028E00090FBF1F0574908805548458804F164006843642190FBF1F05249488050488588DD
:2029000004F164006843642190FBF1F04D4988804B48C58804F164006843642190FBF1F04F
:202920004849C8804648058904F164006843642190FBF1F0434908810B461022CD2142489D
:2029400001F00BFC3B48408A3B4908803F480078864203D13E480078874265D0032E1DD071
:2029600005DC012E08D0022E33D10EE054E0042E1DD0332E2DD123E0324800882D49488256
:202980002F4800882D49088029E02E484088294948822B4840882949088020E02948808809
:2029A00024494882264880882449088017E02548C088204948822248C088204908800EE005
:2029C000204800891B4948821D4800891B49088005E00020174948821849088000BF00BF68
:2029E0001448408A144908801248408A114988820846408A002807DD16488068898AB0FB1C
:202A0000F1F00C49C88203E04FF6FF700949C88201200849487607E000200649087048823B
:202A200088824FF6FF70C8820848067008480770BDE8F081E00200204E0300205003002005
:202A400044780108680B0020180400204C0300204D030020000300202DE9F0470746894677
:202A60001546AD10002414E057F82460300E144A02F82400C6F30741A000401C1154C6F37E
:202A80000721A000801C1154A000C01C1654601CC4B2AC42E8DB57F825A0A1000848F2F7F6
:202AA0006FFB8046BAEB080007D1AA0004494846F0F7F5FF0020BDE8F0874FF0FF30FAE776
:202AC0005017002010B5B0F900205243B0F9023003FB03210C4A914214D909163939CBB22B
:202AE0000A4C34F81320B0F9003003FB02F1CB131BB20380B0F9023003FB02F1CB131BB2B2
:202B0000438000BF10BD0000400AC139187401082DE9F14181B0BDF90400DFF86880B8F9EA
:202B2000008000FB08F1C913BDF90600DFF85480B8F9028000FB08F2D2130EB217B2F0193F
:202B400000B2ADF80000BDF90400DFF83880B8F9028000FB08F3DB13BDF90600DFF8248087
:202B6000B8F9008000FB08F4E4130FFA83FC25B2CCF10000284400B2ADF802000098BDE818
:202B8000FC8100004C00002010B504462078012808D10B4B302269210A4801F0DEFA002036
:202BA00020700AE02078022807D1074B10229B21044801F0D2FA00202070002010BD00001B
:202BC000380A002018040020680A00204FF055301F4A106040001F4A10601D480168B1F19F
:202BE000553F01D0002070471A480168B1F1AA3F01D00020F7E74FF0AA30154A1060400844
:202C0000144A106012480168B1F1AA3F01D00020E9E710480168B1F1553F01D00020E2E726
:202C20004FF055300A4A106040000A4A106008480168B1F1553F01D00020D4E705480168B7
:202C4000B1F1AA3F01D00020CDE70120CBE70000000800201008002001200C490968B1F188
:202C6000EE3F00D0002009494968B1F1CC3F00D0002006498968B1F1BB3F00D0002003497F
:202C8000C968B1F1DD3F00D000207047F82A002010B5214800780D282FD2DFE800F0070AB8
:202CA0000D101316191C1F2225282B00F0F786FA24E0F0F7B7FA21E0F0F7F3FA1EE0F0F723
:202CC00035FB1BE0F0F778FB18E0F0F7BCFB15E0F0F700FC12E0F0F744FC0FE0F0F789FC8D
:202CE0000CE0F0F7CFFC09E0F0F710FD06E0F0F751FD03E0F0F792FD00E000BF00BF064839
:202D00000078401C04490870084600780C2801DD0020087010BD0000E805002010B5F0F724
:202D20004DFAF0F77FFAF0F7BCFAF0F7FFFAF0F743FBF0F788FBF0F7CDFBF0F712FCF0F755
:202D400058FCF0F79FFCF0F7E1FCF0F723FDF0F765FD10BD10B53B480068B0F1AA3F70D141
:202D600038480068384909684840401C002866D136490860C0433649086034480068801CE5
:202D800032490860FFF784FF31480068801E304908602E4800680D302C490860FFF75CFF2E
:202DA00008B9F4F791FE2A4800680D3828490860264800680B302549086000F0C5FC0446FE
:202DC00034B1012C0AD0032C04D0042C05D100E007E006E0F4F778FE03E000BFF4F774FEF1
:202DE00000BF00BF1A4800680B381949086017480068C01C1549086000F044F808B9F4F73D
:202E000063FE13480068C01E114908600F480068401D0E490860FFF7D9FE08B9F4F754FE48
:202E20000B480068401F0A490860222003F0A2FD08B9F4F749FE00200249086001E0F4F757
:202E400043FE10BDC0260020E4260020B0260020D426002010B500F047FC00F055FC00F0FB
:202E600001F810BD4FF0EE30054908604FF0CC3048604FF0BB3088604010C8607047000055
:202E8000F82A0020F0B55527552F01D00020F0BDAA27AA2F01D00020F9E74FF05531B1F1CB
:202EA000553F01D00020F2E74FF0AA31B1F1AA3F01D00020EBE74FF47A714A008C1840F6FA
:202EC000B830844201D00020E1E74FF0FF3102228C18012C01D00020D9E74FF47A73F94D00
:202EE0005E1916F57A7F01D00020D0E76FF0004301255E19B6F1004F01D00020C7E76FF07C
:202F0000004302255E19981C864201D00020BEE76FF0004303255E19D81C864201D00020D0
:202F2000B5E74FF4FA614A108C1AB4F57A7F01D00020ACE74FF4FA614A1C8C1A601C08B152
:202F40000020A4E7002101228C1A601C08B100209DE74FF47A735D005E1B16F57A7F01D028
:202F6000002094E7002301255E1B701C08B100208DE74FF0004301255E1B581E864201D0EB
:202F8000002084E74FF47A71491C0846814201D000207CE74FF0FF31491C09B1002076E7A3
:202FA0000021491C012901D0002070E74FF47A735B1C1846834201D0002068E700235B1C75
:202FC000012B01D0002062E76FF000435B1CB3F1004F01D000205AE74FF000435B1C1846F6
:202FE000834201D0002052E74FF47A71491E0846814201D000204AE70021491E481C00B17D
:2030000045E74FF0FF31491E881C00B13FE74FF47A735B1E1846834201D0002037E74FF019
:2030200000435B1E1846834201D000202FE76FF000435B1E1846834201D0002027E700234A
:203040005B1E581C00B122E764210A2201FB02F4B4F57A7F01D0002019E76FF07041112250
:2030600001FB02F49848844201D000200FE74FF0FF31012201FB02F4601C08B1002006E70B
:203080006421002201FB02F40CB10020FFE64FF47A710A22B1FBF2F4642C01D00020F6E68C
:2030A00001210A22B1FBF2F40CB10020EFE600210A22B1FBF2F40CB10020E8E64FF47A71C6
:2030C0000022B1FBF2F40CB10020E0E64FF0FF310122B1FBF2F4601C08B10020D7E6022140
:2030E0004C00042C01D00020D1E602210C02B4F5007F01D00020CAE60221CC070CB10020DF
:20310000C5E64FF6FF714C084810844201D00020BDE64FF6FF710C0AFF2C01D00020B6E6C6
:203120004FF6FF71CC0F0CB10020B0E6012109B90020ACE6002109B10020A8E6FF2109B98B
:203140000020A4E664210A22914201D800209EE664216422914201D9002098E60A216422BD
:20316000914201D9002092E64FF0FF310022914201D800208BE66FF00043DD07AB4201DCEC
:20318000002084E60A216422914201D300207EE664216422914201D2002078E664210A22E9
:2031A000914201D2002072E600214A1E914201D300206CE64FF000435D1EAB4201DB002069
:2031C00065E664210A22914201D200205FE664216422914201D2002059E60A216422914254
:2031E00001D3002053E64FF0FF310022914201D200204CE66FF00043DD07AB4201DA0020AB
:2032000045E60A216422914201D900203FE664216422914201D9002039E664210A22914265
:2032200001D8002033E600214A1E914201D900202DE64FF000435D1EAB4201DD002026E61F
:2032400064216422914201D0002020E64FF0FF310A46914201D0002019E600210022914201
:2032600001D0002013E64FF000431D46AB4201D000200CE600230025AB4201D0002006E69D
:203280006FF000431D46AB4201D00020FFE564216422914201D00020F9E54FF0FF310A46FB
:2032A000914201D00020F2E500210022914201D00020ECE54FF000431D46AB4206D00020D3
:2032C000E5E5000030F8FFFFEFFFFF0F00230025AB4201D00020DAE56FF000431D46AB422B
:2032E00001D00020D3E50121002221B9022904D0032906D103E0921C04E0121D02E0083245
:2033000000E000BF00BF022A01D00020BFE502210022012904D0022904D0032906D103E066
:20332000921C04E0121D02E0083200E000BF00BF042A01D00020AAE503210022012904D060
:20334000022904D0032906D103E0921C04E0121D02E0083200E000BF00BF082A01D000202A
:2033600095E504210022012904D0022904D0032906D103E0921C04E0121D02E0083200E0EC
:2033800000BF00BF0AB1002081E50021002211B10AB100207BE501B90AB1002077E500211C
:2033A000012211B10AB1002071E511B90AB900206DE50121012201B10AB9002067E511B908
:2033C0000AB9002063E50121FF2201B10AB900205DE511B90AB9002059E50021FF2211B1B9
:2033E0000AB1002053E511B90AB900204FE54FF055310A4681EA02040CB1002047E54FF00B
:2034000055314A0081EA0204601C08B100203EE50021002281EA02040CB1002037E54FF007
:20342000FF310A4681EA02040CB100202FE500214A1E81EA0204601C08B1002027E54FF010
:203440005531CC43B4F1AA3F01D000201FE5E443B4F1553F01D0002019E50021CC43601C59
:2034600008B1002013E5E4430CB100200FE501200DE5000008B500BF7148806940F004001E
:203480006F4988610846806900F00400009000BF00BF00BF0846806940F0080088610846ED
:2034A000806900F00800009000BF00BF00BF0846806940F0100088610846806900F01000C7
:2034C000009000BF00BF00BF0846806940F0200088610846806900F02000009000BF00BF5A
:2034E0005848F4F745FB08B9002008BD5648F4F73FFB08B90020F8E75448F4F739FB08B95C
:203500000020F2E75248F4F733FB08B90020ECE74B48806920F00400494988610846806909
:2035200020F0080088610846806920F0100088610846806920F0200088614648F1F7E2F8AA
:2035400000BF3F48C06940F000703D49C8610846C06900F00070009000BF00BF3E48F1F75A
:20356000C9FD08B90020C0E73548C06920F000703349C86100BF0846406940F001004861A2
:203580000846406900F00100009000BF00BF3348F2F762FB08B90020A7E72948406920F0DB
:2035A00001002749486100BF0846806940F4007088610846806900F40070009000BF00BFC5
:2035C00000BF0846806940F4806088610846806900F48060009000BF00BF2148F0F7AAFFE6
:2035E00008B9002081E71F48F0F7A4FF08B900207BE71348806920F40070114988610846F5
:20360000806920F48060886100BF0846806940F4006088610846806900F40060009000BF97
:2036200000BF114801F081FB08B900205DE70448806920F4006002498861012055E70000A6
:203640000010024000080140000C01400010014000140140000001400064004008000240AD
:203660000024014000280140002C014010B5002419480068194909684840401C48BB164845
:2036800000681749884210D316490846F0F7FEF8012801D1042400E0032411484B380E49CE
:2036A0000860C0430D49086014E00E490A480068F0F7ECF801280AD10748006810300649C7
:2036C000086008460068C0430449086002E0032400E00124204610BD1C060020200600204B
:2036E0007B000020FC05002004480549086008460068C04303490860704700003000002098
:203700001C0600202006002010B50A480A490860C0430A4908600A480A4908600846F6F749
:20372000A8FD08480068806840F0010005490968886010BD00300008CC260020F02600201F
:2037400000300240F005002010B502241F4800681F4909684840401C002834D11B48006873
:203760001C49884223D2002006E01849096851F82010194A1160401C18498908174A9209B6
:20378000B1FBF2F18142F0D814498908134A9209B1FBF2F10D4A126802EB81010B4A116094
:2037A00011460968C9430A4A116000240CE00A48006808490968884201D1042400E0032419
:2037C000FFF7A2FF00E00124204610BDCC260020F0260020008D010800300240005D01006C
:2037E00070B50A2050490870F7F740FA00F0DAFF00204E490860C0434D4908604B4800685D
:20380000801C4A490860FFF789FA49480068801E47490860EFF786FC0C20434908704348E6
:2038200000680B304149086042484349086008460068806840F00100096888603E48F6F7DA
:2038400018FD002405E03D4951F8240039490860641C3B48B4EB900FF5D3364805683948F8
:203860000068854201D0F4F72FF9314800680B382F4908600E202C4908702C480068C01C5E
:203880002A490860FFF7FEFA08B9F4F71DF928480068C01E26490860102023490870234891
:2038A0000068401D21490860FFF790F908B9F4F70BF91F480068401F1D49086012201A49B1
:2038C00008701A480068C01D18490860FFF7D2FD08B9F4F7F9F8142013490870FFF7CAFDD9
:2038E00008B9F4F7F1F812480068C01F1049086016200D4908701C2003F03CF808B9F4F7BE
:20390000E3F81820084908704FF400510804F0F736F808B9F4F7D8F800F0AEFFAA200549E5
:203920000871EFF7E3FB70BDEC050020B0260020D426002000300240F0050020003000083D
:20394000005D0100008D010810B5124800780A281EDB00200F4908704FF0AA300E490860E9
:2039600040080E49086072B6FFF780FE044662B634B1012C08D0032C05D0042C02D100E071
:2039800005E004E000BF00BFF4F79EF800BF00BF10BD000059000020C0260020E42600206B
:2039A000002107E041F64C5100BF0A00A1F1010399B2FAD10200A0F1010398B2F2D170475B
:2039C000002106E0072100BF0A00A1F1010399B2FAD10200A0F1010398B2F3D17047704730
:2039E0002DE9F143BDF9000044F2F30100FB01F9BDF902004FF416514843C0F10008444678
:203A000008EB09004710A8EB09004610002F0FDA002E03DA0520F749088018E0002C03DC4E
:203A20000420F449088012E00320F24908800EE0002E03DB0220EF49088008E0002C03DCF6
:203A40000620EC49088002E00120EA4908800020E9490870E748008807287BD2DFE800F011
:203A60007A044D97E0FCFB0004F51650801B4FF4966101EBA040E14908800846008800EB9A
:203A80006640488008464088A0EB6440888008460088C0F5166080B2E22803DD40F65F10A9
:203AA000C88029E0D5480088D4494988401A85B2B5F58B7F05DBD14800883338CF49C88091
:203AC0001AE0CE480088C0F5166080B28A2813DDCA480088E230C949C8800846C088B0F50E
:203AE000166F09DB0120C4490870C448C088C0F59650401EC149C88074E107F51650801BC6
:203B00004FF4966101EBA040BC4908800846008800EB6640488008460088A0EB67408880D3
:203B200008464088C0F5166080B2E22803DD40F65F10C8802AE0B1484088B0490988401A8C
:203B400085B2B5F58B7F06DBAC4840883338AB49C8801BE045E1A9484088C0F5166080B2FF
:203B60008A2813DDA5484088E230A449C8800846C088B0F5166F09DB01209F4908709F489B
:203B8000C088C0F59650401E9C49C8802AE1C4F5165038444FF4966101EBA04097490880A3
:203BA00008460088A0EB674088800846808800EB6440488008464088C0F5166080B2E228CB
:203BC00003DD40F65F10C88029E08C4840888B498988401A85B2B5F58B7F05DB87484088D2
:203BE00033388649C8801AE084484088C0F5166080B28A2813DD81484088E2307F49C88003
:203C00000846C088B0F5166F09DB01207A4908707A48C088C0F59650401E7849C880E1E0D7
:203C200004F51650801B4FF4966101EBA040734908800846008800EB6640488008464088FB
:203C4000A0EB6440888008468088C0F5166080B2E22806DD01E078E02EE040F65F10C88059
:203C600029E06648808865494988401A85B2B5F58B7F05DB6148808833386049C8801AE0DA
:203C80005E488088C0F5166080B28A2813DD5B488088E2305949C8800846C088B0F5166F10
:203CA00009DB0120544908705448C088C0F59650401E5249C88095E007F51650801B4FF475
:203CC000966101EBA0404D4908800846008800EB6640488008460088A0EB67408880084676
:203CE0008088C0F5166080B2E22803DD40F65F10C88029E04148808840490988401A85B243
:203D0000B5F58B7F05DB3D48808833383B49C8801AE03A488088C0F5166080B28A2813DDC8
:203D200036488088E2303549C8800846C088B0F5166F09DB0120304908703048C088C0F5FA
:203D40009650401E2D49C8804CE0C4F5165038444FF4966101EBA0402849088008460088C5
:203D6000A0EB674088800846808800EB6440488040F65F10C88008460088C0F5166080B23C
:203D8000E22803DD40F65F10C88029E01B4800881A498988401A85B2B5F58B7F05DB174860
:203DA000008833381549C8801AE014480088C0F5166080B28A2813DD10480088E2300F4943
:203DC000C8800846C088B0F5166F09DB01200A4908700A48C088C0F59650401E0749C880E0
:203DE00000E000BF00BF0448007848B9002000F0FBFA08E0340000203600002038000020B1
:203E0000022000F0F1FA40F64C100949C880088800F0D2FA0649488800F0D4FA04498888F3
:203E200000F0D6FA0249C88800F0D8FABDE8F883380000202DE9F0410446002500260027EA
:203E4000F3F79AF8A84618E000BF334800780128FBD10020304908703048008805442F4888
:203E6000408806442D48808807440C212C48F8F789F908F101001FFA80F8B8F10A0FE3DB4B
:203E80000A20B5FBF0F0274908800A20B6FBF0F048800A20B7FBF0F088800846008846F21B
:203EA000A81188421DDB1F48008849F64041884217DC1C48408846F2A811884211DB1948E7
:203EC000408849F6404188420BDC1648808846F2A811884205DB1348808849F640418842BB
:203EE00016DD206820F4802000F58020206006200D4948800846F3F759FB00200B490870C2
:203F00000B484089401C0A494881022009490870F3F732F8BDE8F08108050020FC040020AA
:203F2000041E00200E050020E414002069030020680A00209201002008B50020009053481B
:203F40000088072870D2DFE800F0933362630405320000BF4E480088404201B211F5004F84
:203F600004DA4FF40040ADF8000009E0B1F5004F04DB47F6FF70ADF8000001E0ADF8001097
:203F800043484088404201B211F5004F04DA4FF40040ADF8020009E0B1F5004F04DB47F642
:203FA000FF70ADF8020001E0ADF8021061E000BF37484088404201B211F5004F04DA4FF461
:203FC0000040ADF8020009E0B1F5004F04DB47F6FF70ADF8020001E0ADF802102C488088D6
:203FE000BDF80220801A01B2B1F5004F04DB47F6FF70ADF8000009E011F5004F04DA4FF419
:204000000040ADF8000001E0ADF8001031E000BF1F480088404201B2B1F5004F05DB47F61F
:20402000FF70ADF800000AE022E011F5004F04DA4FF40040ADF8000001E0ADF80010144833
:204040008088BDF80020801A01B211F5004F04DA4FF40040ADF8020009E0B1F5004F04DB1C
:2040600047F6FF70ADF8020001E0ADF8021000E000BF00BFBDF900000011ADF80000BDF9D5
:2040800002000011ADF80200009808BD34000020140500202DE9F04781460D461646304643
:2040A000F11706EB9171C1F38707002415E015F824000106A000401C285C01EB0041A00025
:2040C000801C285C01EB0021A000C01C285C08440A4941F82400601CC4B2BC42E7DB31468E
:2040E0002846F1F74DF88046044840F827807A1C01464846F3F75CFBBDE8F08750180020E4
:204100002DE9F04190B080460D4616463046F11706EB9171C1F38707002414E0A000C01C5C
:20412000285C0106A000801C285C01EB0041A000401C285C01EB002015F8241008444DF8A9
:204140002400601CC4B2BC42E8DB3A4669464046F3F72EFB10B0BDE8F0812DE9F8438146D2
:204160000D4616461F46002000908046002420E02819C1B26A464846F3F75EF8401C18B932
:204180004FF0FF30BDE8F883385D9DF8001088420DD0385D00902819C1B29DF80020484694
:2041A000F3F7A0F8401C10B94FF0FF30EAE7601CC4B2B442DCDB31463846F0F7C9FF804610
:2041C0004FEA28200090A819C1B29DF800204846F3F788F8401C10B94FF0FF30D2E708F0A9
:2041E000FF000090A819401CC1B29DF800204846F3F778F8401C10B94FF0FF30C2E70020A7
:20420000C0E7000070B505460C4664BB1A4800691A4948600B46302269212846FFF79DFF13
:20422000401C28B9154B302269212846FFF795FF11480068124908600F48406848600E488C
:20424000806888600C48C068C8600B461022AD212846FFF782FF401C28B9094B1022AD2123
:204260002846FFF77AFF064800680A21B0FBF1F004494882002070BDC80A0020380A00203C
:20428000580B0020140800202DE9F04706468846174699460025FCB255201F490870AA20CA
:2042A0004870084680F80280A01CC870380A08710846447122464946801DEFF7F0FB552072
:2042C00016490870AA20487030128870CE70221D1149891C1148001DEFF7E1FB04F1080199
:2042E0000E48F0F74DFF0546280EA11D0A4A5054C5F30741E01D1154C5F30721401C1154FB
:20430000401C1554F021401C1154421C02493046F0F752FEBDE8F087760D0020750E00204E
:204320002DE9F04781460E4690461F46DDF820A00025FCB255201E490870AA204870300A62
:204340008870CE70084680F80480A01C4871380A88710846C471224651460830EFF79FFBF3
:2043600004F1080212491348EFF799FB04F108011048F0F705FF0546280E04F108010C4AF8
:204380005054C5F3074104F109001154C5F30721401C1154401C1554F021401C1154401C82
:2043A000C2B20349484601F0A2F9BDE8F0870000740F00200A10002001490968486370470D
:2043C000041E00200149096888637047041E002001490968C8637047041E00200149096862
:2043E00008647047041E002008490968096A21F40051064A1268116204490968096A41EA24
:204400000031024A1268116270470000041E002010B51048007801281BD10F4A32210F488C
:2044200000F048F90446EFF739FD0D49086008460068EFF756FD0B49086000200549087096
:20444000084800681E2804DA0348008800B20649088010BD080100201401002028070020AA
:204460000C01002010010020040100202DE9F04705460C4616461F46DDE90889F6F7B4FB1B
:2044800019490968401A32282BD3F6F7ADFB1649086005FB06F090FBF7F000FB08F000EBF5
:2044A000C000000142F2107190FBF1F0208020880E49096808440D4908600D480078401CD7
:2044C0000B4908700846007808280ADB0020087006480068C0F3CF00A9F800000020034958
:2044E0000860BDE8F0870000D4030020DC030020D803002070B504460D461646F6F774FBCD
:2045000024490968401A322841D3E07828B9F6F76BFB214908600120E070F6F765FB1E4972
:204520000968401AB0F57A6F04D90020A0704FF6FF70A060208980B24FF6FF71884202D134
:204540000020A07001E00120A070A078012812D1A06810B94FF0FF30A0604FF4B47070439C
:20456000A168B0FBF1F0208020880A220B49FDF771FC288007E00020208028800A2107480C
:20458000F0F747F970BDF6F72FFB0249086000BFF8E70000E0030020E4030020B015002070
:2045A00000B585B000BF1048806940F020000E4988610846806900F02000009000BF00BF2C
:2045C00004200190094802900120039001A90848F6F76AF9002202210820F6F7D4FB0820F4
:2045E000F6F7C4FB05B000BD0010024000001110001401402DE9F04104460D4617461E4630
:20460000F6F7F2FA28490968401A32284AD3E07828B9F6F7E9FA254908600120E070F6F7D1
:20462000E3FA22490968401A4FF47A6191FBF6F1884201D90020A070A078012822D1A068C6
:2046400010B94FF0FF30A0604FF4B4707843B0FBF6F0A168B0FBF1F0208020880A2214490A
:20466000FDF7F8FB2880F6F7BFFA6168411AA068B1EB400F12D940F20E41A0684843800A65
:20468000A0600BE00020208028800A210848F0F7C0F84FF0FF30A060BDE8F081F6F7A4FA9E
:2046A0000149086000BFF7E7CC030020D00300209C1500202DE9F74F88B0044689464FF00C
:2046C000000BDA460020069000210F4688460D460E4600BF0FE034F81B00EFF7F5FB3A46C3
:2046E0004346CDE90401EFF7C3FA074688460BF1010000F0FF0BCB45EDDB4846EFF7E4FB96
:2047000002460B46CDE9020138464146EFF757FBCDE90401EFF75DFC06900698EFF7FAFB01
:2047200081B20A9801804FF0000A23E034F81A00EFF7B4FB00900699EFF762FA029034F8CD
:204740001A00EFF7ABFB00900699EFF759FA01900299EFF75BFA0390EFF728FC2A4633465E
:20476000CDE90401EFF784FA05460E460AF1010000F0FF0ACA45D9DB2846314602F0C4FB2D
:20478000CDE90201EFF7F9FB80B20590EFF79CFB05460E4628463146EFF7EFFB80B20BB001
:2047A000BDE8F08F10B594B009200A904FF480300B9000200C9001200E901090022011909D
:2047C000C10312914FF4E01113910AA8F6F7BAFD18B1CD211AA001F02DFF0F2005900220D0
:2047E0000690002007904FF48060089000200990022105A8F6F764FC18B1DB2110A001F075
:2048000019FF022001908003039001A8F6F7C0FB18B1E2210AA001F00DFFF6F723FD4FF4A3
:204820007A71B0FBF1F42046F7F7C6F80420F6F7A9FF00221146501EF6F7A5FA14B010BD2E
:204840002E2E5C53656C6654657374557365725C7372635F6D6964646C6577617265735CE7
:2048600073746D33326678785F535455737461727475702E6300000010B590B0022006906D
:2048800001200A9010200B9000200D9006A8F6F759FD20B140F2031114A001F0CBFE0F2030
:2048A00001900020029003904FF48060049000200590002101A8F6F703FC20B140F21111DB
:2048C0000AA001F0B7FEF6F7CDFC4FF47A71B0FBF1F42046F7F770F80420F6F753FF0022D3
:2048E0001146501EF6F74FFA10B010BD2E2E5C53656C6654657374557365725C7372635FAC
:204900006D6964646C6577617265735C73746D33326678785F535455737461727475702EFF
:2049200063000000034618044843B0FBF2F0704710B5F6F78FF9F7F759F803480078401C48
:204940000149087010BD00005900002010B594B009200A904FF480300B9000200C90012018
:204960000E90109002201190C10312914FF4E01113910AA8F6F7E6FC20B140F293111CA013
:2049800001F058FE0F20059002200690002007904FF48060089000200990022105A8F6F76C
:2049A0008FFB20B140F2A11111A001F043FE022001908003039001A8F6F7EAFA20B14FF47E
:2049C000D4710BA001F036FEF6F74CFC4FF47A71B0FBF1F42046F6F7EFFF0420F6F7D2FEAD
:2049E00000221146501EF6F7CEF914B010BD00002E2E2F436F72652F5372632F6D61696E4C
:204A00002E6300001148006840F001000F490860084640680E4908400C494860084600680B
:204A20000C490840094908600846006820F4802008600846406820F4FE0048604FF41F003B
:204A40008860C8030449086070470000001002400000FFF8FFFFF6FE08ED00E010B5024818
:204A6000F7F7C2F910BD0000041E002000220268184B984208D0B0F1804F05D0164B98425D
:204A800002D0164B984203D122F070024B681A43104B984208D0B0F1804F05D00E4B98421C
:204AA00002D00E4B984203D122F44072CB681A4322F080024B691A4302608B68C3620B6833
:204AC0008362044B984201D10B6903630123436170470000002C01400004004000080040A4
:204AE00030B50023012404FA01F3046A9C430462046A02FA01F52C43046230BD30B50023BA
:204B0000042404FA01F3046A9C430462046A02FA01F52C43046230BD30B50C460021816865
:204B200021F47F4142EA032525432943816030BD0A460021816821F0700142F00703194336
:204B40008160704730B5002400220023056A25F001050562026A4368846924F0700424F0DE
:204B600003040D682C4322F002028D682A430D4DA84206D100BF22F00802CD682A4322F028
:204B80000402084DA84207D123F4807323F400734D692B438D692B43436084614D684563F7
:204BA000026230BD002C014030B5002400220023056A25F010050562026A4368846924F4CD
:204BC000E04424F440740D6844EA052422F020028D6842EA05120F4DA84207D100BF22F0BE
:204BE0008002CD6842EA051222F04002094DA84209D123F4806323F400634D6943EA85036E
:204C00008D6943EA8503436084614D688563026230BD0000002C014030B5002400220023B8
:204C2000056A25F480750562026A4368C46924F0700424F003040D682C4322F400728D6848
:204C400042EA05220E4DA84207D100BF22F40062CD6842EA052222F48062094DA84209D113
:204C600023F4805323F400534D6943EA05138D6943EA05134360C4614D68C563026230BDB4
:204C8000002C014030B5002200230024056A25F480550562036A4468C26922F4E04222F403
:204CA00040720D6842EA052223F400538D6843EA0533074DA84204D124F480444D6944EAE3
:204CC00085144460C2614D680564036230BD0000002C014030B50B46144600210022026A58
:204CE000056A25F001050562816921F0F00141EA041122F00A021A438161026230BD30B504
:204D00000B46144600210022056A25F0100505628169026A21F4704141EA043122F0A00275
:204D200042EA03128161026230BD0146002240F205100860086882B240F20510824201D067
:204D40000020704740F28A200860086882B240F28A20824201D00020F3E70020086045F26A
:204D600055504860486882B245F25550824201D00020E6E742F6A8204860486882B242F6E0
:204D8000A820824201D00020DBE70020486045F255508860886882B245F25550824201D0B3
:204DA0000020CEE74AF6A2208860886882B24AF6A220824201D00020C3E70020886045F270
:204DC0005550C860C86882B245F25550824201D00020B6E742F6AA20C860C86882B242F6AE
:204DE000AA20824201D00020ABE70020C86045F255508861886982B245F25550824201D0FF
:204E000000209EE74AF6AA208861886982B24AF6AA20824201D0002093E70020886145F25C
:204E20005550C861C86982B245F25550824201D0002086E74AF6AA20C861C86982B24AF669
:204E4000AA20824201D000207BE70020C86141F255500862086A82B241F25550824201D0D3
:204E600000206EE742F6AA200862086A82B242F6AA20824201D0002063E70020086245F2E9
:204E800055504862486A82B245F25550824201D0002056E74AF6AA204862486A82B24AF635
:204EA000AA20824201D000204BE70020486245F255508862886A82B245F25550824201D01A
:204EC00000203EE74AF6AA208862886A82B24AF6AA20824201D0002033E70020886245F259
:204EE0005550C862C86A82B245F25550824201D0002026E74AF6AA20C862C86A82B24AF605
:204F0000AA20824201D000201BE70020C86255200863086B82B2552A01D0002011E7AA200D
:204F20000863086B82B2AA2A01D0002009E70020086345F255504863486B82B245F25550D5
:204F4000824201D00020FCE64AF6AA204863486B82B24AF6AA20824201D00020F1E6002068
:204F6000486345F255508863886B82B245F25550824201D00020E4E64AF6AA208863886B55
:204F800082B24AF6AA20824201D00020D9E60020886345F25550C863C86B82B245F255500A
:204FA000824201D00020CCE64AF6AA20C863C86B82B24AF6AA20824201D00020C1E6002068
:204FC000C86345F255500864086C82B245F25550824201D00020B4E64AF6AA200864086CA1
:204FE00082B24AF6AA20824201D00020A9E60020086441F215508864886C82B241F215505F
:20500000824201D000209CE640F60A208864886C82B240F60A20824201D0002091E6002039
:205020008864086101208CE62DE9F04104460E461746984627480078012812D1264801788E
:205040000078401C244A1070244820F811601046007832281CDB00201E49087011460870AC
:2050600016E032221D493046FCF7F4FE05462088A84209DDF5F7B8FD19490968401AB0F5EF
:205080007A7F05D9258003E0F5F7AEFD1449086040F634007843642190FBF1F0C0F58050BA
:2050A0002188884203DBF5F79FFD0E490860F5F79BFD0C490968401A42F21071884206D956
:2050C0000948007820F00100401C07490870BDE8F0810000ED030020EE0300201216002053
:2050E000F4030020F0030020E80300202DE9F04104460E461746984627480078012812D168
:20510000264801780078401C244A1070244820F811601046007832281CDB00201E490870D3
:205120001146087016E032221D493046FCF792FE05462088A84209DDF5F756FD1949096822
:20514000401AB0F57A7F05D9258003E0F5F74CFD1449086040F634007843642190FBF1F0E1
:20516000C0F580502188884203DBF5F73DFD0E490860F5F739FD0C490968401A42F210717D
:20518000884206D90948007820F00200801C07490870BDE8F0810000F8030020F9030020DA
:2051A0007616002000040020FC030020E80300202DE9F04104460E461746984627480078EE
:2051C000012812D1264801780078401C244A1070244820F811601046007832281CDB0020E6
:2051E0001E4908701146087016E032221D493046FCF730FE05462088A84209DDF5F7F4FC1B
:2052000019490968401AB0F57A7F05D9258003E0F5F7EAFC1449086040F63400784364211C
:2052200090FBF1F0C0F580502188884203DBF5F7DBFC0E490860F5F7D7FC0C490968401ACB
:2052400042F21071884206D90948007820F00400001D07490870BDE8F081000004040020F0
:2052600005040020DA1600200C04002008040020E80300202DE9F04704460F46E7824FF0FA
:20528000090841462046F3F75BF8C01B0FFA80F919F1780F41DDB9F1780F3EDA002606E072
:2052A000701C34F8100024F81600701CC6B2A8F10100B042F4DC24F8107041462046F3F721
:2052C000BFF805B2608AA84200DA658241462046F3F7C7F805B2A08AA84200DDA58211480D
:2052E000844206D12346182215210F48FEF735FF16E00E48844206D12346182232210A4887
:20530000FEF72BFF0CE00A48844209D1234618224F210548FEF721FF02E000200549087053
:20532000BDE8F087C415002018040020DE150020F8150020EC03002003B5642202760021F6
:2053400006E000EB4102BDF8043013804A1CD1B20C29F6D30CBD000008B5024602F50040D1
:2053600081B20846CB1701EB936399114FF6FE70014001F4407038B3B0F5807F36D0B0F56B
:20538000007F03D0B0F5407F40D10DE0C8B2214B33F81000ADF80200C8B2C0F1FF0033F83C
:2053A0001000ADF8000032E0C8B2C0F1FF00194B33F81000ADF80200C8B233F8100040427F
:2053C00000B2ADF8000022E0C8B2124B33F81000404200B2ADF80200C8B2C0F1FF0033F832
:2053E0001000404200B2ADF8000010E0C8B2C0F1FF00084B33F81000404200B2ADF8020041
:20540000C8B233F81000ADF8000000E000BF00BF009808BDA674010870B505466C6A0020EE
:20542000E085E0842046F7F710F870BD2DE9F04106460D461446002025490870F5F7D4FB19
:205440002349486005F0FF08A5F50040083830B1A0F6FA70B8B1B0F5545F2DD108E0424612
:2054600021461C48EEF71BFB00201B4908702BE023462A46314640F21560FEF705FF01204E
:205480001649087020E02178627801EB02218FB2002007E0124931F81010B94200DD03E00C
:2054A000411CC8B20B28F5D300BF00F14601CAB20C4981F8272007E023462A46314640F229
:2054C0001560FEF7E1FE00BF00BFBDE8F0810000A80100209C010020A60100205D00002025
:2054E0006C7801085408002010B50A46C37893421EDBC3681B68DB6823F02003C468246846
:20550000E360C3789B1AC370C3681B68DB6843F02003C4682468E360114683780B4499B2F7
:2055200003788B4202DC0378CB1A99B281701BE0C3681B68DB6823F02003C4682468E3608C
:20554000C1780023C370C3681B68DB6843F02003C4682468E3608378194403788B4202DCFC
:205560000378CB1A99B2817010BD0168C96821F490710268D1600168496921F001010268DF
:205580005161202180F83A10704710B504462068C06820F040002168C860202084F83900EA
:2055A0002046F7F798F8002010BD00BFC27803789A42FBD0C2681268D26822F08002C36862
:2055C0001B68DA60C2788AB9C26812681268C2F3C0125AB1C26812685160C2681268D268AE
:2055E00042F08002C3681B68DA60704743788268D1544278521CD2B2427003789A4201D107
:2056000000224270C278521CC270C2681268D26842F08002C3681B68DA6000BFE5E710B512
:2056200002460B461946D4789C4209DB94780C44A1B214788C4204DC14780C1BA1B200E095
:2056400000219468605C10BD70B5044694F83A0022284AD1A068B0F5805F13D1A56A206902
:2056600040B920684068C0F308002880A06A801CA06219E020684068C0B22880A06A401C4D
:20568000A06211E0206938B920684068C1B2A26A501CA062117007E02068406800F07F0178
:2056A000A26A501CA0621170E08D401E80B2E085C8B92068C06820F020002168C8602068F3
:2056C000C06820F480702168C8602068406920F0010021684861202084F83A002046F6F730
:2056E000F9FF002070BD0020FCE70220FAE7F0B507460D461646002405E0295D3846FFF7BB
:2057000054FF601CC4B2B442F7DBF0BD2DE9F041044600252068006920F44050E1680843F0
:20572000216808612169A06808436169084305432068C06841F20C61884328432168C86006
:205740002068406920F44070A1690843216848615F49206888425CD1F5F79AFD00EBC00177
:2057600001EB001061688900B0FBF1F6F5F790FD00EBC00101EB001061688900B0FBF1F04A
:205780006421B0FBF1F000EBC00101EB0010A6EB8000322101EB00106421B0FBF1F000F0EF
:2057A000F006F5F775FD00EBC00101EB001061688900B0FBF1F06421B0FBF1F006EB0016F7
:2057C000F5F766FD00EBC00101EB001061688900B0FBF1F7F5F75CFD00EBC00101EB001000
:2057E00061688900B0FBF1F06421B0FBF1F000EBC00101EB0010A7EB8000322101EB0010B1
:205800006421B0FBF1F000F00F003044216888605BE0F5F72DFD00EBC00101EB00106168D1
:205820008900B0FBF1F6F5F723FD00EBC00101EB001061688900B0FBF1F06421B0FBF1F0AA
:2058400000EBC00101EB0010A6EB8000322101EB00106421B0FBF1F000F0F006F5F708FD58
:2058600000EBC00101EB001061688900B0FBF1F06421B0FBF1F006EB0016F5F7F9FC00EBBE
:20588000C00101EB001061688900B0FBF1F7F5F7EFFC00EBC00101EB001061688900B0FBEA
:2058A000F1F06421B0FBF1F000EBC00101EB0010A7EB8000322101EB00106421B0FBF1F0DC
:2058C00000F00F00304421688860BDE8F081000000380140014691F8390021282CD1886816
:2058E000B0F5805F0FD10A6A1088C0F308000B685860086918B9086A801C086209E0086A3D
:20590000401C086205E00B6A581C086218780B685860C88C401E80B2C88458B90868C068F5
:2059200020F080000B68D8600868C06840F040000B68D860002070470220FCE710B505488B
:2059400000F00EF8044800F040F80448F6F77EFD10BD0000C8050020D805002070260020BC
:2059600008B5C26812681268C2F3401262B3C26812685268D1B2C268126812680022B2B9A4
:2059800043788268D1544278521CD2B2427003789A4201DB00224270C278521CD2B2C2707A
:2059A00003789A4203DD0278C2700122027100BF00220092C268126812680092C2681268A7
:2059C0005268009200BF00BF08BDC16809680968C1F3C01139B3C1680968C96801F080017F
:2059E00009B36FF08001C26812681160C17891B1C178491EC17082788168895CC26812683E
:205A000051608178491CC9B28170027891420ADB0021817007E0C1680968C96821F0800183
:205A2000C2681268D160704710B50248F3F7D0FF10BD00002C24002010B54FF4FA71024818
:205A400000F004F810BD0000C80500202DE9F34F83B00398C0780D2873DB00210398FFF70D
:205A6000DEFD01906B490198087001210398FFF7D6FD8146674981F80190019855287DD18A
:205A8000B9F1AA0FFBD102210398FFF7C8FD6149887003210398FFF7C2FD5E49C870042144
:205AA0000398FFF7BCFD06465A490E71112E03D0162E01D00C2E7DD105210398FFF7AFFD1C
:205AC00007465448477107210398FFF7A8FD834606210398FFF7A3FD0BEB00201FFA80F8FF
:205AE0004FEA18204B49887181F8078007210398FFF795FD0446381B02287AD10398C17877
:205B000007F10B0081421DDA43480078012806D1F5F76AF84149086000203F490870F5F779
:205B200063F83E490968411A0498814206D9F5F75BF83A49086001203749087005B0BDE8DC
:205B4000F08F64E001203449087000250FE005F10800C1B20398FFF762FD31494855084692
:205B6000415D05F108002B4A1154681C85B2A542EDDB04F10800C1B2039800E043E0FFF741
:205B80004EFD4FEA006B04F10900C1B20398FFF746FD0BEB004B04F10A00C1B20398FFF78D
:205BA0003EFD0BEB002B04F10B00C1B20398FFF736FD00E022E05844029004F108011548E7
:205BC000EFF7DEFA82460298B0EB0A000CD1144A41463046FFF72AFC07F10B00C1B203989B
:205BE000FFF782FCAAE704E001210398FFF77CFC0DE001210398FFF777FC08E001210398D9
:205C0000FFF772FC03E001210398FFF76DFC00BF94E7000036110020F0010020EC01002062
:205C2000A0100020012806D002282AD003284ED0042873D173E0FE49FE4A13680B60536835
:205C40004B6092688A60FC4A1368CB6053680B6192684A61F94A13688B615368CB61926872
:205C60000A62F74A13684B6253688B629268CA620A46F4490B6813634B68536389689163BD
:205C800073E0EB4AF0490B6813604B685360896891601146ED4A1368CB6053680B619268C0
:205CA0004A61EB4A13688B615368CB6192680A62E84A13684B6253688B629268CA62E64AF8
:205CC00013680B6353684B6392688A634DE0D849E24A13680B6053684B6092688A60E04AB7
:205CE0001368CB6053680B6192684A61DD4A13688B615368CB6192680A620A46DA490B6871
:205D000053624B6893628968D1621146D74A13680B6353684B6392688A6326E024E0C4493A
:205D2000D34A13680B6053684B6092688A60D14A1368CB6053680B6192684A61CE4A1368F6
:205D40008B615368CB6192680A62CC4A13684B6253688B629268CA62C94A13680B63536847
:205D60004B6392688A6300E000BF00BFC549897B78290DDCC349897B502909DBAC490988A1
:205D8000C04A927B5143642291FBF2F1A84A1180BC49097C78290DDCBA49097C502909DBE7
:205DA000A3498989B74A127C5143642291FBF2F19F4A9181B349897C78290DDCB149897C48
:205DC000502909DB9A49098BAE4A927C5143642291FBF2F1964A1183AA49097D78290DDCE9
:205DE000A849097D502909DB9149898CA54A127D5143642291FBF2F18D4A9184A149897DFD
:205E000078290EDC9F49897D50290ADB8849498E9C4A927D5143642291FBF2F18AB284497C
:205E20004A869849C97B5A2905DC8149097A491E7F4A117208E09349C97B6E2904DB7C49C6
:205E4000097A491C7A4A11728E49497C5A2906DC7749097D491ECAB275490A7509E08949F1
:205E6000497C6E2905DB7249097D491CCAB270490A758449C97C5A2908DC6D4991F82010A4
:205E8000491ECAB26A4981F820200BE07D49C97C6E2907DB664991F82010491CCAB264494E
:205EA00081F820207749497D5A2908DC604991F82C10491ECAB25E4981F82C200BE07149DA
:205EC000497D6E2907DB5A4991F82C10491CCAB2574981F82C206B49C97D5A2908DC5449D7
:205EE00091F83810491ECAB2514981F838200BE06449C97D6E2907DB4D4991F83810491C60
:205F0000CAB24B4981F838205F49C97C78290DDC5D49C97C502909DB4549C9885A4AD27C10
:205F20005143642291FBF2F1414AD1805649497D78290EDC5449497D50290ADB3C49498AF3
:205F4000514A527D5143642291FBF2F18AB238494A824D49C97D78290EDC4B49C97D50290B
:205F60000ADB3349C98B484AD27D5143642291FBF2F18AB22E49CA834349497E78290EDC24
:205F80004149497E50290ADB2949498D3E4A527E5143642291FBF2F18AB225494A853A492D
:205FA000C97E78290EDC3849C97E50290ADB2049C98E354AD27E5143642291FBF2F18AB295
:205FC0001B49CA863049897C78290DDC2E49897C502909DB164949892B4A927C514364225E
:205FE00091FBF2F1124A51812749097D78290EDC2549097D50290ADB0D49C98A224A127D8D
:206000005143642291FBF2F18AB20949CA821E49897D78293DDC1C49897D502939DB0449B1
:20602000498C194A927D5143642291FBF2F12DE01C0B0020827801088E7801089A7801080F
:20604000A6780108B2780108BE780108CA780108D6780108E2780108EE780108FA780108B8
:2060600006790108127901081E7901082A79010836790108427901084E7901085A79010890
:2060800066790108E8090020080A00208AB214494A841449097E78290EDC1249097E5029A4
:2060A0000ADB0F49C98D0F4A127E5143642291FBF2F18AB20A49CA850A49897E78290EDC18
:2060C0000849897E50290ADB0549498F054A927E5143642291FBF2F18AB201494A877047EE
:2060E0001C0B0020080A002000BFFEE700B587B00020C1490860C1490880C14908700720CA
:20610000C04908701821C048EDF7E2FC1821BF48EDF7DEFC1821BE48EDF7DAFC1022BD49CC
:20612000BD48EDF7BCFCBD48BD490A680260496841601022BBA1C048EDF7D5FC1022BFA1B0
:20614000BD481030EDF7CFFC2E21BB48203880F83F102022BEA1C748EDF7C5FC00BFC6A25E
:2061600007CA04AB07C3C7A207CA01AB07C39DF81A0030389DF81910303901EB810100EB8E
:206180004100BC4988760322C1A104A8EDF7CDFC18B90120B749C87670E00322BDA104A82C
:2061A000EDF7C3FC18B90220B249C87666E00322B9A104A8EDF7B9FC18B90320AD49C876DE
:2061C0005CE00322B5A104A8EDF7AFFC18B90420A849C87652E00322B1A104A8EDF7A5FCCF
:2061E00018B90520A349C87648E00322ADA104A8EDF79BFC18B906209E49C8763EE003225E
:20620000A9A104A8EDF791FC18B907209949C87634E00322A5A104A8EDF787FC18B9082074
:206220009449C8762AE00322A1A104A8EDF77DFC18B909208F49C87620E003229DA104A8AA
:20624000EDF773FC18B90A208A49C87616E0032299A104A8EDF769FC18B90B208549C8768D
:206260000CE0032295A104A8EDF75FFC18B90C208049C87602E000207E49C8769DF8151027
:2062800030399DF81400202801D1002002E09DF81400303800EB800001EB400075490877EB
:2062A0009DF8051030399DF80400202801D1002002E09DF80400303800EB800001EB40007E
:2062C0006C4948779DF8081030399DF80700202801D1002002E09DF80700303800EB80000D
:2062E00001EB4000634988779DF80B1030399DF80A00202801D1002002E09DF80A003038EC
:2063000000EB800001EB40005A49C87700BF6C48007828B930214848203880F82A102CE041
:2063200067480078012805D131214348203880F82A1022E062480078022805D132213E4853
:20634000203880F82A1018E05D480078032805D133213948203880F82A100EE05848007838
:20636000042805D134213448203880F82A1004E030213148203880F82A10102251A12E48EE
:206380002038EDF7B0FB102253A12B481038EDF7AAFB082255A15848EDF7A5FB082257A146
:2063A00055480830EDF79FFB082257A152481030EDF799FB5748584B0ECB0EC000F0D8F86D
:2063C00000F0B0F85548007B544991F91B100844524989794843C0EB001001034F48C079B8
:2063E00041F2C6125043B1FBF0F04D49888108468089C88107B000BD840100209C0100205E
:20640000E803002088010020C4080020D0090020B8090020D0760108DC0800208901002005
:20642000AC77010854544B5A303130442E2020202020202000000000740800205633723435
:2064400072335F3230323331313138430000000054433031313030302D4D53303030302DF0
:20646000563072302E202020202020202020202000000000940800204465632032372032C3
:206480003032330031343A35363A3336000000004A616E00466562004D6172004170720051
:2064A0004D6179004A756E004A756C0041756700536570004F6374004E6F760044656300B3
:2064C000D00100205047383058582026205053583058582E0000000030303030303030302D
:2064E0003030303030303030000000004D4F54494E4F564100000000780A002057554841D8
:206500004E2E202000000000323032313039303100000000F00A0020E8F7FF1FE809002008
:20652000DC01002010B5302209490A48EDF7B7FA102209490948EDF7B2FA0948094C1ECC19
:206540001EC0102208490948EDF7A9FA10BD000004780108380A002034780108680A002007
:20656000580B00205478010844780108680B002010B50C221AA11E48EDF7B5FA1D480189D5
:206580001D48FEF7D9FE1B4841891C48FEF7D4FE184881891A48FEF7CFFE1A481A490A68AD
:2065A0000260496841604FF4B87018490880202217491848EDF773FA1648007816490870D3
:2065C000202216491648EDF76AFA102215491648EDF765FACC2215491548EDF760FA10BD8F
:2065E00030303030303030303030303000000000FC0A0020C41E0020C4150020DE15002027
:20660000F81500209301002064780108EA030020B4770108E809002091010020D47701085C
:20662000080A0020F4770108280A0020E0760108EC08002088B004460D4631E01948FAF7B7
:2066400044F80020FBF792FEF0F756FC20216846EDF73EFA2046EDF752FA06463246214657
:206660006846EDF71CFA2046EDF749FA694608440DA10A880280897881702046EDF73FFAB3
:2066800069460844C0F803506B464FF620720C214FF4E260FDF7F8FDC820F3F7BFFF00BF82
:2066A000CCE70000F8000020202C200008B52B4988420DD100BF2A49896941F00401284AFE
:2066C00091611146896901F00401009100BF43E0244988420DD100BF2149896941F00801AC
:2066E0001F4A91611146896901F00801009100BF32E01D4988420DD100BF1949896941F048
:206700001001174A91611146896901F01001009100BF21E0154988420DD100BF1049896969
:2067200041F020010E4A91611146896901F02001009100BF10E00E4988420DD100BF084913
:20674000896941F04001064A91611146896901F04001009100BF00BF08BD000000080140FB
:2067600000100240000C014000100140001401400018014070B504460E46A1882068F4F71C
:2067800021FA28B9A07908B9012506E0002504E0A07908B9002500E00125012E04D1207A6B
:2067A00068402840E07102E0207A6840E071257270BD10B50446A18801222068F4F70EFA69
:2067C00010BD00BF704702E008C8121F08C1002AFAD170477047002001E001C1121F002A49
:2067E000FBD1704700F0010181F31388704700000149086070470000F8050020F0B50446E9
:206800000E4619681F683D14A54206DA31440814A04212DD204601040FE0A5420CDD02EB8B
:2068200004473DB2A94202DA2046010405E0891A081410B9002100E020461960F0BD0000F2
:2068400010B50A46437993421EDB1E4B1B685B6923F002031B4C2468636143799B1A4371F5
:20686000184B1B685B6943F00203164C24686361114603790B4499B283788B4202DC837876
:20688000CB1A99B201711BE00E4B1B685B6923F002030C4C24686361417900234371094B16
:2068A0001B685B6943F00203064C246863610379194483788B4202DC8378CB1A99B201719B
:2068C00010BD00002C24002010B502460B46194654799C4209DB14790C44A1B294788C4225
:2068E00004DC94780C1BA1B200E000219468605C10BD00007FB50646002404E0305D184936
:206900000855601CC4B2082CF8DB3823154A02A9304600F093FB00241EE0002504E002A8F3
:2069200000F0B4FA681CC5B20F48005DA842F6DC40230E4A694602A800F080FB002507E0C3
:206940001DF805000A4901EBC4014855681CC5B2082DF5DB601CC4B2102CDEDB7FBD000059
:2069600061030020348001080C8301086C8001086214002001460120064A12688A4206D1DE
:20698000044A1268044B1B685A40521C02B1002070470000B0260020D42600202DE9F04F66
:2069A00087B082460F469046994600250AE0785D3A49495D884203D03846FFF79BFF0725EA
:2069C000681CC5B2082DF2DB4023354A05A9504600F034FB012536E0002405E005A8005D26
:2069E00003A90855601CC4B2082CF7DBB8F1000F04D1681E2B4901EBC00B04E0C5F11000AE
:206A0000284901EBC00B002406E003A9201D085C05A90855601CC4B2042CF6DB01AA05A9A0
:206A2000584600F043F8002409E003A8005D01A9095D484005AA211D5054601CC4B2042C2D
:206A4000F3DB681CC5B2112DC6DB9DF814609DF818008DF814008DF818609DF815609DF8A3
:206A600019008DF815008DF819609DF816609DF81A008DF816008DF81A609DF817609DF870
:206A80001B008DF817008DF81B604023064A494605A800F0D3FA07B0BDE8F08F6103002034
:206AA000747F010862140020B47F0108F0B587B005460E4617464023104A05A9304600F05F
:206AC000BDFA002410E005A8005D295D484000F03F0003A908550A4800EB8410095D405CC8
:206AE00001A90855601CC4B2082CECDB2023054A394601A800F0A2FA07B0F0BDAC800108C3
:206B00000C810108EC8001081CB5F6F76DF8F6F773F8B9490870F4F7A9F8FDF717FFF6F7F2
:206B200097F9FAF769FFFBF709F8FBF771F8FBF7B9F8FAF747FFFAF7F1FDFAF7BDFEFAF7C8
:206B400013FFFBF7F9F8FCF785F9EDF7BFFC1420F3F764FDA948F5F78FF8FFF7C7FAFAF7A5
:206B6000CDFFFAF789FBA648F0F776FA6921A448EEF7E6FCA3490870F0F714FCA048F0F728
:206B80001BFAF0F761FCA0490870084601789C48FDF738FB9D499E48F0F734FCF9F7B6FCE4
:206BA000F1F75CF900209B49087024E19A480078401C9949087008460078C82801DD002053
:206BC000087096480088F1F7CBFBFBF77BF9EEF75BFCFEF731FF924A5178924AD07A924BBA
:206BE000924A1278F8F79CF9FAF754FD8D48807EAA2841D18E48007BC0B18D48B0F9020070
:206C00000B2190FBF1F084B289498648007B854A92F91B20104480B2CDE900018148C379B4
:206C2000827984492046FDF721FC46E08048B0F902000B2190FBF1F07D49897A884206DD6E
:206C40007B48B0F902000B2190FBF1F001E07848807A84B276497348007B724A92F91B20E6
:206C6000104480B2CDE900016E48C379827971492046FDF7FBFB20E06A48807EEE280AD13F
:206C80006848007B6749C97E0844C2B268496948FDF730FC11E06348007B6249C97E08443B
:206CA000C2B26048007E08B9012001E05D48007E03465F495F48FDF79DFC5F48F1F732FB73
:206CC0005E48EDF7FBFE00BF5D48007818BB5D48007828B1F3F788FF42F21071884229D99A
:206CE0005348C0880A2190FBF1F084B2564880884C4A0090127B4B4D95F91B502A4490B24A
:206D0000524A137B4F4A11782246FBF773FD01204B4908700EE0464C23894B4C627AA18868
:206D2000444CE068FBF740FC494A11783E4A1078FBF796FD00BFFAF78FF8F8F7F7F94548F9
:206D4000FAF7F6F9FAF70EFC394B9A7D1989987AF7F706FF404908703D48807910B93F4847
:206D6000F0F746FB3A48807930B93D493D48F0F7E1FB3D48FBF708FF3C480078E8B93C481A
:206D800000683C4908603A48406848603848806888603748C068C8602E48001F4068086107
:206DA00028221B480830FDF775F9042232A11848FDF770F901202D490870F8F723FBF9F7CA
:206DC000E7FC2F480068FAF70DFA18480078FAF731FA16480078FAF7D9F92A48FAF776FA99
:206DE000FDF716FBF1F79AF8FCF7AEFDFBF7B2FF2548F3F727FFD9E6D0010020441E002024
:206E000018040020D801002010040020FFF7010800F401085C0000205A000020D401002022
:206E200089010020E8090020D2000020D000002014080020BC030020290400202804002001
:206E40005B000020C0010020B4080020280A0020D60000203C0A0020E60000201104002011
:206E600069030020E414002092010020D7010020580B0020C80A0020464C41470000000034
:206E800084010020080B0020F00700200CB5002104E0425C0DF801204A1CD1B20829F8DB8C
:206EA000002112E0425C5206120E425406290ADA4A1C1DF8022002F08002802A03D1425CD3
:206EC00042F0010242544A1CD1B20729EADB9DF8002002F0800222B1C27842F01002C2705D
:206EE00003E0C27822F01002C2709DF8032002F0080222B1827942F00102827103E0827997
:206F000022F0010282710CBD2DE9F04106460F46EDF734F904000D4618BF0120284320F0DD
:206F20000040C0F17F6000F1E040C00F0ED0301C18BF0120384320F00040C0F17F6000F133
:206F4000E040C00F04BF0120FFF752FC20462946BDE8F08130B502460023002952D0334819
:206F6000007890B13248334C247830F81400324C2468201A304C20602046006810442060A5
:206F80002B482C4C247820F814202A480078401C284C2070204600781E280FDB0020207016
:206FA0002248007818B90120204C207006E01F480078012802D102201C4C20701B4800784B
:206FC000022806D11C4800681E24B0FBF4F083B211E01648007801280CD11648007808B97A
:206FE000134608E014480068124C2478B0FBF4F083B200E01346052093FBF0F0904212DD41
:20700000134610E0002005E00024094D25F81040441CE0B21E28F7DB0020064C2070064CDD
:207020002060024C2070184630BD0000B80300204C150020B0030020B40300202DE9F0415A
:2070400004461D46154E002000BF4FF000080746401C01F807800828F7DB002000BF12F8E6
:20706000013B04EBE3073F7803F0070C16F80CC007EA0C0767B101EBE0073F7800F0070CBB
:2070800016F80CC047EA0C0701EBE00C8CF80070471C3846AF42E2DBBDE8F0811C830108B9
:2070A000000000000000000001020304060708090000000001020304204E00040300000425
:2070C00000000004000000009CFFFFFFFF7F0000000000FE00FCFF0100000000204E000429
:2070E0000300000400000004000000000080FFFFFF7F0000000000FE00FCFF01000000008F
:20710000400000040300000400000004000000000000FCFF00000000000000F00000000035
:2071200000000000307500012C0100040000000400000000CCF7FFFF000000000030DFFFA5
:207140000000000000000000001000040100000400000004000000009CFFFFFF1A0400005B
:207160000070FEFF0068100000000000307500042C0100040000000400000000E6FBFFFF6D
:20718000000000000098EFFF0000000000000000204E0004030000040000000400000000EC
:2071A0009CFFFFFFFF7F0000000000FE00FCFF0100000000204E0004030000040000000441
:2071C000000000000080FFFFFF7F0000000000FE00FCFF010000000040000004030000046E
:2071E00000000004000000000000FCFF00000000000000F0000000000000000030750001FA
:207200002C0100040000000400000000CCF7FFFF000000000030DFFF00000000000000006A
:20722000001000040100000400000004000000009CFFFFFF1A0400000070FEFF0068100095
:2072400000000000307500042C0100040000000400000000E6FBFFFF000000000098EFFFEB
:207260000000000000000000204E00040300000400000004000000009CFFFFFFFF7F00007A
:20728000000000FE00FCFF0100000000204E00040300000400000004000000000080FFFFF9
:2072A000FF7F0000000000FE00FCFF01000000004000000403000004000000040000000007
:2072C0000000FCFF00000000000000F00000000000000000307500012C01000400000004E8
:2072E00000000000CCF7FFFF000000000030DFFF00000000000000000010000401000004A6
:2073000000000004000000009CFFFFFF1A0400000070FEFF00681000000000003075000424
:207320002C0100040000000400000000E6FBFFFF000000000098EFFF0000000000000000B3
:20734000204E00040300000400000004000000009CFFFFFFFF7F0000000000FE00FCFF019F
:2073600000000000204E00040300000400000004000000000080FFFFFF7F0000000000FE96
:2073800000FCFF0100000000400000040300000400000004000000000000FCFF00000000A7
:2073A000000000F00000000000000000307500012C0100040000000400000000CCF7FFFF41
:2073C000000000000030DFFF00000000000000000010000401000004000000040000000082
:2073E0009CFFFFFF1A0400000070FEFF0068100000000000307500042C0100040000000413
:2074000000000000E6FBFFFF000000000098EFFF0000000000000000657F367E107D807CE6
:20742000657B527A467940784177C476CE75DF74F47310739F72C271EA701770486F7D6EF0
:207440001A6E566D966CDA6B216B6D6A136A6469B8680F68696718677666D8653D65A46444
:207460000E64C4633263A26215628A614561BE603960B55F345FB55E765EFA5D805D085DF4
:20748000915C1C5CE25B705BFF5A905A235AED5981591859AF584858E357B1574D57EB5660
:2074A0008A562B56CC550000C90092015B022403ED03B6047F0548061107D907A2086A09D9
:2074C000330AFB0AC40B8C0C540D1C0EE30EAB0F72103A110112C8128F1355141C15E215E0
:2074E000A8166E173318F918BE19821A471B0B1CCF1C931D571E1A1FDD1F9F206121232226
:20750000E522A62367242825E825A82667272628E528A329612A1F2BDC2B992C552D112ED1
:20752000CC2E872F4130FB30B5316E322633DF3396344D350436BA366F372438D9388C39C0
:20754000403AF23AA53B563C073DB83D683E173FC53F73402141CE417A422543D0437A44C1
:207560002445CD4575461C47C34769480F49B449584AFB4A9D4B3F4CE04C814D204EBF4E93
:207580005D4FFB4F97503351CE51685202539B533254C9546055F5558A561D57B0574258D7
:2075A000D3586459F359825A0F5B9C5B285CB35C3E5DC75D4F5ED75E5D5FE35F6860EB6015
:2075C0006E61F0617162F1627063EE636C64E8646365DD655666CF664667BC673268A668B2
:2075E00019698B69FD696D6ADC6A4A6BB76B236C8E6CF86C616DC96D306E966EFB6E5E6FF2
:20760000C16F22708370E27040719D71F9715472AE7207735E73B5730A745F74B2740475F1
:207620005575A575F37541768D76D87622776B77B377FA773F788478C77809794A798979A7
:20764000C879057A417A7C7AB67AEE7A267B5C7B917BC57BF87B297C597C887CB67CE37CDB
:207660000E7D397D627D897DB07DD57DFA7D1D7E3E7E5F7E7E7E9C7EB97ED57EEF7E097F25
:20768000217F377F4D7F617F747F867F977FA67FB47FC17FCD7FD87FE17FE97FF07FF57FF4
:2076A000F97FFD7FFE7F00000500000000000000050000000000000005000000000000004A
:2076C00005000000000000000500000000000000A0282400000000000000000000000000B4
:2076E000983A38100810F90FEE0FE60FE00FDB0FD70FD30FCF0FCB0FC70FC20FBC0FB50FCF
:20770000AD0FA40F9B0F900F850F7A0F6F0F640F5A0F4F0F460F3D0F340F2B0F230F1B0F62
:20772000120F0A0F030FFA0EF20EE90EE10ED70ECE0EC40EB90EAF0EA40E990E8F0E840E70
:207740007A0E700E670E5D0E550E4C0E440E3D0E350E2E0E270E210E1B0E150E0F0E090E86
:20776000030EFE0DF80DF40DEE0DE90DE40DDF0DDA0DD40DCE0DC80DC30DBC0DB60DAF0D89
:20778000A70D9F0D970D8E0D850D7B0D700D640D570D490D3B0D2E0D250D1C0D120D080D76
:2077A000FD0CF10CE00CC70C930C1C0C045500000000000055026400190310101187A5555B
:2077C000DB046464646464646464646401025500B80B3C870000000055020C0C96004B00B4
:2077E0009600000000006464646464646464646400000000FA000807C8000A000A0080BBEB
:20780000300000000100000000000000000000000000000000000000000000000000000037
:207820000000000000004141000000004141414100000000000000000000000000000000C2
:20784000000000006400A000BE000E01B400000000000000000000000000000000000000A3
:207860000000000041564F4E49544F4D7401E8025C04D1054507B9082D0AA20B160D8A0E5A
:20788000FF0F880100006400200302010002120300006400E8030201AE021D05BC0264006A
:2078A000140503016603AC07480364003408050100040000CC016400340804010004C4015F
:2078C00000006400480302010002BA0300006400B0040201AE02E005BC0264003606030125
